:020000040800F2
:1000000000000120896A0008EF330008F13300087E
:10001000F3330008F5330008F73300080000000050
:10002000000000000000000000000000F93300089C
:10003000FB33000800000000FD330008FF33000818
:10004000D96A0008D96A000801340008D96A000892
:10005000D96A0008D96A00080D3400081D34000868
:10006000D96A00082D340008D96A00083534000820
:10007000413400084D340008D96A0008D96A0008E4
:10008000593400085D340008D96A0008D96A0008AC
:1000900000000000D96A000869340008D96A000825
:1000A000D96A0008D96A0008D96A0008D96A000824
:1000B000D96A0008D96A0008D96A0008D96A000814
:1000C000D96A0008D96A00086D340008D96A0008A6
:1000D000D96A000879340008D96A0008D96A00088A
:1000E000D96A0008D96A000885340008D96A00086E
:1000F000D96A00080000000000000000D96A00086A
:10010000D96A0008D96A000891340008D96A000841
:10011000D96A0008D96A0008D96A0008D96A0008B3
:10012000D96A0008D96A0008D96A0008D96A0008A3
:08013000D96A0008D96A000831
:1001400010B5054C237833B9044B13B10448AFF311
:1001500000800123237010BDA005002000000000D6
:10016000EC1F030808B5034B1BB103490348AFF369
:10017000008008BD00000000A4050020EC1F03085B
:1001800014214160704714207047406A7047000096
:1001900081010008870100088B010008A101000807
:1001A00010B5044604F1100000F05CFCC4F8F8003F
:1001B0000148C4F87C0110BD90010008F8B5E6B014
:1001C00004460D4616461F460A4906A800F0CAFE18
:1001D00070996F9A05910492009733466E996D9AC3
:1001E000039102922A466C990191214600F060F831
:1001F00067B0F0BD9C010008F8B5E6B004460D46B6
:1002000016461F46094906A800F0ACFE6F996E9A83
:100210000491039200976D996C9A02910192334672
:100220002A46214600F087F867B0F0BD9C0100081F
:1002300038B500281CBF01680029184A23D1184B83
:100240001C684FF6F0710C404CF24025AC421FBFC9
:100250001B6819404CF27024A14212D1114D29683B
:1002600079B911490B68C3F30B03B3F58A6F1FBF4C
:100270000968C1F30B0140F28343994204BF012195
:10028000117028B905E0094B994204BF0121117092
:100290004068BDE8324002F073BC00BFBC050020DE
:1002A00000ED00E0002004E00010005C0000374892
:1002B0002DE9F04104460D46216816464A681F465E
:1002C00090478046B8F5403F2ED122680A9993683E
:1002D000204698478046B8F5403F25D12368089AC4
:1002E0000799D3F80CC02046E0478046B8F5403F58
:1002F0001AD12368069A39461F692046B8478046B6
:10030000B8F5403F10D1236829465D693246204642
:10031000A8478046B8F5403F06D123680B9A099953
:100320009D692046A847804621680A682046904774
:100330004046BDE8F0812DE9F04104460D462168B4
:1003400016464A681F4690478046B8F5403F2ED172
:1003500022680A999368204698478046B8F5403F3E
:1003600025D12368089A0799D3F80CC02046E047A6
:100370008046B8F5403F1AD12368069A39461F696E
:100380002046B8478046B8F5403F10D1236829463B
:100390005D6932462046A8478046B8F5403F06D101
:1003A00023680999DD6900222046A8478046216814
:1003B0000A68204690474046BDE8F0814FF440303F
:1003C00070470000F0B50C4685B0114600281A466B
:1003D0001CBF0568002D0B4B11D082B104B971B957
:1003E0000D9860B10F9E0E9F0A9B02900496039792
:1003F0000B980C9E009001962046A847034618468D
:1004000005B0F0BD020003002DE9F04F0646D0B064
:100410000868F56DD6F860E0726EB76EF36E00BADC
:1004200000906C46486800BA60600DF1400888682A
:1004300000BAA060C86800BAE060086900BA20612C
:10044000486900BA6061886900BAA061C86900BAE9
:10045000E061086A00BA2062486A00BA6062886A8D
:1004600000BAA062C86A00BAE062086B00BA2063F2
:10047000486B00BA6063886B00BAA063C86B00BAAF
:10048000E063402058F80C1C58F820CC58F838ACE1
:100490008CEA010158F840CC8AEA01018CEA010992
:1004A0004FEAF979401E48F8049BEBD187EA020035
:1004B00000EA0E00784010EBF5610098DFF824C4E4
:1004C00041186144C81882EABE032B404FEAF0612C
:1004D00053405918636859186144CF194FEAB5035E
:1004E00083EABE01014081EABE0111EBF765A16814
:1004F0004D196544A91883EAB0023A404FEAF16504
:100500005A405519E26855194FEAB70282EAB00716
:1005100065440F4005EBBE0E97EAB00717EBFE658A
:1005200027697D194FEAB10782EA0701654401EAAC
:100530000E01EB18514011EBF36561694D194FEA5B
:10054000BE0187EA010E65440EEA030E15EBB0000A
:100550008EEA070E0EEBF065D4F818E0754465449A
:10056000AA1881EAB30505404FEAF26E4D40AE4449
:10057000E569AE44E64477444FEAB00080EAB30E42
:100580000EEA020E8EEAB30E0EEBF765D4F820E009
:1005900075446544691880EAB2053D404FEAF16E42
:1005A0004540AE44656AAE44E6440EEBB3034FEA01
:1005B000B70787EAB20E0EEA010E8EEAB20E0EEB14
:1005C000F365D4F828E075446544281887EAB10536
:1005D0001D404FEAF06E7D40AE44E56AAE44E6440D
:1005E0000EEBB2024FEAB30383EAB10E0EEA000E3D
:1005F0008EEAB10E0EEBF265D4F830E07544654436
:10060000EF1983EAB00515404FEAF76E5D40AE443E
:10061000656BAE44E6440EEBB1014FEAB20282EAEA
:10062000B00E0EEA070E8EEAB00E0EEBF165D4F8AE
:1006300038E075446544EB1882EAB7050D404FEA8F
:10064000F36E5540AE44E56BAE44E6440EEBB000AD
:100650004FEAB10181EAB70E0EEA030E8EEAB70E39
:100660000EEBF065D4F840E07544654481EAB30EC2
:10067000AA180EEA000E4FEAF2658EEA010E7544E2
:10068000DDF844E04FEAB000754480EAB30E6544FB
:100690000EEA020E15EBB7078EEAB30E0EEBF76506
:1006A000DDF848E04FEAB202754480EA020E654484
:1006B0000EEA070E69188EEA000E0EEBF165DDF802
:1006C0004CE07544654405EBB3034FEAB70E1427BD
:1006D0000DF1500CDFF810528EEA010B82EA0B0B81
:1006E0000BEBF36A5CF804BBDA44AA44504483EA97
:1006F000B10B4FEAF06A8EEA0B0BDA445CF804BBEC
:10070000DA44AA44524480EAB30B4FEAF26A8BEA15
:10071000B10BDA445CF804BBDA444FEAB000AA44F7
:1007200080EA020BD6448BEAB30B0BEBFE6A5CF853
:1007300004BBDA444FEAB202AA4482EA0E0B0AEB87
:10074000B10180EA0B0B0BEBF16A5CF804BBDA44F5
:100750007F1DAA44282F0AEBB3034FEABE0EBBD37A
:100760003C2F61D3502F4DD204EB870CC7F15407B7
:100770005E4CA7FB04A504465D4FA8088EEA010A5B
:1007800082EA0A0A5CF804BB0AEBF3655D447D1952
:100790002C1983EAB10A4FEAF4658EEA0A0A554435
:1007A0005CF804AB5CF804BB55447D19AA1884EAD4
:1007B000B30A4FEAF2658AEAB10A55445D444FEA4A
:1007C000B4047D1984EA020AAE448AEAB30A0AEB49
:1007D000FE655CF804AB55444FEAB2027D1982EA2B
:1007E0000E0A15EBB10184EA0A0A5CF804BB0AEBB5
:1007F000F1655D447D1915EBB303401E4FEABE0E53
:10080000BCD12046F46D1B19F365336EC9183166EF
:10081000716E71447166B36ED218B266F16E401893
:10082000F06650B0BDE8F08F4EEA010B0EEA010A07
:100830000BEA020B4BEA0A0A0AEBF36554F827A00D
:10084000DFF8B0C0554443EAB10B654403EAB10A8E
:100850000BEA0E0B28184BEA0A0A7F1C0AEBF0651C
:1008600054F827A0554440EAB30B654400EAB30AA4
:100870000BEAB10BAA184BEA0A0A7F1C0AEBF265D5
:1008800054F827A055444FEAB00040EA020B6544F3
:1008900000EA020A0BEAB30BAE444BEA0A0A7F1CD9
:1008A0000AEBFE6554F827A055444FEAB20242EA2B
:1008B0000E0B654402EA0E0A0BEA000B15EBB101C0
:1008C0004BEA0A0A7F1C0AEBF16554F827A055444D
:1008D0007F1C65443C2F05EBB3034FEABE0EA3D348
:1008E00040E700BF9979825AA1EBD96ECDCCCCCC30
:1008F000D6C162CADCBC1B8F00B581B00168074A53
:10090000914200D110B9064801B000BD7C212EF003
:100910001CF94FF4003001B000BD00BF040A00080C
:10092000030002002DE9F0410B4A92E8F85188B02B
:10093000694681E8F8510268084B9A4200D118B91B
:10094000074808B0BDE8F0811422083000F04FFBE2
:1009500008B0BDE8F08100BFE4090008040A0008FF
:1009600003000200152904D20268044B9A4200D108
:1009700008B903487047083000F048BB040A000873
:100980000300020010B481B013460268074CA24273
:1009900000D118B901B010BC0548704701B000F192
:1009A000240210BC083000F035BB00BF040A000868
:1009B0000300020010B481B013460268074CA24243
:1009C00000D118B901B010BC054870470A4601B003
:1009D00000F1240110BC083000F070BB040A0008CC
:1009E000030002000123456789ABCDEFFEDCBA9816
:1009F00076543210F0E1D2C3000000000000000085
:100A000000000000F9080008250900086509000831
:100A100085090008B509000809040008810F0008CD
:100A2000CD0F0008890F0008F0B5A3B004460B48AD
:100A300002900D4616461F46094B0822402104A885
:100A400000F0D1FA28980190009733462A462146B3
:100A500002A800F01BF823B0F0BD00BF040A000894
:100A6000180A000810B5040008BF002408D0054883
:100A7000054B20600822402104F1080000F0B3FA81
:100A8000204610BD040A0008180A00082DE9F041AC
:100A900004460E46216817464A681D469047804620
:100AA000B8F5003F19D12268069993682046984707
:100AB0008046B8F5003F10D123683146DE683A46DB
:100AC0002046B0478046B8F5003F06D12368079A14
:100AD00029461D692046A847804621680A682046A5
:100AE00090474046BDE8F08110B500F033FA4FF46E
:100AF000403400280EBF034C4FF4C0712EF025F88F
:100B0000204610BD0200030010B5044600F022FA92
:100B100008B9054810BD0021A160D0F87C211168FA
:100B200088474FF4403010BD0200030070B5044602
:100B30000D4600F00FFA064E40B1D0F87C01416836
:100B40008847A84224BF65604FF44036304670BDE8
:100B5000020003002DE9FF4715000C4600D02CB120
:100B6000064600F0F7F95FEA000801D16448C3E0E7
:100B7000D8F8F80001684A689047B0F5003F17D1EF
:100B8000D8F87C118A68404690478146B9F1810FB8
:100B900080F09E80A94508F1FC0A17D2D8F8F80029
:100BA0000368D3F80CC02A462146E047B0F5003F61
:100BB00040F08E80D8F8F8000368D3F810C06A4679
:100BC0005146E047B0F5003F76D10AE0002004E04E
:100BD000215C0AF800100098401C00900098A84280
:100BE000F6D34FF0000C4749474A484B01AC0098F8
:100BF000844558D2D3E9007001ADC5E90070107882
:100C000000281ABF042086464FF0000E085854F8FA
:100C10000E5028443E4D05600127D0F800E0876063
:100C2000019D4F681AF80C007D408EEA050585F09D
:100C3000040E65680F687D4085F0FC05754485F0FD
:100C4000A30568400AF80C000CF1010CCFE7D3E9CA
:100C5000004501A8C0E9004510782E4D002814BFBA
:100C60004FF0040E4FF0000E01A8744651F80EE04C
:100C70000459A6440127CEF80050DEF80040CEF813
:100C800008704D68019F40687D406C400D68684069
:100C900084F0040480F0FC00041984F057040AF87E
:100CA0000C400CF1010CCC45D1D3D8F8F800016808
:100CB0004A689047B0F5003F0AD1D8F8F8000368B9
:100CC000D3F80C804A465146C047B0F5003F01D0EA
:100CD000114811E0002006E05AF8201081F06A3136
:100CE0004AF82010401CB0EB990FF5D3B06840F0E3
:100CF0000100B0604FF4403004B0BDE8F08700BFA1
:100D00000200030034610308BC0500202C0F00081A
:100D1000ADBE4ED70DBE75A10100030038B50C461F
:100D2000017A1546CA0702D500F014F908B9084837
:100D300032BDD0F8F80003682146DC682A46A04797
:100D4000B0F5003F01D0034832BD4FF4403032BD12
:100D500002000300010003002DE9F84191B00546AF
:100D60000E461746402101A82DF0EFFE297AC8074C
:100D700004D5284600F0EEF8040002D1DFF8A48084
:100D80004BE0D4F8F800DFF8A0800368D3F810C077
:100D90006A4601A9E047B0F5003F3ED1D4F8F8001B
:100DA00001684A689047B0F5003F36D1D4F87C110D
:100DB0008A6820469047D4F8F830024618461B68E7
:100DC000D3F80CC004F1FC01E047B0F5003F24D19A
:100DD000D4F87C0141688847D4F8F83002461846B8
:100DE0001B68D3F80CC001A9E047B0F5003F14D14F
:100DF000D4F8F8000268696893689847B0F5003F36
:100E00000BD1D4F8F80003681C693A463146A04774
:100E1000B0F5003F08BF4FF44038404612B0BDE87F
:100E2000F08100BF02000300010003002DE9F8413A
:100E3000A5B0074688461646402115A82DF085FE28
:100E400000220492402105A82DF07FFE387AC107C8
:100E50005ED5384600F07EF8050059D0D5F8F80088
:100E60002D4C0368D3F810C06A4605A9E047B0F5D9
:100E7000003F3CD1D5F8F80001684A689047B0F5CA
:100E8000003F34D1D5F87C118A6828469047D5F8C0
:100E9000F830024618461B68D3F80CC005F1FC0177
:100EA000E047B0F5003F22D1D5F87C014168884782
:100EB000D5F8F830024618461B68D3F80CC005A9CF
:100EC000E047B0F5003F12D1D5F8F8000268796824
:100ED00093689847B0F5003F09D1D5F8F80003684A
:100EE0001D6904AA15A9A847B0F5003F01D0204606
:100EF0000FE00A4B0A490B4A0396029101924046C1
:100F00001C68049B009415AA796800F0E5F900E0DC
:100F1000054826B0BDE8F081010003003C610308EC
:100F2000936E030026C703000200030004B0010112
:100F300000170145E90A0008090B00082D0B0008FD
:100F4000BD030008550B00081D0D0008590D0008D1
:100F50002D0E00080168024A914218BF0020704718
:100F6000340F000810B5040008BF002404D0034863
:100F70002060204609688847204610BD340F0008CD
:100F800020225C302DF0DDBDF0B58468A30800227E
:100F900004F0030407E000F15C0555F8226035BA5F
:100FA00041F82250521C9A42F5D300220BE000F186
:100FB0005C0502EB830755F82360D500C5F11805E1
:100FC000EE40CE55521CA242F1D3F0BD30B5C468FC
:100FD00003690022E31AD5188C5C0544521C082AC8
:100FE0002C77F8D330BD0360C1600261704738B51B
:100FF000044615460022626023685A689047002024
:101000006061A061A5604FF4003032BD81604FF493
:10101000003070472DE9F84304462079D4F80C805D
:10102000450748BF244845D466691D46A8F101001C
:1010300000EAD60306EBC506B6EBC50F666102D221
:10104000A669761CA6611746A66906EB5576A661C9
:101050000E46E918884225D2A8EB03094A463146D4
:10106000F8182DF06EFD2268136839460FE04246ED
:1010700038462DF066FD23681A68394620469047A9
:1010800007E0311811F00300F1D1226813682046FF
:101090009847484600EB0809A9F10101A942F0D39D
:1010A000002300E000202A1A3118F8182DF049FD1D
:1010B0004FF40030BDE8F283040002002DE9FC4F3C
:1010C000024685B0D0681369DFF86CC1DFF86C8127
:1010D000A0EB030A506840F004005060002703A80A
:1010E00002900DF10C0ED8E9003403A8544DC0E96C
:1010F00000342878534D00280CBF00230423994660
:101100005CF803305EF80940234401261D601C682A
:101110009E60DCF80430039DDCF80090DEF804608B
:101120005D406540484C654089EA0606474C66408C
:101130007519474C6540D8E9006B03AC0028C4E939
:10114000006B0EBF002404200424029E5CF8000003
:10115000345920183F4C04600126046886600398C7
:10116000029E43406340384C7068634089EA000047
:10117000364C6040034438484340280018BF0120E3
:101180005B1E9B41042F2CBFC0B2D80F02F1140389
:1011900053F8200007F00303C3F10303DB00D8403A
:1011A0000DF807007F1C082F9DD315460C466A6971
:1011B000AB69E868D20842EA4372401E00EA0207BF
:1011C000002302409B420AD8524508D28020E055B5
:1011D0007F1C574516D2AAEB0701E01910E08020CA
:1011E000E05500E0E355E8687F1C8742FAD32A689F
:1011F000136828469847BAF1000F03D0514620469D
:101200002DF0A3FC2A68069E059F93686946284630
:1012100098472A68D2F8009021462846C8472B688C
:10122000DA683946284690470EB1A86830604FF416
:10123000003007B0BDE8F08F346103085C1200088D
:10124000BC0500205FC5109304850012FC68017A7C
:10125000C0F524FF24AF33D426AF698B04B001015D
:1012600000170145F8B501240094002300240DE087
:10127000009D065D0F5D7E40F643761CF60F86F0FE
:10128000010635400095641C009DEB189442EFD395
:101290001846F2BDF8B5002301240094002A11E09D
:1012A000009C85188F1815F8016C17F8015C6E40CA
:1012B000F643761CF60F86F0010634400094009C3D
:1012C000E318521EECD11846F2BD0000651200086A
:1012D00095120008010000002DE9F84F1D46DDF8C9
:1012E00028900B9F0D9C4FF0FF3300930E469246C3
:1012F000D9F800B0804632465146D847834664B399
:10130000D9F8043032465146404698476FEA0B02FE
:10131000521C42EA0B0200996FEAD2735B1C19401F
:10132000C2430091521C024300996FEAD2735B1CC6
:101330001940009186F05531484087EA000181F05C
:101340005531216080F05531C943491C0843009A4A
:101350006FEAD070401C82430092D9F8080001283F
:1013600009D17540E943491C0D4300986FEAD572D5
:10137000521C90430AE0F11C85EA9102D243521CB0
:10138000154300986FEAD5735B1C984386F0AA3624
:10139000009086EA0B0686F0AA33F243DB430C98F2
:1013A000C2F3C0725B1C42EAD3720099D243521C52
:1013B00091430091774000998843009987F0AA37BC
:1013C0000F403843BDE8F28F00000000000000002D
:1013D00001F0FF01102A2BDB10F0070F08D010F8E6
:1013E000013B013A8B422DD010F0070F42B3F6D1EA
:1013F000F0B441EA012141EA014122F007047FF003
:1014000000070023F0E80256083C85EA010586EA59
:10141000010685FA47F5A3FA87F586FA47F6A5FA95
:1014200087F68EB9EED1F0BC01F0FF0102F00702A1
:1014300032B110F8013B013A83EA010313B1F8D14C
:101440000020704701387047002D06BF354603382D
:10145000073815F0010F07D1013015F4807F02BF66
:10146000013015F4C03F0130F0BC0138704700BFB7
:10147000034613F8012B002AFBD1181A01387047D4
:1014800081F0004102E000BF83F0004330B54FEA35
:1014900041044FEA430594EA050F08BF90EA020FA2
:1014A0001FBF54EA000C55EA020C7FEA645C7FEA35
:1014B000655C00F0E2804FEA5454D4EB5555B8BF58
:1014C0006D420CDD2C4480EA020281EA030382EAC9
:1014D000000083EA010180EA020281EA0303362D5B
:1014E00088BF30BD11F0004F4FEA01314FF4801C2E
:1014F0004CEA113102D0404261EB410113F0004F40
:101500004FEA03334CEA133302D0524263EB4303F6
:1015100094EA050F00F0A780A4F10104D5F1200E94
:101520000DDB02FA0EFC22FA05F2801841F10001EF
:1015300003FA0EF2801843FA05F359410EE0A5F1C3
:1015400020050EF1200E012A03FA0EFC28BF4CF0F4
:10155000020C43FA05F3C01851EBE37101F00045AA
:1015600007D54FF0000EDCF1000C7EEB00006EEBB7
:101570000101B1F5801F1BD3B1F5001F0CD3490841
:101580005FEA30004FEA3C0C04F101044FEA445298
:1015900012F5800F80F09A80BCF1004F08BF5FEA1F
:1015A000500C50F1000041EB045141EA050130BDFF
:1015B0005FEA4C0C404141EB0101013C28BFB1F511
:1015C000801FE9D291F0000F04BF01460020B1FA5C
:1015D00081F308BF2033A3F10B03B3F120020CDA2F
:1015E0000C3208DD02F1140CC2F10C0201FA0CF00D
:1015F00021FA02F10CE002F11402D8BFC2F1200C72
:1016000001FA02F120FA0CFCDCBF41EA0C01904027
:10161000E41AA2BF01EB0451294330BD6FEA040470
:101620001F3C1CDA0C340EDC04F11404C4F120025B
:1016300020FA04F001FA02F340EA030021FA04F36D
:1016400045EA030130BDC4F10C04C4F1200220FAC4
:1016500002F001FA04F340EA0300294630BD21FA02
:1016600004F0294630BD94F0000F83F4801306BFC8
:1016700081F480110134013D4EE77FEA645C18BFBC
:101680007FEA655C29D094EA050F08BF90EA020F53
:1016900005D054EA000C04BF1946104630BD91EA4B
:1016A000030F1EBF0021002030BD5FEA545C05D14E
:1016B0004000494128BF41F0004130BD14F580048D
:1016C0003CBF01F5801130BD01F0004545F0FE4101
:1016D00041F470014FF0000030BD7FEA645C1ABF36
:1016E000194610467FEA655C1CBF0B46024650EA6D
:1016F000013406BF52EA033591EA030F41F4002199
:1017000030BD00BF90F0000F04BF0021704730B51E
:101710004FF4806404F132044FF000054FF00001F3
:1017200050E700BF90F0000F04BF0021704730B5B4
:101730004FF4806404F1320410F0004548BF404289
:101740004FF000013EE700BF42004FEAE2014FEADE
:1017500031014FEA02701FBF12F07F4393F07F4FB9
:1017600081F06051704732F07F4208BF704793F0BC
:101770007F4F04BF41F40021704730B54FF46074CF
:1017800001F0004521F000411CE700BF50EA0102D2
:1017900008BF704730B54FF000050AE050EA01027B
:1017A00008BF704730B511F0004502D5404261EBEB
:1017B00041014FF4806404F132045FEA915C3FF42C
:1017C000D8AE4FF003025FEADC0C18BF03325FEAC9
:1017D000DC0C18BF033202EBDC02C2F1200300FA7A
:1017E00003FC20FA02F001FA03FE40EA0E0021FA9F
:1017F00002F11444BDE600BF70B54FF0FF0C4CF48D
:10180000E06C1CEA11541DBF1CEA135594EA0C0F3E
:1018100095EA0C0F00F0DEF82C4481EA030621EA79
:101820004C5123EA4C5350EA013518BF52EA0335B4
:1018300041F4801143F4801338D0A0FB02CE4FF066
:101840000005E1FB02E506F00042E0FB03E54FF096
:101850000006E1FB03569CF0000F18BF4EF0010E8E
:10186000A4F1FF04B6F5007F64F5407404D25FEA8A
:101870004E0E6D4146EB060642EAC62141EA55513D
:101880004FEAC52040EA5E504FEACE2EB4F1FD0C7F
:1018900088BFBCF5E06F1ED8BEF1004F08BF5FEAFD
:1018A000500E50F1000041EB045170BD06F00046AF
:1018B00046EA010140EA020081EA0301B4EB5C045C
:1018C000C2BFD4EB0C0541EA045170BD41F4801154
:1018D0004FF0000E013C00F3AB8014F1360FDEBF79
:1018E000002001F0004170BDC4F10004203C35DA55
:1018F0000C341BDC04F11404C4F1200500FA05F3D8
:1019000020FA04F001FA05F240EA020001F0004278
:1019100021F0004110EBD37021FA04F642EB0601EE
:101920005EEA430E08BF20EAD37070BDC4F10C0418
:10193000C4F1200500FA04F320FA05F001FA04F2DC
:1019400040EA020001F0004110EBD37041F10001C8
:101950005EEA430E08BF20EAD37070BDC4F12005D3
:1019600000FA05F24EEA020E20FA04F301FA05F23B
:1019700043EA020321FA04F001F0004121FA04F2E3
:1019800020EA020000EBD3705EEA430E08BF20EAB3
:10199000D37070BD94F0000F0FD101F000464000ED
:1019A00041EB010111F4801F08BF013CF7D041EA6F
:1019B000060195F0000F18BF704703F00046520073
:1019C00043EB030313F4801F08BF013DF7D043EA44
:1019D0000603704794EA0C0F0CEA135518BF95EAFA
:1019E0000C0F0CD050EA410618BF52EA4306D1D181
:1019F00081EA030101F000414FF0000070BD50EAA0
:101A0000410606BF1046194652EA430619D094EA29
:101A10000C0F02D150EA013613D195EA0C0F05D113
:101A200052EA03361CBF104619460AD181EA030167
:101A300001F0004141F0FE4141F470014FF000001F
:101A400070BD41F0FE4141F4780170BD70B54FF0BA
:101A5000FF0C4CF4E06C1CEA11541DBF1CEA13553A
:101A600094EA0C0F95EA0C0F00F0A7F8A4EB05041C
:101A700081EA030E52EA03354FEA013100F0888013
:101A80004FEA03334FF0805545EA131343EA1263DC
:101A90004FEA022245EA111545EA10654FEA002691
:101AA0000EF000419D4208BF964244F1FD0404F54A
:101AB000407402D25B084FEA3202B61A65EB0305A6
:101AC0005B084FEA32024FF480104FF4002CB6EB63
:101AD000020E75EB030E22BFB61A754640EA0C00E3
:101AE0005B084FEA3202B6EB020E75EB030E22BF23
:101AF000B61A754640EA5C005B084FEA3202B6EB64
:101B0000020E75EB030E22BFB61A754640EA9C0022
:101B10005B084FEA3202B6EB020E75EB030E22BFF2
:101B2000B61A754640EADC0055EA060E18D04FEAB0
:101B3000051545EA16754FEA06164FEAC30343EA50
:101B400052734FEAC2025FEA1C1CC0D111F4801F1D
:101B50000BD141EA00014FF000004FF0004CB6E716
:101B600011F4801F04BF01430020B4F1FD0C88BFB5
:101B7000BCF5E06F3FF6AFAEB5EB030C04BFB6EBC0
:101B8000020C5FEA500C50F1000041EB045170BDB3
:101B90000EF0004E4EEA113114EB5C04C2BFD4EBE0
:101BA0000C0541EA045170BD41F480114FF0000E64
:101BB000013C90E645EA060E8DE60CEA135594EAE0
:101BC0000C0F08BF95EA0C0F3FF43BAF94EA0C0FE3
:101BD0000AD150EA01347FF434AF95EA0C0F7FF458
:101BE00025AF104619462CE795EA0C0F06D152EAAC
:101BF00003353FF4FDAE1046194622E750EA410690
:101C000018BF52EA43067FF4C5AE50EA41047FF4A0
:101C10000DAF52EA43057FF4EBAE12E74FF0FF3C05
:101C200006E000BF4FF0010C02E000BF4FF0010CD6
:101C30004DF804CD4FEA410C7FEA6C5C4FEA430C4F
:101C400018BF7FEA6C5C1BD001B050EA410C0CBF9E
:101C500052EA430C91EA030F02BF90EA020F002000
:101C6000704710F1000F91EA030F58BF994208BF67
:101C700090422CBFD8176FEAE37040F00100704724
:101C80004FEA410C7FEA6C5C02D150EA013C07D17B
:101C90004FEA430C7FEA6C5CD6D152EA033CD3D0C6
:101CA0005DF8040B704700BF8446104662468C46C0
:101CB0001946634600E000BF01B5FFF7B7FF0028F3
:101CC00048BF10F1000F01BD4DF808EDFFF7F4FF1C
:101CD0000CBF012000205DF808FB00BF4DF808EDA7
:101CE000FFF7EAFF34BF012000205DF808FB00BFCA
:101CF0004DF808EDFFF7E0FF94BF012000205DF8EC
:101D000008FB00BF4DF808EDFFF7CEFF94BF0120A0
:101D100000205DF808FB00BF4DF808EDFFF7C4FF99
:101D200034BF012000205DF808FB00BF4FEA410CE2
:101D30007FEA6C5C02D150EA013C0AD14FEA430CC5
:101D40007FEA6C5C02D152EA033C02D14FF0000002
:101D500070474FF0010070474FEA410212F5001240
:101D600015D211D56FF47873B3EB625212D94FEAE2
:101D7000C12343F0004343EA505311F0004F23FACC
:101D800002F018BF404270474FF00000704750EA21
:101D9000013005D111F0004008BF6FF000407047DE
:101DA0004FF00000704700BF4FEA4102B2F1E0433C
:101DB00024BFB3F5001CDCF1FE5C0DD901F0004C32
:101DC0004FEAC0024CEA5070B2F1004F40EB830082
:101DD00008BF20F00100704711F0804F21D113F1AE
:101DE0003872BCBF01F00040704741F480114FEAE7
:101DF0005252C2F11802C2F1200C10FA0CF320FA70
:101E000002F018BF40F001004FEAC1234FEAD3238C
:101E100003FA0CFC40EA0C0023FA02F34FEA4303F6
:101E2000CCE77FEA625307D150EA01331EBF4FF07F
:101E3000FE4040F44000704701F0004040F0FE409A
:101E400040F40000704700BF80F0004002E000BF97
:101E500081F0004142001FBF5FEA410392EA030F95
:101E60007FEA226C7FEA236C6AD04FEA1262D2EBDF
:101E70001363C1BFD218414048404140B8BF5B42E4
:101E8000192B88BF704710F0004F40F4000020F07D
:101E90007F4018BF404211F0004F41F4000121F093
:101EA0007F4118BF494292EA030F3FD0A2F10102DD
:101EB00041FA03FC10EB0C00C3F1200301FA03F11B
:101EC00000F0004302D5494260EB4000B0F5000F3E
:101ED00013D3B0F1807F06D340084FEA310102F1FD
:101EE0000102FE2A51D2B1F1004F40EBC25008BFAF
:101EF00020F0010040EA03007047490040EB000079
:101F0000013A28BFB0F5000FEDD2B0FA80FCACF179
:101F1000080CB2EB0C0200FA0CF0AABF00EBC250A6
:101F200052421843BCBFD0401843704792F0000F94
:101F300081F4000106BF80F400000132013BB5E7E7
:101F40004FEA41037FEA226C18BF7FEA236C21D05D
:101F500092EA030F04D092F0000F08BF08467047C2
:101F600090EA010F1CBF0020704712F07F4F04D190
:101F7000400028BF40F00040704712F100723CBFA3
:101F800000F50000704700F0004343F0FE4040F4CD
:101F9000000070477FEA226216BF08467FEA23638B
:101FA0000146420206BF5FEA412390EA010F40F476
:101FB000800070474FF0000304E000BF10F00043C2
:101FC00048BF40425FEA000C08BF704743F09643A9
:101FD00001464FF000001CE050EA010208BF7047C4
:101FE0004FF000030AE000BF50EA010208BF70474B
:101FF00011F0004302D5404261EB41015FEA010C60
:1020000002BF84460146002043F0B64308BFA3F157
:102010008053A3F50003BCFA8CF2083AA3EBC25339
:1020200010DB01FA02FC634400FA02FCC2F1200258
:10203000BCF1004F20FA02F243EB020008BF20F08F
:102040000100704702F1200201FA02FCC2F12002F5
:1020500050EA4C0021FA02F243EB020008BF20EAEA
:10206000DC7070474FF0FF0C1CEAD0521EBF1CEA18
:10207000D15392EA0C0F93EA0C0F6FD01A4480EA06
:10208000010C400218BF5FEA41211ED04FF00063EF
:1020900043EA501043EA5111A0FB01310CF000401B
:1020A000B1F5000F3EBF490041EAD3715B0040EA41
:1020B000010062F17F02FD2A1DD8B3F1004F40EB11
:1020C000C25008BF20F00100704790F0000F0CF0E4
:1020D000004C08BF49024CEA502040EA51207F3AA8
:1020E000C2BFD2F1FF0340EAC250704740F4000083
:1020F0004FF00003013A5DDC12F1190FDCBF00F074
:1021000000407047C2F10002410021FA02F1C2F121
:10211000200200FA02FC5FEA310040F1000053EABD
:102120004C0308BF20EADC70704792F0000F00F00B
:10213000004C02BF400010F4000F013AF9D040EA11
:102140000C0093F0000F01F0004C02BF490011F4A5
:10215000000F013BF9D041EA0C018FE70CEAD153A3
:1021600092EA0C0F18BF93EA0C0F0AD030F0004C23
:1021700018BF31F0004CD8D180EA010000F00040D7
:10218000704790F0000F17BF90F0004F084691F095
:10219000000F91F0004F14D092EA0C0F01D14202CF
:1021A0000FD193EA0C0F03D14B0218BF084608D198
:1021B00080EA010000F0004040F0FE4040F40000E2
:1021C000704740F0FE4040F4400070474FF0FF0C75
:1021D0001CEAD0521EBF1CEAD15392EA0C0F93EABC
:1021E0000C0F69D0A2EB030280EA010C49024FEA0E
:1021F000402037D04FF0805343EA111143EA1013C7
:102200000CF000408B4238BF5B0042F17D024FF47E
:10221000000C8B4224BF5B1A40EA0C00B3EB510F59
:1022200024BFA3EB510340EA5C00B3EB910F24BF42
:10223000A3EB910340EA9C00B3EBD10F24BFA3EBC7
:10224000D10340EADC001B0118BF5FEA1C1CE0D18F
:10225000FD2A3FF650AF8B4240EBC25008BF20F042
:10226000010070470CF0004C4CEA50207F32C2BF96
:10227000D2F1FF0340EAC250704740F400004FF033
:102280000003013A37E792F0000F00F0004C02BF64
:10229000400010F4000F013AF9D040EA0C0093F02E
:1022A000000F01F0004C02BF490011F4000F013B88
:1022B000F9D041EA0C0195E70CEAD15392EA0C0FF0
:1022C00008D142027FF47DAF93EA0C0F7FF470AF28
:1022D000084676E793EA0C0F04D14B023FF44CAF6B
:1022E00008466EE730F0004C18BF31F0004CCAD100
:1022F00030F000427FF45CAF31F000437FF43CAF3C
:102300005FE700BF4FF0FF3C06E000BF4FF0010C5D
:1023100002E000BF4FF0010C4DF804CD4FEA40023F
:102320004FEA41037FEA226C18BF7FEA236C11D089
:1023300001B052EA530C18BF90EA010F58BFB2EB3C
:10234000030088BFC81738BF6FEAE17018BF40F0BC
:10235000010070477FEA226C02D15FEA402C05D170
:102360007FEA236CE4D15FEA412CE1D05DF8040BF5
:10237000704700BF844608466146FFE70FB5FFF788
:10238000C9FF002848BF10F1000F0FBD4DF808ED40
:10239000FFF7F4FF0CBF012000205DF808FB00BF31
:1023A0004DF808EDFFF7EAFF34BF012000205DF88B
:1023B00008FB00BF4DF808EDFFF7E0FF94BF0120D8
:1023C00000205DF808FB00BF4DF808EDFFF7D2FFD5
:1023D00094BF012000205DF808FB00BF4DF808ED18
:1023E000FFF7C8FF34BF012000205DF808FB00BFE5
:1023F0004FEA40024FEA41037FEA226C02D15FEAD2
:10240000402C08D17FEA236C02D15FEA412C02D133
:102410004FF0000070474FF0010070474FEA400254
:10242000B2F1FE4F0FD34FF09E03B3EB12620DD902
:102430004FEA002343F0004310F0004F23FA02F06C
:1024400018BF404270474FF00000704712F1610F13
:1024500001D1420205D110F0004008BF6FF00040EA
:1024600070474FF00000704742000ED2B2F1FE4FAD
:102470000BD34FF09E03B3EB126209D44FEA002353
:1024800043F0004323FA02F070474FF0000070471A
:1024900012F1610F01D1420202D14FF0FF307047BB
:1024A0004FF00000704700BF53B94AB9002908BF78
:1024B00000281CBF4FF0FF314FF0FF3000F06AB929
:1024C000ADF1080C6DE904CE00F006F8DDF804E08B
:1024D000DDE9022304B070472DE9F047089D0C4662
:1024E000002B4ED194468C458646B2FA82F262D9D0
:1024F0004AB1C2F12003914020FA03F30CFA02FC26
:10250000194300FA02FE4FEA1C471FFA8CF6B1FB92
:10251000F7F44FEA1E4307FB141143EA014304FB9F
:1025200006F199420AD91CEB030304F1FF3080F055
:102530001281994240F20F81023C6344591A1FFAFA
:102540008EF3B1FBF7F007FB101143EA014300FBE8
:1025500006F69E420AD91CEB030300F1FF3180F01E
:10256000FC809E4240F2F980634402389B1B40EAA3
:10257000044000211DB1D3400022C5E90032BDE86E
:10258000F0878B4205D90DB1C5E90001002108464D
:10259000F5E7B3FA83F1002946D1A34202D3904272
:1025A000C0F0F080861A64EB03030120002DE6D012
:1025B000C5E90063E3E7002A40F09080A1EB0C043A
:1025C0004FEA1C481FFA8CF70121B4FBF8F64FEADA
:1025D0001E4308FB164443EA044307FB06F09842F7
:1025E00008D91CEB030306F1FF3402D2984200F233
:1025F000CD8026461C1A1FFA8EF3B4FBF8F008FBB8
:10260000104443EA044300FB07F79F4208D91CEB40
:10261000030300F1FF3402D29F4200F2B080204653
:10262000DB1B40EA0640A5E7C1F120068B4022FAF9
:1026300006F71F4320FA06FC04FA01F343EA0C03F1
:10264000F44000FA01F8380C4FEA1349B4FBF0FEED
:102650001FFA87FC00FB1E4449EA04440EFB0CF9F8
:10266000A14502FA01F20AD93C190EF1FF3A80F0B5
:102670008480A14540F28180AEF1020E3C44A4EB7F
:1026800009041FFA83F9B4FBF0F300FB134449EA91
:10269000044403FB0CFCA44507D93C1903F1FF30AB
:1026A00067D2A44565D9023B3C4443EA0E40A0FBF7
:1026B0000293A4EB0C049C42CE469C4651D34ED0D0
:1026C00055B1B8EB0E0364EB0C0404FA06F6CB40EC
:1026D0001E43CC40C5E90064002150E7C2F120034D
:1026E00020FA03F10CFA02FC24FA03F394400C43A1
:1026F0004FEA1C4800FA02FE1FFA8CF7B3FBF8F011
:1027000008FB1031230C43EA014300FB07F1994217
:1027100008D91CEB030300F1FF362CD299422AD9C9
:10272000023863445B1AA4B2B3FBF8F108FB11331F
:1027300044EA034401FB07F3A34208D91CEB040459
:1027400001F1FF3613D2A34211D902396444E41ACD
:1027500041EA004139E70446F0E6084606E7C84585
:10276000AED2B9EB020E63EB070C0138A8E7314695
:10277000EDE7034699E73046D4E7D6467FE7634462
:1027800002384DE70646234608460FE7023E6344FB
:1027900030E700BF704700BF00487047001BB74BD1
:1027A00070B50C4601F0ECF9104E05460821304694
:1027B00005F08EFA012804D001F0E2F9431BA34290
:1027C00007D30821094805F083FA431E58425841AF
:1027D00070BD72B60821304605F07AFA012800D0A3
:1027E00030BF62B6BFF36F8FE0E700BF0004004860
:1027F00008B5002210214FF0904005F06FFA05480F
:102800000022202105F06AFABDE80840022001F00C
:10281000BFB900BF0004004810B50C4C01221021C4
:10282000204605F05BFA052001F0B2F920460122AE
:10283000202105F053FA4FF090400122102105F0BD
:102840004DFABDE81040022001F0A2B90004004892
:1028500070B54FF090400C46164610210022144DE2
:1028600005F03CFA00232B701248B3B222462146F1
:1028700006F028FCD8B901F083F941F28736044606
:102880002B783BB1BDE87040012210214FF0904001
:1028900005F024BA01F074F9031BB342F2D872B602
:1028A0002B7803B930BF62B6BFF36F8FE8E770BD16
:1028B000BD05002020070020014B01221A7070473F
:1028C000BD050020004870474061030813B5114B57
:1028D0000446186800909B88ADF804300120FFF78B
:1028E0009BFF062269460120FFF7B2FF0120FFF798
:1028F0007FFF9DF80430112B08D19DF80520122A86
:1029000004D101202370627002B010BD00231A466A
:102910001846F7E7082003080CB4F0B5ADB032ABA9
:1029200006AF53F8042B059305460E46384696210C
:102930002CF05AF89528C1BF42F62E63ADF8AA30A4
:102940002E23ADF8AC3000F037F83C24042D4FF4C2
:102950007A7E1449B0FBFEFCB0FBF1F14EF6602329
:10296000B0FBF3F3B3FBF4F204FB1232BCFBF4F361
:1029700004FB13C30EFB1C049ABF0B48405D3F20B1
:10298000CDE90040CDE9026708482BF0ADFF084BC8
:102990001B6898682BF0D2FE2DB0BDE8F04002B065
:1029A000704700BF80EE36009E6103087C6103081B
:1029B000CC03002001F0ECB801F0E2B81348144A4F
:1029C00008B54FF00043C0E9002304224261012210
:1029D0000023C2614FF480510722C0E90233C0E9ED
:1029E0000933C0E90C1203610383837680F8203039
:1029F00080F82C30826380F83C30C36404F0C0F867
:102A000018B1BDE8084000F099BB08BDC005002022
:102A1000002401400268084B9A4282B00AD14FF06C
:102A2000B0431A6E42F400721A661B6E03F4007310
:102A30000193019B02B07047002401400268054BDE
:102A40009A4201BF4FF0B042136E23F40073136635
:102A5000704700BF0024014030B585B00024054612
:102A6000CDE901440394FFF7A9FF144804F01CFCCE
:102A700008B100F063FB1148039401A9CDE90154AA
:102A800004F0DCF908B100F059FB0C4804F036FB07
:102A900008B100F053FB4FF0FF31084804F070F923
:102AA000064804F0E3FB054804F0C4F90446034873
:102AB00004F086FB204605B030BD00BFC0050020F5
:102AC000014B024A1A607047C005002000240140F3
:102AD00008B50948FFF7C0FF68B1084BB3F8AA3042
:102AE0004FF6FF72934216BF40F6E442044B534345
:102AF000B3FBF0F398B208BD002000B40075FF1FCF
:102B0000D8084C0013B50023ADF80630FFF7E0FFFE
:102B100004461948FFF7A0FF184BB3F8C820B3F8D4
:102B2000A8108A4204FB00F018D040F6E443B0FB42
:102B3000F3F364205B1A4343521A93FBF2F31E3300
:102B40001BB2ADF80630BDF806305BB21B02ADF823
:102B50000630BDF8060000B202B010BD4FF47A7224
:102B600040F6FF73B0FBF3F35343A3F53923A3F50A
:102B70000C6340F6C412E0E7001000B00075FF1FC0
:102B80004FF0B04382B09A6A22F480529A629A6CF3
:102B900042F480529A649B6C03F480530193019B2E
:102BA000002002B070474FF0B04307B59A6C42F076
:102BB00004029A649A6C02F004020192019A9A6CDF
:102BC00042F001029A649B6C002203F0010311465B
:102BD00000930B20009B04F005FC0B2004F034FC58
:102BE000002211460C2004F0FDFB0C2004F02CFC0C
:102BF000002211460D2004F0F5FB0D2004F024FC0A
:102C0000002202210F2004F0EDFB0F2004F01CFC39
:102C100000221146102004F0E5FB102004F014FC03
:102C200000221146112004F0DDFB112003B05DF8F5
:102C300004EB04F009BC000008B504F049FE10B133
:102C40006FF0040008BD064B9A6942F040429A6159
:102C50004CF2FA321A6104F04DFE0028F2D0EFE790
:102C600000400058F0B585B000230D46009306469D
:102C7000A8B3FFF7E1FF044670BB04F029FE88BB50
:102C80001A481B4A02230193D0F8E01506F1784355
:102C900002EA8121B3FBF1F701FB1733DB0A029350
:102CA000D0F8E00505F178410139314402EA80228B
:102CB000B1FBF2F002FB1011C3EBD12301336946E3
:102CC00001A8039304F096FE20B1022814BF6FF010
:102CD0000104012404F00EFE204605B0F0BD6FF0A3
:102CE0000504F9E76FF00404F6E700BF0070FF1F6A
:102CF00000FCFF03014B18600020704724060020F1
:102D00002DE9F04FB0F1006F89B006460F469046AE
:102D1000C0F0C080DFF89091644DD9F8E03505EA45
:102D2000832303F10063013B984200F2B380002942
:102D300000F0B38040EA02035B0740F0AE80FFF78B
:102D40007BFF044690BB04F0C3FD002840F0A88040
:102D5000D9F8E015009705EA812106F17842B2FB27
:102D6000F1F301FB132208F17843013B3344B3FB39
:102D7000F1F001FB1033DB0A01334FEAD22AA3EB57
:102D8000D222012A039388BFC6F30A050AF58037C9
:102D9000C6F108038CBFC5F500654546FF02B34682
:102DA0000693039B9A4505D304F0A4FD204609B081
:102DB000BDE8F08FA6F10803069A1A4495421CD884
:102DC000009B04950193CDF814B04FF00009059BCA
:102DD00009EB0301049B99453DD3009BAB442B4475
:102DE000A8EB0505B5F5006F009328BF4FF400650B
:102DF0000AF1010A07F50067D3E753F8081F5A687C
:102E0000B2F1FF3F08BFB1F1FF3FD5D0284B1868A2
:102E100010B96FF00504C7E727B14FF400623946D7
:102E200011F0EAFFDFF888900099D9F80030CBF371
:102E30000A001844AAB211F0DFFF4FF400613846CF
:102E4000FFF710FF00BBD9F8003001934FF4006387
:102E500005970493B9E7019B07914B440293012026
:102E6000D3E9002304F080FD88B90799019BD1E9DB
:102E7000000259F80310029B5B689A4208BF88421F
:102E800005D109F10809A2E76FF001048CE76FF0A2
:102E9000030489E74FF0FF3488E76FF0050485E706
:102EA0006FF0040482E700BF0070FF1F00FCFF0307
:102EB00024060020B1F1006F70B510D30B4BD3F88E
:102EC000E0650B4B03EA862303F10063013B994263
:102ED00005D838B192B211F08FFF002070BD4FF0CD
:102EE000FF30FBE76FF00500F8E700BF0070FF1F41
:102EF00000FCFF03B0F1006F10B40DD3084BD3F802
:102F0000E045084B03EA842303F10063013B984248
:102F100002D810BCFFF7A6BE4FF0FF3010BC7047C0
:102F20000070FF1F00FCFF034FF0B04382B0DA6C6B
:102F30000243DA64DB6C03400193019B02B07047EB
:102F40002DE9F04186B01422002101A82BF06AFD82
:102F50000220464EFFF7E8FF0420FFF7E5FF0120BF
:102F6000FFF7E2FF04213046002204F0B7FE002202
:102F700010214FF0904004F0B1FE042300240125FD
:102F800002270DEB03013046CDE901354FF0100863
:102F9000CDE9034704F07CFD01A93046CDE9018568
:102FA000CDE9037404F074FD202301A93046CDE976
:102FB0000135CDE9037404F06BFD01A94FF0904099
:102FC000CDE90185CDE9034404F062FD08224FF408
:102FD000881301A93046CDE901234FF00308CDE95C
:102FE000034704F055FD4FF4441301A94FF09040FE
:102FF000CDE90183CDE9035704F04AFD4FF4405376
:1030000001A93046CDE90135CDE9034804F040FD82
:103010004FF404134021CDE901131548039501A98C
:1030200004F036FD22460F21062004F0DBF90620CD
:1030300004F00AFA22460F21072004F0D3F90720F2
:1030400004F002FA22462146092004F0CBF90920B7
:1030500004F0FAF922462146092004F0C3F90920B8
:1030600004F0F2F906B0BDE8F08100BF00040048AA
:103070000008004800B59BB04822002108A82BF0AA
:10308000D1FC1822002102A82BF0CCFC04F040FE59
:103090004FF0B0420120D2F8903023F01803C2F86C
:1030A0009030D2F8003423F4C06343F40073C2F8C4
:1030B0000034D2F8003403F4C0630193019B24234D
:1030C000089381230B930023CDE91003B02208A8B5
:1030D000CDE9122304F094FF08B172B6FEE74F2346
:1030E000CDE90230CDE90400CDE90600022102A8B5
:1030F00005F020FA08B172B6FEE71BB05DF804FBDC
:1031000008B503F0EBFCFFF7B5FFFFF719FFFFF77A
:103110004AFD00F0D1FF00F063FE00F089F8064898
:103120000122042104F0DAFD02F080F900F018FC1D
:1031300002F083F9FCE700BF0004004872B6FEE726
:1031400000B58DB02C22002101A82BF06BFC174894
:10315000174B03601F2383604FF080420023C0E9B8
:103160000433C0E9072383614FF48073436205F0A1
:1031700087FC08B1FFF7E2FF0C4805F0ADFD08B190
:10318000FFF7DCFF4FF00053002207930748089237
:103190004FF4807301A9029206920B9305F0D0FCC4
:1031A00008B1FFF7CBFF0DB05DF804FB2806002047
:1031B0000028004010B5044690B03822002102A833
:1031C0002BF030FC2268194B9A422CD14FF48033FB
:1031D000029302A84FF480730F9305F0CFFA08B161
:1031E000FFF7ACFF4FF0B0430220D3F8902042F439
:1031F0000042C3F890209A6D42F480629A659B6DFC
:10320000002203F4806311460193019B04F0EAF865
:10321000022004F019F900222A20114604F0E2F8F5
:103220002A2004F011F910B010BD00BF00280040A2
:103230001148124A08B54FF48273C0E900230023F5
:103240004FF4E062C0E902324FF400712822C0E975
:1032500006120722C0E90433C0E90833C0E90B2392
:1032600083620823436305F0A7FE18B1BDE8084058
:10327000FFF764BF08BD00BF2007002000300140F9
:10328000F0B5054689B01422002103A82BF0CAFB33
:103290002A68374B9A4269D14FF0B04302261A6E22
:1032A00042F480521A661A6E02F480520292029A16
:1032B000DA6C42F00102DA64DA6C02F00102019287
:1032C000019ADA6C42F00202DA64DB6C03F002036A
:1032D00000930524009B0327D02303A94FF09040BF
:1032E000CDE90336CDE9067404F0D2FB2023CDE905
:1032F00003364FF09040002603A90794CDE90567F7
:103300001C4C04F0C5FB1C4826620723C4E90003DB
:1033100080232046C4E90266C4E90436C4E906668F
:1033200004F0F2F808B1FFF709FF144AAC65A56292
:10333000134C0823C4E900231021002380222046D7
:10334000C4E90213C4E90423C4E90633236204F088
:10335000DBF808B1FFF7F2FE002222206C6511466F
:10336000A56204F03FF8222004F06EF809B0F0BD29
:1033700000300140C00600201C0002403000024026
:10338000600600207047000008B503F0BDFB044B49
:103390000120C3F88800BDE8084004F011BD00BF5B
:1033A0000004005808B503F0B6FB00F095FFFFF7E6
:1033B000C7FDFFF7F8FB00F013FDBDE80840FFF77D
:1033C00037BF08B503F0A7FBFFF7BAFDFFF7EBFB2C
:1033D000BDE80840FFF72CBF08B503F095FBBDE83A
:1033E00008400121002004F09BBC70477047FEE7B5
:1033F000FEE7FEE7FEE7FEE770477047704770475D
:10340000014805F08FBC00BF28060020024B0120B8
:10341000187004F071BC00BF721C0020024B012226
:1034200002201A7004F068BC711C0020082004F00F
:1034300063BC0000014804F0DDB900BF2C1100207E
:10344000014804F0D7B900BFC0060020014804F0CD
:10345000D1B900BF6006002070470000014804F0A9
:10346000C9B900BFE011002070470000014806F014
:1034700017B800BF20070020014807F095B900BF2A
:1034800040120020014805F081BA00BF2806002044
:10349000014806F096BA00BF181100202DE9F0434C
:1034A00089B080460020109E0790894615461F4629
:1034B000FCF7BEFEF0B9104CCDE90090CDE9020456
:1034C00007AB0E480593142304933A464346294616
:1034D0000068FCF777FF2346324604F1140153F8E5
:1034E000044B42F8044B8B42F9D1079B337509B06A
:1034F000BDE8F0830120FAE79A0700203061030855
:103500001FB50E4C00233C2202A8CDE902336275A0
:10351000237500F0DFFA042303AA0094122108485F
:10352000FFF7BCFF0749142220462BF06BFAB0FAD4
:1035300080F35B09637504B010BD00BF84070020F1
:10354000BC610308361F0020034A044840F21B53A5
:10355000002106F059BF00BFAE0700208C110020EB
:10356000312BF0B52DD81825102415FB0343194D28
:1035700000244FF0800C4CFA04F6A3F110073142FE
:1035800005EB470714BF4FF0240E4FF0140EA7F8B9
:1035900006E0A3F10807304205EB470714BF4FF0E0
:1035A000240E4FF0140E0134324205EB4306A7F807
:1035B00006E00CBF14272427082CF78003F1010331
:1035C000D9D1054B1B781BB9BDE8F040FFF7BCBF54
:1035D000F0BD00BFAE070020DC1C002010B50024A9
:1035E0000022E3B2114610460134FFF7B9FF322C36
:1035F000F6D1BDE81040FFF7A7BF000070B5044644
:103600000D46FFF7EBFF0F4B04EB440400261C4470
:10361000142000F0BDFAA2786178207812FB05F240
:1036200011FB05F110FB05F0F3B2D2B2C9B2C0B282
:103630000136FFF795FF322EEAD1BDE870400A202F
:1036400000F0A6BA080000202DE9F04106460F461A
:103650002048904600214FF416622BF0E3F91E4AF1
:1036600010254FF0800C2B4600244CFA04F1A3F1F6
:1036700010000F4202EB400014BF4FF0240E4FF039
:10368000140EA0F806E0A3F108000E4202EB400081
:1036900014BF4FF0240E4FF0140E013418EA010F3E
:1036A00002EB4301A0F806E00CBF14202420082CF4
:1036B000C88003F10103D8D11835B5F5986FD2D180
:1036C000064B1B781BB9BDE8F041FFF73DBFBDE8D5
:1036D000F08100BFB4070020AE070020DC1C0020F2
:1036E00000F00F000B4607281ED8DFE800F00407A3
:1036F0000A0F1316191B0022114600E00022104683
:1037000002E0002211461846FFF79EBF0A4600213C
:103710000020F9E700220846F6E70A460021EEE716
:103720000A46F5E70A46E7E770470000024B1878BB
:10373000024B1978FFF7D4BF0600002000000020DC
:1037400070B57248724C0378DBB20B2B12D8DFE8ED
:1037500013F00C002C00300036003D006300900098
:10376000A600B600C500C500C5006A4B1B78DBB2D9
:10377000694A13700378694E012B06D0684D2A7888
:1037800002F0FF03002A00F0AE80634A00231370AA
:1037900023703370FFF722FF624A00231370624ADE
:1037A0001370624B01221A7070BD5B4B00221A70BD
:1037B000E0E75F4A1278012A08BF0123D8E75D4B92
:1037C0001A78002A76D1544B0122F0E7594B5A4916
:1037D0001A7852B9594A1278012A06D10A78012A70
:1037E000D5B202D14C4B1D70C4E71B78012B05D01C
:1037F000524B1B7813B10B78002BBBD1464B0222E6
:103800001A704F4A1578022DEAB22BD0032A28D01D
:10381000012A29D1232225E0464A3F4B1578464903
:103820009DB9464D2D78012D0FD10D78012DEEB2A9
:103830000BD11E70424A1578022DEAB212D0032A2B
:103840000FD0012AE6D002220CE01278012A05D01E
:103850003A4A127812B10A78002AEBD102221A7081
:10386000E8E7042222701A700A78002A82D1232203
:103870009DE7304B1A783AB92D4A1278012AD1B215
:1038800002D1254B197075E71B78012B04D0284B0A
:103890001B78002B7FF46EAF1F4B022287E7254B6E
:1038A0001A781AB9274A1278002A8CD01B78012B73
:1038B000F2D0244B1B78012B7FF45CAFECE71D4B5F
:1038C0001A7822B9204A1278042A3FF47CAF1B7878
:1038D000012BE1D01C4B1B78052BEDE71A4B1A7816
:1038E000042AF8D16FE72A7812B90B4B1B78DBB2A8
:1038F0002370164B20781978FFF7F2FE2B7803B16E
:1039000023782378DBB2337046E700BF3E00002007
:103910000600002004000020070000200100002015
:10392000DC1C0020661C0020651C0020D41C00202C
:10393000351F0020631C00204100002042000020B1
:10394000EA120020621C0020611C00200000002000
:10395000024803680021596306F0D0BD8C11002095
:1039600038B501240A25294620461435FFF7B8FE4C
:10397000EDB2322000F00CF96E2DF4D10134E4B236
:10398000FFF72CFE082CEDD138BD0000054808B526
:103990000823036005F032FE18B1BDE80840FFF7C8
:1039A000CDBB08BD181100204FF0B04307B55A6ECB
:1039B00042F001025A665B6E002203F0010301939C
:1039C00011463220019B03F00DFD322003B05DF85B
:1039D00004EB03F039BD00000CB407B5054A05AB94
:1039E0001021019311F0D4FD03B05DF804EB02B097
:1039F000704700BFCE61030830B585B0044602A809
:103A00000D4611F05DFBBDF90C30064A0093102104
:103A1000029B2046FFF7E0FF2046FDF729FD2880A6
:103A200005B030BDCE6103084FF0B04210B59368C9
:103A300023F40043936011F05FFC104B01241C70D1
:103A400000F0ACF811F068F80D4811F07FF80D4B5C
:103A50004FF400421A61002011F07EF8FFF730F8B1
:103A600000F0F8F811F072F92146204611F08EF9B5
:103A700021462046BDE8104011F072B92411002003
:103A8000F93900080040005811F096B908B5FFF761
:103A90001FF840F6B83398420CD8B0F5E16F0BD35D
:103AA000FE23A0F5E16058434FF49663B0FBF3F0BA
:103AB000C0B208BDFE20FCE70020FAE77FB56846EB
:103AC00000F0ACF80198FEF7A9FC00B207B05DF871
:103AD00004FB0000194A38B5D2F88035591C044659
:103AE00019D103F01FF8054603F028F8054403F048
:103AF0001FF82B0EE3712B0CA3712B0A6371030EBD
:103B0000E370C0F30742C0F307232571C0B2A2706F
:103B10006370207038BD190AC3718171190C1B0EB6
:103B200041710371D2F88435C370D2F88405C0F3B3
:103B30000722C0F30743000EE9E700BF0070FF1F34
:103B400038B5094BD3F8803503600133054609D1F8
:103B500002F0E8FF044602F0EBFF444002F0EEFF03
:103B600044402C6038BD00BF0070FF1F01210220BF
:103B700011F0F6B80021022011F0F2B800207047D1
:103B8000024B187808B100F0D3B970472411002017
:103B900082B00190019802B000F066BAF0B589B029
:103BA00002F0D2FF02F0D8FF02F0DEFF01230493FF
:103BB0000323069300254FF0B04305950795DA6C73
:103BC000154C42F00202DA64DA6C02F00202029250
:103BD000029ADA6C42F00202DA64DB6C03F0020350
:103BE00001934FF4805703A92046019B03974FF49C
:103BF000005603F04DFF03A92046039603F048FF4B
:103C00002A463946204604F069F82A4631462046BD
:103C100004F064F809B0F0BD0004004810B5044693
:103C2000FEF770FF074BA36040F30F20FEF7C6F9C5
:103C3000054B064A2360064B6060C4E9032300205D
:103C400010BD00BF0000484200007A440D093E004C
:103C5000AB030500002070470120704708B52AF02B
:103C600043FF162303604FF0FF3008BD08B52AF06C
:103C70003BFF16230360FEE770B50D4614460E4663
:103C8000731B9C4201DC204670BDAFF3008006F838
:103C9000010BF5E730B5104600234FF06042834238
:103CA00000DB30BDD2F8804EE50707D5D2F8004ED4
:103CB000E40703D5CC5C156815B114700133EEE749
:103CC00000BFF8E74FF0FF3070474FF400534B60F0
:103CD0000020704701207047002070470B4A116890
:103CE00010B5034609B90A491160106809490A4C20
:103CF0000344091B8B4206D92AF0F6FE0C2303600D
:103D00004FF0FF3010BD1360FCE700BF281100200A
:103D1000783F0020000001200008000037B5184B54
:103D200002689A42054628D14FF0B043154C1A6EEE
:103D300042F400621A661B6E134A03F40063019397
:103D4000019B1723C4E90023102100238020C4E92C
:103D500002134FF48073C4E904034FF4806C2023F2
:103D6000C4E906C320464FF40053236203F0CCFBA2
:103D700008B1FFF7E3F96C62A56203B030BD00BF84
:103D8000002C01402C1100200800024010B5044610
:103D900086B01422002101A82AF044FE22680F4BAD
:103DA0009A4218D14FF0B04301A9DA6C42F00102F7
:103DB000DA64DB6C03F0010300930222009B4FF4F2
:103DC0008073CDE901324FF090400123CDE90332F9
:103DD000059303F05DFE06B010BD00BF002C01404E
:103DE00010B510229CB0002400210DEB02002AF037
:103DF00019FE1C22214608A8CDE9014403942AF0AB
:103E000011FE342221460FA82AF00CFE2B482C4B21
:103E10008460C0E900343B23C0E90334C0E90544B1
:103E200006F038F808B1FFF789F94FF480532348BA
:103E3000049304A906F04CF908B1FFF77FF91F4875
:103E400006F058F808B1FFF779F900241B480394ED
:103E500001A9CDE9014406F053FB08B1FFF76EF963
:103E6000602316480E94002208A9CDE90834CDE954
:103E70000A44CDE90C4406F0A5F808B1FFF75EF955
:103E800000234FF40052CDE914230C4813934FF054
:103E900000720FA9CDE90F33CDE91133CDE9163307
:103EA000CDE91823CDE91A3306F056FB08B1FFF728
:103EB00045F90248FFF76AFF1CB010BD8C110020C5
:103EC000002C0140014B1868704700BFD81100203A
:103ED0000320704708B501464FF47A720023800230
:103EE000890DFEF7E1FA08BD4FF47A73A0FB0303D6
:103EF000800A40EA83507047034B98689A68904262
:103F0000FBD1C043704700BF0028004008B5FFF751
:103F1000F3FF014B186008BDD811002008B5FFF76A
:103F2000EBFF024B1B68C01A08BD00BFD811002070
:103F3000024B187808B1FFF7DFBF7047DC11002093
:103F400010B5074B074C0122DA654FF4807120460B
:103F500004F0E2FC4FF0FF332363002010BD00BFEC
:103F6000002800402806002002460021014804F0F5
:103F7000EABE00BF2806002002460121014804F0E5
:103F8000E2BE00BF2806002010B58CB02C22002114
:103F9000044601A82AF046FDFFF7D2FF0C4B0D485E
:103FA0001B681C440023089306934FF00053E4431E
:103FB000079301224FF4807301A902940B9304F03C
:103FC000BFFD08B1FFF7BAF800200CB010BD00BF6C
:103FD000D81100202806002038B50546FFF78CFFD1
:103FE00002210446074804F0B5FEC4F309024FF469
:103FF0007A71A2FB0121920AA30A2A8043EA805027
:1040000038BD00BF280600200148002104F0A2BEF0
:10401000280600200148012104F09CBE280600204B
:10402000F8B50F4D2E78CEB90E4C4FF0FF37276301
:10403000FFF786F8FFF784FF4FF48071204604F005
:104040006BFC2046276304F029FE324620460221FD
:1040500004F079FEFFF75AFF01232B700020F8BD12
:10406000DC11002028060020014610B54FF47A72BA
:1040700000238002890DFEF717FA0146FFF73CFF87
:104080000446FFF739FF031B8B4200D310BD00BF6E
:10409000F7E711F039BA000010B5064C02212046AE
:1040A00004F058FE0221421C2046BDE8104004F0F6
:1040B0004ABE00BF280600201648174A08B54FF42C
:1040C000E133C0E9002300230C22C0E90233C0E938
:1040D0000523C0E90733C0E90933036107F049F953
:1040E00008B1FFF72BF80B48002107F0BAFA08B126
:1040F000FFF724F80748002107F0D3FA08B1FFF7CB
:104100001DF8044807F08DFA18B1BDE80840FFF724
:1041100015B808BD401200200044004070B596B0AC
:1041200006461422002103A82AF07CFC3822002134
:1041300008A82AF077FC3268274B9A424AD102231A
:10414000089308A84FF440230A9304F017FB08B122
:10415000FEF7F4FF4FF0B04300259A6D1F4C42F478
:1041600000329A659A6D02F400320292029ADA6C79
:1041700042F00102DA64DB6C03F001030193019B5E
:104180000C220223CDE9032303A907234FF090401B
:104190000793CDE9055503F07BFC114925621423F3
:1041A000C4E900131023C4E9023520468023C4E982
:1041B0000435C4E9065503F0A7F908B1FEF7BEFFC0
:1041C0002520F46700220221A66203F00BF92520C6
:1041D00003F03AF916B070BD00440040E011002031
:1041E0008000024002680C4B9A4210B5044612D17E
:1041F0004FF0B0420C21936D23F4003393654FF0E0
:10420000904003F0F1FCE06F03F0F0F9BDE81040DE
:10421000252003F027B910BD0044004008B50A4628
:104220000146024806F024FA002008BD4012002092
:1042300013B5114B114C18604FF40013009302ABEF
:1042400013E90600204607F090F92368DA69D103E4
:10425000FCD4DA695202FCD59A68084842F480021C
:104260009A6007F0C8F906490448012207F036F9B8
:10427000002002B010BD00BFD41200204012002068
:10428000DC12002008B5074B1860FEF78CFCFFF726
:1042900013FF054AD2F8803043F00063C2F8803043
:1042A000002008BDD81200200008005808B54FF0C3
:1042B000B04308489A6B42F400329A639A6B22F436
:1042C00000329A63FFF78EFF112003F0CBF8002035
:1042D00008BD00BF4012002008B5074807F049F8A4
:1042E00008B1FEF72BFF054803F00EF918B1BDE841
:1042F0000840FEF723BF08BD40120020E011002057
:104300000268044B9A4203D1034B00201B681847F4
:10431000704700BF00440040D812002002680B4BD9
:104320009A4210B504460FD1094B1B682BB1D0F847
:10433000902012B907480121984720460549BDE859
:104340001040012207F0CAB810BD00BF0044004071
:10435000D4120020DC12002030B59BB0FEF7B2FA78
:1043600013F07AFD48B1012013F01EFE12F01AFB83
:104370000446019020B913F0E3FD01201BB030BDCD
:104380003A4D296812F05EFF6968204612F074FF0A
:10439000297A204612F0A4FF697A204612F0D4FF51
:1043A0006969204613F060F8E868FEF75DF881B2AD
:1043B000204612F0E3FF2969204612F0ABFFA97AEC
:1043C000204612F073FF0221204613F025F8102139
:1043D000204613F063F8019812F06CFB029018B9B4
:1043E00001A812F03FFBC6E701A812F03BFB0298C0
:1043F00012F0C8FE18B902A812F07AFCBBE71C4DF7
:10440000029800232B600A2203AB06A912F0ACFC31
:1044100060B129680798FDF71DFD03AB28600A22EB
:10442000029806A912F0A0FC0446C0B9002428682E
:104430001049FDF717FE4FF07C51FDF713FE286081
:10444000029812F0CFFE054602A812F051FC13F0BC
:1044500077FD002D91D084F00100C0B28EE729686D
:104460000798FDF7F7FC2860E1E700BF2000002077
:10447000741C002000007A442DE9F04FADF21C4D71
:104480004FF40072002106A82AF0CCFA4FF4007213
:10449000002186A8B74F2AF0C5FA00243E464FF007
:1044A00000082546B1682846FDF7D4FC716805462A
:1044B0002046FDF7CFFC08F10408B8F5007F04465C
:1044C00006F11006EED14FF070512846FDF7CAFDF7
:1044D0004FF0705106462046FDF7C4FD0024DFF87A
:1044E000948282464FF000092546D8F808003146EC
:1044F000FDF7AEFC0146FDF7B5FD01462846FDF788
:10450000A9FC51460546D8F80400FDF7A1FC014678
:10451000FDF7A8FD01462046FDF79CFC09F10409C2
:10452000B9F5007F044608F11008DED14FF0705154
:104530002846FDF797FD8346FDF706F98E4B0022CE
:104540002CF0E6F9CDE900014FF070512046FDF75F
:1045500089FDFDF7F9F8884B00222CF0D9F9FDF719
:1045600023FC06AD82462C464FF000094FF00008B0
:10457000B968B869FDF76CFCFDF750FF0028B8BFBB
:104580004042FDF71BFD44F8040B01464046FDF791
:1045900061FC09F10409B9F5FE7F804607F11007B7
:1045A000E6D17649FDF712FE06AC07464FF000094A
:1045B0004FF00008394654F8040BFDF749FC01465A
:1045C000FDF750FD01464846FDF744FC08F101089F
:1045D0001FFA88F8B8F17F0F8146EBD16749FDF7E4
:1045E000F5FDFDF7B1F8644B00222CF091F9CDE90F
:1045F000020186ACA04600234FF000092A46296834
:1046000050680493FDF724FCFDF708FF0028B8BFAD
:104610004042FDF7D3FC049B48F8040B01461846C2
:10462000FDF718FC09F101091FFA89F9B9F17E0FAC
:1046300005F104050346E1D15149FDF7C7FD4FF0EF
:10464000000905464FF00008294654F8040BFDF711
:10465000FFFB0146FDF706FD01464846FDF7FAFB64
:1046600008F101081FFA88F8B8F17E0F8146EBD1F6
:104670004349FDF7ABFDFDF767F83F4B00222CF0F7
:1046800047F9404A13889BB2FA2BCDE9040100F2A6
:10469000C680108880B2FDF791FC5146FDF794FE6C
:1046A000394C08B105232370384B1A78384B1B88D6
:1046B0009BB29A4280F08480364B1A78364B1B8826
:1046C0009BB29A4206D235493046FDF787FE08B1C3
:1046D00001232370324C334D238801339BB2238056
:1046E00023889BB20A2B04BF0023238022884FF02B
:1046F0001C0892B208FB02F2DDE90001AE502288EC
:1047000092B208FB0252C2F804B0FDF74DFBB4F8B8
:1047100000B0228892B208FB02521FFA8BFB08FB02
:104720000B5BC2F80CA0B4F800A0CBF808004FF067
:1047300086413846FDF796FC1FFA8AFA08FB0A5AAA
:104740002788CAF81000DDE90201FDF72DFB4FF0C4
:104750008641FDF787FC22880B4C92B2BFB208FB62
:10476000075708FB0255217878612976DDE90401B5
:104770001AE000BF041400200000E03F0000FE42E9
:104780000000FC423C000020EA120020030100204F
:10479000E212002002010020E0120020CDCC4C3FAC
:1047A000041C0020EC120020FDF7FEFA4FF08641B9
:1047B000FDF758FCFDF758FE244BC0B21880237853
:1047C000DFF88C80234C98F80030234F012B1DD14B
:1047D000DFF88890224DB9F80030B9F800204FF08A
:1047E0001C0A9BB292B20AFB03F30AFB0252E8587E
:1047F0009168FDF72FFB3146FDF7F0FD88B10223EC
:10480000237023782378DBB288F800302378DBB27A
:1048100088F800303E600DF21C4DBDE8F08F114865
:104820003BE7B9F80030D7F800909BB20AFB03557C
:104830003046A968FDF70EFB4946FDF7CFFD10B1E4
:1048400003232370E2E72070E0E700BFDE120020C0
:10485000E8120020EA120020E4120020041C0020CC
:10486000EC12002000007A432DE9F04F93B0FEF7E0
:1048700029F813F0F1FA48B1012013F095FB10F07C
:10488000A9FF0446069028B913F05AFB012013B083
:10489000BDE8F08F584E3378012BDDB24CD0022D9D
:1048A00063D0002D39D1042111F05AFB012120469B
:1048B00011F084FA5149204611F0B4FA50492046CB
:1048C00011F096FA4F49204611F044FA4E4920461D
:1048D00011F05AFA0221204611F076FB4B4920468E
:1048E00011F058FB2146684611F0B6FA484A0D927D
:1048F000484A0E924FF07C5300220CA920460C939C
:104900000F921092119311F0D3FA2946204611F01C
:10491000F3FA0321204611F009FB069800243470B5
:1049200010F0EEFF0790002861D106A810F0C0FF3C
:1049300007A811F073F8A7E72946374D11F03EFAA2
:1049400020462E4911F06EFAA968204611F002FAAD
:10495000E968204611F018FA696A204611F048FA11
:10496000E96C204611F016FBD7E72B4D012111F021
:1049700025FAE969204611F055FA696A204611F0D6
:1049800037FAA968204611F0E5F9E968204611F0E8
:10499000FBF9A86CFDF768FD81B2204611F014FB0D
:1049A000E96C204611F0F6FA2146684611F054FAF7
:1049B0002B6B0C936B6B0D93AB6B0E93EB6B0F939D
:1049C0002B6C10930CA96B6C1193204611F070FAAC
:1049D000A86AFDF749FDC1B2204611F08DFA286A98
:1049E000FDF742FDC1B2204611F008FB95E711F03A
:1049F000ABF898B900204AE7701C00200000824202
:104A00009A99993FCDCC4C3F000020406666263FE6
:104A1000000020410AD7233C081C00200026DFF8B4
:104A200018A2864DDFF818924FF0210837460798F4
:104A300008A911F0E1F800282FD09DF820305BB1D3
:104A40000A993846FDF706FA099907463046FDF7F8
:104A500001FA0134E4B206469AF80030012B16D16F
:104A60002B880A9A9BB209EB03139A602B88099A48
:104A70009BB209EB03135A602B889BB25A1C92B26B
:104A8000802B2A8003D1FFF7F7FC00232B800F2017
:104A9000FDF790FFB8F10108C9D1079811F074F83B
:104AA000069D0121284611F089F90421284611F0BC
:104AB00057FA6449284611F0B5F96349284611F0C0
:104AC00097F96249284611F045F96149284611F0E5
:104AD0005BF90221284611F077FA5E49284611F069
:104AE00059FA2946684611F0B7F95B4A0D925B4ABC
:104AF0000F924FF07C534FF07E520CA928460C9336
:104B00000E931092119311F0D3F90021284611F061
:104B1000F3F90321284611F009FA069907A810F0C5
:104B2000A7FF00283FF401AF079811F00DF8002807
:104B30003FF460AF06A810F0BBFEDFF8FCB0DFF872
:104B4000FC80DFF8FCA04FF02109079808A911F0BC
:104B500053F80546002837D09DF82D3073BB9DF8DB
:104B600020305BB10A993846FDF774F90999074678
:104B70003046FDF76FF90134E4B206469BF8003089
:104B8000012B1BD1B8F800300A9A9BB20AEB031331
:104B90009A60B8F80030099A9BB20AEB03135A6086
:104BA000B8F800309BB25A1C92B2802BA8F80020B3
:104BB00004D1FFF761FC0023A8F800300F20FDF7B7
:104BC000F9FEB9F10109C0D1012C254B94BF002297
:104BD00001221A70234A127822B91B78012B01D1C5
:104BE00000F008FC20493846FDF73CFA074620460D
:104BF000FDF7E4F9044601463846FDF7E7FA1A499D
:104C000007463046FDF72EFA2146FDF7DFFA174B2F
:104C10001F60174B1860079810F0B6FF044607A8EE
:104C200010F0FCFE13F08CF9002C3FF42FAE85F051
:104C30000100C0B22BE600BF00010020061C0020CE
:104C400004140020000082429A99993FCDCC4C3F39
:104C5000000020406666263F00002041CDCC4C3E3F
:104C6000631C0020601C002000007A445C1C0020B3
:104C7000581C002000B5ABB014230DF1060202A9A8
:104C8000ADF8063013F070FB28B1BDF80610002314
:104C90009AB2914202D82BB05DF804FB02AA02EB53
:104CA000C30201331279002A08BF1046F0E710B59D
:104CB00086B010220021044602A8019129F0B2FE1C
:104CC000FDF700FE13F0C8F88DF8040013F06EF93C
:104CD000031E18BF012301218DF80530009013F049
:104CE00083F9009813F022FB009813F097F90098CD
:104CF000FFF7C0FF002840F09980684613F066F97E
:104D000013F01EF9009813F0A5F9009813F0BEF9FE
:104D10000098FFF7AFFF002840F08C80684613F042
:104D200055F913F00DF9009813F0CCF9009813F031
:104D3000E5F90098FFF79EFF00287FD1684613F041
:104D400045F913F0FDF8009813F0F4F9009813F00A
:104D50007DFA0098FFF78EFF002873D1684613F0A4
:104D600035F913F0EDF8009813F08CFA009813F071
:104D7000A5FA0098FFF77EFF002867D1684613F078
:104D800025F913F0DDF8009813F0B4FA009813F049
:104D9000EDF90098FFF76EFF00285BD1684613F02D
:104DA00015F913F0CDF8009813F0FCF9009813F002
:104DB00015FA0098FFF75EFF00284FD1684613F000
:104DC00005F913F0BDF8009813F024FA009813F0D9
:104DD0003DFA0098FFF74EFF002843D1684613F0D4
:104DE000F5F813F0ADF8009813F04CFA009813F0B2
:104DF00065FA0098FFF73EFFC0BB684613F0E6F87F
:104E000013F09EF8009813F075FA01238DF80F3017
:104E100001AB03CB206018686160A060684613F0A6
:104E2000D5F813F08DF8002006B010BD01238DF8E1
:104E3000063067E701238DF8073074E701238DF80A
:104E4000083080E701238DF809308CE701238DF8C5
:104E50000A3098E701238DF80B30A4E701238DF881
:104E60000C30B0E701238DF80D30BCE701238DF83D
:104E70000E30C7E702480122102102F02FBF00BF09
:104E80000004004802480022102102F027BF00BFA2
:104E90000004004810B50A4C23780BB9E37C6BB1D1
:104EA000FEF72EFB0038074B18BF0120400018709A
:104EB0001B78022B02BF00232370E37410BD00BFD8
:104EC000361F0020DC1C002038B5114C2378F3B9C4
:104ED000E37CE3B90F4D2B68012B07D92B68042B1A
:104EE00004D80D4A0421012000F074FD2B68042B26
:104EF0000DD9FEF705FB0038084B18BF0120400014
:104F000018701B78022B02BF00232370E37438BD96
:104F1000361F0020D81C002028620308DC1C00205B
:104F200010B5124C237863B101214FF0904002F08C
:104F3000CFFE0F4B0022187022701B780D4ADBB297
:104F400013700D4C237863B102214FF0904002F0B2
:104F5000BFFE0A4B0022187022701B78084ADBB291
:104F60001370BDE81040FEF7EBBB00BF721C0020C1
:104F70004200002040000020711C00204100002061
:104F80003F00002010B5164B1A78022A26D91B784C
:104F9000082B23D8FFF768FC1248134A03781178CE
:104FA0005B1A124918BF01230B7003781048DBB25B
:104FB0001370104B104A1C780378E31A18BF0123B2
:104FC00013700E4B04701B7823B100230B700C4937
:104FD0000B701370BDE81040FEF7B2BB10BD00BFF0
:104FE0003E000020631C0020601C0020641C002088
:104FF000E8120020EA120020E9120020DC1C002048
:10500000661C002008B501214FF0904002F060FEC0
:10501000064B012816BF022218701A701878044B2C
:105020001978BDE80840FEF7E9BA00BF0600002085
:105030000000002038B5324D324C287BFCF7BAFF17
:105040003149FDF70FF8A060687BFCF7B3FF2E49EC
:10505000FDF708F8E060A87BFCF7ACFF2A49FDF7F4
:1050600001F86062E87BFCF7A5FF2849FCF7FAFF2E
:10507000274BE0642361287CFCF79CFF6060687C20
:10508000FCF798FFA061A87CFCF794FFE061E87C46
:10509000FCF790FF2062287DFCF78CFFA062687D02
:1050A000FCF78CFF1849FCF7DDFF2063A87DFCF7B7
:1050B00081FF6063E87DFCF781FF1449FCF7D2FFB4
:1050C000A063287EFCF776FFE063687EFCF776FF3E
:1050D0000D49FCF7C7FF2064A87EFCF76FFF0A4963
:1050E000FCF7C0FF6064E87EFCF764FFA064287FE3
:1050F000FCF760FF074BE06202221A7038BD00BF68
:10510000B5000020081C0020CDCCCC3D0AD7233CA4
:10511000CDCCCC3E701C002038B5114D114C287BF5
:10512000FCF74CFF1049FCF79DFFA060687BFCF783
:1051300045FF0D49FCF796FFE060A87BFCF73EFFBA
:105140000949FCF78FFF6062E87BFCF737FF0749EE
:10515000FCF788FF064BE06401221A7038BD00BFDF
:10516000B5000020081C0020CDCCCC3D0AD7233C44
:10517000701C002070B52A4D2A4E2B7803702A4BE4
:105180001B784370044601214FF0904002F0A0FDCF
:105190003378A070E37002214FF0904002F098FD48
:1051A000224B20711B7863713378012B35D1204B52
:1051B0001868FDF759F91F4BE0801868FDF754F99E
:1051C00080B21D4BA0831B78191F4A424A41A27727
:1051D0001A4A92F82B1084F82B10D26AE262012B43
:1051E00084F8283007D1164B1B8884F82930154BDA
:1051F0001B8884F82A30144B1B7853B1134B1B685F
:105200003BB1134B1B78012B01BF124A23231370B0
:105210002B70114B01221A7070BD0020E080D0E786
:1052200006000020631C00203E000020621C0020BD
:105230005C1C0020581C0020EA120020781C002072
:10524000E2120020DE120020010100206C1C002070
:10525000331F002007000020D41C002008B5FFF7F2
:1052600009FEFFF7E7FE034A00231370024A13709A
:1052700008BD00BF701C0020311F002010B5104B6E
:105280001A78104BD2B25A700024012263211A708E
:1052900083F8331083F834209C63DC631C645C6403
:1052A0009C64DC641C655C6583F82B40DC625C629A
:1052B0009C77FFF7DFFDFFF7D1FF034B1C7010BD9C
:1052C0003E000020781C0020311F002008B5FFF7A9
:1052D00043F8BDE808406420FEF75ABC2DE9F041D0
:1052E00086B00D460446FFF7C5FD01F0F7FBFDF75C
:1052F00027FE9620FEF74CFC154F00264FF00508C0
:10530000AE420FD14FF47A70FEF742FC01AB03CBF3
:105310001B8823810F4B2060002261601A7006B049
:10532000BDE8F081FEF71CFB87F80080FEF7FEF970
:105330004FF47A70FEF72CFC01A8FFF7B8FC41F29D
:105340008830FEF725FC0136FFF7C0FFD8E700BF25
:1053500006000020311F002013B50023044601A8D9
:10536000ADF80430FDF7B2FA30B19DF80430237087
:105370009DF805306370012002B010BD022801D8ED
:10538000FFF778BD7047022801D8FFF77BBD704753
:10539000022803D80248102102F0A5BC704700BFC4
:1053A0000004004807B568460FF0B0FE054B1B78B7
:1053B00003F0FF021BB9044B00999963DA6303B051
:1053C0005DF804FB03000020781C002007B5684648
:1053D0000FF09CFE054B1B7803F0FF021BB9044B3A
:1053E000009919645A6403B05DF804FB02000020C0
:1053F000781C002007B568460FF088FE0849009B1E
:105400000A689A1A022A08D9064A1278012A01BFA4
:10541000054A00209364D0640B6003B05DF804FB80
:10542000681C0020631C0020781C002008B5FEF7D3
:10543000FBFABDE8084000F0E5BC4FF0FF300FF08C
:105440001FBD7047014B01221A707047401D00209C
:1054500070470000014BD870704700BF500000201B
:10546000014B1874704700BF50000020002101203C
:105470000FF0CEBC10B50A4A0A4C42F21073002855
:1054800018BF03460848236013600FF09DFF216892
:10549000054810F021F8BDE8104003480FF0E2BFC6
:1054A000F80000204C000020981E002010B5094C88
:1054B000206023680BB9084B236008480FF084FF75
:1054C0002168064810F008F8BDE8104003480FF0C6
:1054D000C9BF00BFF8000020A0860100E01C00202A
:1054E00010B5094C2060236813B942F21073236091
:1054F00006480FF069FF216804480FF0EDFFBDE892
:10550000104002480FF0AEBFFC000020F81C002045
:1055100010B5044698B190F9063083B90E480FF0E3
:1055200053FFFEF75BF80D4B01221A70FEF70CF8E3
:105530000B4BE2791A700B4B1868FFF7B7FF0A4B59
:105540000122022000211A700FF062FCBDE8104019
:1055500006480FF087BF00BF441D00200600002052
:10556000321F0020F8000020301F0020281D0020DE
:105570000A460149FDF79EBC00F0030838B50C4807
:105580000FF022FF06F0EEFC60B90A4C0A48012534
:10559000257006F07BFB2078294606F0CFF80448FA
:1055A0000FF060FFBDE8384004480FF05BBF00BF5C
:1055B000981E0020B400002050000020801E002013
:1055C00006F084BD30B599B0FEF760FA044606F0E7
:1055D000AFF9002847D101A8FFF7CCFD52490B785D
:1055E000042B524B12BF0A7811221A70504A1078BD
:1055F00000F0FF05002838D00021117012221A7027
:105600004C4A5968127862F07F020A705A6820B2D8
:1056100000EB400000EB4010FE21B0FBF1F05070B9
:1056200002224549454C0978012988BF00225A7059
:10563000237823B906F0B8FE08B901232370404C43
:10564000637A33B106F060F9012802D120460FF0E9
:10565000BBFE3C4B3548D978002206F07FF9063076
:1056600001D106F04BF919B030BD3748047804F089
:10567000FF02002CD5D02F4A05701278586862F0CE
:105680007F0202705A689DF8040050705A689DF8B5
:10569000050090700A78042A11D15A689DF8060016
:1056A000D0705A689DF8070010715A689DF808007C
:1056B000507106220878052818BF0978B1E70A78E2
:1056C000052A2FD15A689DF80600D0705A689DF8B7
:1056D000070010715A689DF8080050715A689DF8CB
:1056E00009009071BDF80A205868120AC2715A6800
:1056F000BDF80A001072BDF82000000A5072BDF813
:10570000200090729DF82200D0729DF82C0010733A
:105710009DF82F0050730C98000A90730C98D0736A
:105720001022C7E70322C5E73E0000204400002006
:10573000301F00208C1D0020DC1C0020401D00209C
:10574000441D002050000020D41C002013B56846E2
:105750000FF0DCFC1A4B009A19781A4B11B9996BAF
:10576000511AD9631849DC6B0878844281BF012043
:1057700083F82B00D86BD8621448007810B9186CE5
:10578000101A58645C6C0878844281BF012083F849
:105790002B00586CD8620E480078012802BF986C24
:1057A000121ADA64D86C0A78904205D9012283F87B
:1057B0003220DA6C92B21A86064B1B7802B010BD0A
:1057C00003000020781C00200101002002000020BE
:1057D000631C0020EA12002020B1037813B10248B4
:1057E0000FF040BE704700BF741D002008B5104B7D
:1057F0000122002102201A700FF00AFB0D480FF061
:1058000031FE0D4B1B788BB10C4B1A7872B9DB7CD7
:1058100063B90B4B1A68042A9EBF1A6801321A60DA
:105820000021BDE8084010200FF0F2BA08BD00BF0B
:10583000301F0020E01C0020321F0020361F0020F7
:10584000D81C002008B5002140200FF0E1FA074BDA
:105850001B7853B1064B1A78012A06D10021197022
:10586000BDE8084002200FF0D3BA08BD321F002067
:10587000641C0020044B1B78022B03D1002108205C
:105880000FF0C6BA704700BFB4000020044B1B786D
:10589000012B03D0002180200FF0BABA704700BF5F
:1058A0003E00002008B506F066FB80B906F02CF833
:1058B00001280CD1BFF34F8F0549064BCA6802F48B
:1058C000E0621343CB60BFF34F8F00BFFDE708BD1D
:1058D00000ED00E00400FA0538B504460D4607481F
:1058E0004FF40061FDF706FB30B92A462146034814
:1058F000BDE83840FDF704BA38BD00BF00F003082A
:1059000038B5104C237822781809D2B20CD10E4D3C
:105910002A7823789A4206D020781E21FDF7E0FEEF
:105920002378DBB22B7038BD084C23781E2133B1AD
:10593000FDF7D6FE237883F001032370F3E702F02E
:105940000F00F5E706000020341F0020F5000020BE
:105950007047704770470000022810B504461CD0FD
:1059600040282AD001282BD1164B1B7843B3FA20AC
:10597000FEF70EF921464FF0904002F0A9F9124BC4
:105980001870FFF70FFD002120200FF041FA0021D1
:105990000220BDE810400FF03BBA0C4B1B787BB1E6
:1059A000FA20FEF7F5F821464FF0904002F090F90A
:1059B000074B1870FFF70AFDE5E700210420E8E730
:1059C00010BD00BF721C002003000020711C0020CD
:1059D0000200002070B505460C46164605F0A8FFEB
:1059E000034620B370BD4A68F05CD0540133DAB28C
:1059F000A242F8D30F4B0D701B78012B88BF0024F7
:105A00004C700D4C637A33B105F07EFF012802D152
:105A100020460FF0D9FC094B0948D978002205F03F
:105A20009DFF0630DED1BDE8704005F067BF044938
:105A3000DDE700BFDC1C0020441D002050000020DA
:105A400044000020044B1B7823B9044A052101209F
:105A5000FFF7C0BF704700BFDC1C00202D620308A9
:105A600010B5002490B03C22214601A8009428F0F3
:105A7000D9FF454B2022DA7219788DF80010597839
:105A80008DF8011099788DF80210D9788DF80310EF
:105A900019798DF8041059798DF8051099798DF8D8
:105AA0000610D9798DF80710197A8DF80810597AEF
:105AB0008DF80910997A8DF80A108DF80B2021467F
:105AC0000DF10B0258180131007B02F8010F142967
:105AD000F8D193F820208DF8202093F821208DF81C
:105AE000212093F822208DF8222093F823208DF88E
:105AF000232093F824208DF8242093F825208DF876
:105B0000252093F826208DF8262093F827208DF85D
:105B1000272093F828208DF8282093F829208DF845
:105B2000292093F82A208DF82A2093F82B2093F827
:105B300028108DF82B20154A19BB93F8291001F075
:105B4000FF00F1B9107093F82C206AB193F83F2050
:105B500052B10DF12B0100229818013290F82C005F
:105B600001F8010F142AF7D109484FF40061FDF73D
:105B7000C1F920B9064840226946FDF7C1F810B0C6
:105B800010BD01211170DEE7B500002000010020EA
:105B900000F80308014940220FF02EB900F803086D
:105BA00038B5454C207963794D2BC0B26AD1C0EB32
:105BB00000108000A379E2790A2838BF0A204D2A14
:105BC000DBB267D1C3EB03139B004FF47A7202FB85
:105BD00003F594F82C30002B64D194F83F30002B5F
:105BE00060D142F21070FFF745FC344B1868FFF7A4
:105BF0005DFC237A32493348DBB20B70324B012211
:105C00001A70637ADBB2037094F827302F48DBB246
:105C100003700B782E49052B2E4B18BF00221A70EB
:105C200094F828302C4A03EB83035B00DBB213703B
:105C300094F82930294A03EB83035B00DBB213702D
:105C400094F82A30264A0133DBB2DB01138094F842
:105C50002B30244A03EB83035B00DBB21370002379
:105C6000E21892F82C20D2B2CA540133142BF7D187
:105C7000A378012B1FD1E37A202B1CD1BDE838403B
:105C8000FFF7FCBA6379482B0ABF4FF4616363796D
:105C900058438FE7E279482A0ABF4FF46162E279FC
:105CA000534392E74FF47A735843FFF7FFFB2846BC
:105CB000FFF716FC9DE738BDB5000020F800002076
:105CC0003E000020DC1C0020060000200500002013
:105CD000361F0020000100200301002002010020E7
:105CE0003C0000200101002010B590B000213C22B2
:105CF00001A8009128F096FE4022404968460FF026
:105D00007BF89DF800203AB99DF80100072803D1DF
:105D10009DF80210012909D0FFF7A2FE4FF47A7016
:105D2000FDF736FFFFF73CFF10B010BD344B1A7083
:105D3000587099709DF80310D9709DF8041019716E
:105D40009DF8051059719DF8061099719DF807107E
:105D5000D9719DF8081019729DF8091059729DF8B3
:105D60000A1099729DF80B1001F03F01D9720DF1E4
:105D70000B019818013211F8014F0473142AF8D15D
:105D80009DF8202083F820209DF8212083F82120F1
:105D90009DF8222083F822209DF8232083F82320D9
:105DA0009DF8242083F824209DF8252083F82520C1
:105DB0009DF8262083F826209DF8272083F82620AA
:105DC00083F827209DF8282083F828209DF8292093
:105DD00083F829209DF82A2083F82A209DF82B207B
:105DE00083F82B200DF12B0100229818013211F8B5
:105DF000014F80F82C40142AF7D193E700F80308EC
:105E0000B50000201FB5002403A92046039406F026
:105E100097F803A9012006F093F8474B47480094F0
:105E200022464FF4FA710FF071FA454B4548009441
:105E300022464FF4FA710FF069FA434B434800943D
:105E400001224FF4FA710FF061FA414B414800947E
:105E500001224FF4FA710FF059FA3F4B3F4800947A
:105E6000012242F210710FF051FA2046FCF742FF76
:105E700008B1FDF763F93A4B009400224FF4FA6140
:105E800038480FF043FA384A002101200FF07CF81F
:105E9000364A002102200FF077F8354A002104200D
:105EA0000FF072F8334A002108200FF06DF800213E
:105EB000012005F0C7FF304B1C7000F069FD2F4931
:105EC0002F4805F0F3FF2F4805F0E0FE1F480FF0C4
:105ED000C9FA2D4B0021187805F030FCFFF704FFBC
:105EE0002A4A002110200FF04FF8294A00212020D3
:105EF0000FF04AF8274A002140200FF045F8264AC3
:105F0000002180200FF040F8244B25481968254BCC
:105F1000009401220FF0FAF921480FF0A3FA224B66
:105F200022481968224B009401220FF0EFF91F4814
:105F30000FF098FA04B010BD53590008741D0020EA
:105F4000555900085C1D00208D580008441D002094
:105F500001590008281D00204D570008101D002081
:105F600075580008801E002091BA0008C555000829
:105F7000C15500087D550008401D002000000301A8
:105F80006800002050000020B4000020C94E000826
:105F9000214F0008854F000805500008FC00002034
:105FA000F81C002045580008F8000020E01C0020E4
:105FB000ED57000838B5074D00242C60FFF786F92F
:105FC000C820FDF7E5FD28682146FCF7DFF9002829
:105FD000F4D138BD741C002030B50024A5B07C225B
:105FE000214605A8049428F01DFD53238DF8103098
:105FF000012540F20713ADF81230ADF800408DF8DE
:106000001450FDF743FDFE23B0FBF3F000EB40001E
:1060100000EB40108DF815006846FFF79DF99DF8DC
:1060200000309DF80120134314D158238DF8163009
:106030000724802200212F4828F0F4FC224604A9DE
:106040002C4828F085FD2B4A21460120FFF7C2FC91
:1060500025B030BD0E23294601A8CDE901448DF8B5
:106060001630ADF80C40FFF739F901AB03CB224CE9
:106070001B88CDF81B10ADF81F30CDF81700FFF7C7
:1060800025F92068FCF7F0F90A254FF47A7380B2FD
:10609000B0FBF3F0B0FBF5F305FB130030308DF8E7
:1060A00021002068FCF7E0F9642380B2B0FBF3F034
:1060B000B0FBF5F305FB130030308DF822002068AB
:1060C000FCF7D2F980B2B0FBF5F0B0FBF5F305FBBD
:1060D000130030308DF823002068FCF7C5F980B23A
:1060E000B0FBF5F305FB130030308DF824001524C8
:1060F0009FE700BFB01E0020741C0020F0B50446CE
:1061000093B0B6480D46802200210EF07FFE237822
:10611000592B40F01C82052D58D86378443B162B30
:1061200054D8DFE813F065015300490153005201D0
:106130005300530053005300AC0053003801530088
:1061400053005300C30153005300CD0053005300CC
:1061500053001700A578482D11D1A14A1421012020
:10616000FFF738FC41F28830FDF712FD40F6B830F9
:10617000FDF70EFD13B0BDE8F040FFF793BB532DC4
:106180000DD1FFF729FF41F28830FDF701FD934A59
:106190001521012013B0BDE8F040FFF71BBC432DD3
:1061A00016D1002402A88DF8084005F0E7FC8B4AC0
:1061B0004C231370072393709DF80830547001200E
:1061C0004133D07013710521FFF704FC13B0F0BD0B
:1061D000442DFBD1814C592323705A236370A57041
:1061E000FFF7E8FE7F220021601C28F01BFC01263F
:1061F00007232570A370E6702671FDF747FC794DE3
:10620000FE23B0FBF3F000EB4000042300EB401052
:106210006071A3712868FCF727F90A274FF47A7395
:1062200080B2B0FBF3F0B0FBF7F307FB13003030A4
:10623000E0712868FCF718F9642380B2B0FBF3F032
:10624000B0FBF7F307FB1300303020722868FCF72F
:106250000BF980B2B0FBF7F0B0FBF7F307FB1300CC
:10626000303060722868FCF7FFF880B2B0FBF7F3BB
:1062700007FB13003030A07222460B2189E7A37878
:10628000303BDBB2092BA1D8574C584A23702378F6
:10629000DBB25372514A592313704D235370237844
:1062A0000321303301209370FFF794FBFFF7D8FBF5
:1062B0002378002B8AD013B0BDE8F040FDF78EB9EB
:1062C000A578482D29D1454C562318220125237045
:1062D00000260723627168460622A370A271E3714B
:1062E0006670E57025710EF0EBFE009802A9123879
:1062F0000EF06EFF079B26726C336372069B2B4475
:10630000A372059BE372049B2373039B6373029B3D
:10631000A37322460F21284656E7432D7FF456AF3C
:1063200000213C2203A82D4C029128F07BFB02A8FF
:10633000FFF730FC9DF8083063709DF80930A370BA
:106340009DF80A30E3709DF80B3023719DF80C30F6
:1063500063719DF80D30A3719DF80E30E3719DF8C7
:106360000F30257023729DF813509DF81030637222
:106370009DF81130A3722A469DF81230E37205A9E8
:1063800004F10D00257328F0E3FB05F10D01224611
:10639000C9B2012018E7A078392800F28E81303880
:1063A000C0B2FEF7EBFF0D4A237813706378537089
:1063B000A37893700321ECE6A078392800F27D8160
:1063C0003038C0B2FEF7DFFFEDE7A078392800F2E1
:1063D00074813038C0B2FEF7DBFFE4E7B01E002066
:1063E00033620308741C0020DC1C0020B500002070
:1063F000A378303BDAB2092A00F25F81E0783038C6
:10640000C2B2092A00F259812179A1F14802D2B21F
:106410000B2A00F25281AB4D45FA02F2D50700F18A
:106420004C810A224D2902FB03003AD13C235843F8
:106430004FF47A735843A44B1860A44B1860FFF7CD
:1064400035F8A34A2378137063785370A378937058
:10645000E378D3700521237913710120FFF7BAFA8D
:106460009C4B00221A7007225A7001229A70DA702F
:10647000A278303A02EB8201E278303A02EB410234
:10648000D2B21A7122795A71934A1278D2B21A7220
:10649000924A1278D2B25A7213B0BDE8F040FFF7B8
:1064A000DFBA4829C4D14FF46163C0E7A278303A1B
:1064B000D3B2092B00F20181E378303BD9B209292C
:1064C00000F2FB802079A0F14801C9B20B2900F24B
:1064D000F4807C4D45FA01F1C90700F1EE800A21F4
:1064E0004D2801FB02332DD13C2253434FF47A72E5
:1064F00053437B4A13601068FEF7F2FF744A237817
:10650000137063785370A3789370E378D370052188
:10651000237913710120FFF75DFA6E4B00221A7088
:1065200007225A7001229A70DA70A278303A02EB90
:106530008201E278303A02EB4102D2B29A712279BA
:10654000DA71A1E74828D1D14FF46162CDE7502B31
:1065500040F08481022D7FF639AE6178A1F13003DD
:10656000012B3FF633AEA378312B7FF42FAE052DF0
:106570002DD1E378302B40F0A080574A59480023B2
:10658000137013781BB92379303BDBB20370534986
:1065900000230B7003785448DBB2037013784D4A24
:1065A000DBB213720B78DBB25372FFF759FA484B28
:1065B00022781A7062785A70A2789A70E278DA704B
:1065C00022791A71FDF7BCF80521414AE1E5082D51
:1065D00067D1E378462B40F0FF802179A1F13000AC
:1065E000C0B2092800F238816279A2F13003092B88
:1065F00000F23281A679A6F13003092B00F22C813A
:10660000E379A3F13005092D00F2268101EB810128
:106610004900364D203102EB8202C9B25200297086
:1066200020323349D2B22F3E0A70F6B2314A03EB20
:106630008303F6015B00168020332F4ADBB2137010
:10664000244A82F828006379303BDBB282F8293093
:10665000A3792F3BDBB282F82A30E379303BDBB2FF
:1066600082F82B302B782BB90B7803F0FF020BB993
:10667000224B1A70FFF7F4F9154B22781A706278E2
:106680005A70A2789A70E278DA7022791A71627977
:106690005A71A2799A71E279DA71FDF751F80821FD
:1066A00093E7042D54D1E278A2F13003DBB2092B39
:1066B00029D9A2F14103192B22D913B0BDE8F0402A
:1066C000FFF7C0B9DEF7FFFF4C000020F800002004
:1066D000B01E0020B50000203E000020DC1C002081
:1066E000FC00002004000020060000200301002020
:1066F000020100203C0000200101002000010020D8
:10670000A2F13703DBB273480370734B20785970E2
:10671000312199706F491870DA700B786F4ADBB2CB
:1067200013720B78052B6E4B0CBF012100211970E1
:106730006C4B1B78DBB25372FFF792F9FDF700F850
:106740004FF4FA60FDF724FAFFF7ACF804213CE7B8
:106750001D2D3ED9A51C0022604E2846114610F87A
:10676000013F303BDBB2092B98BFB71802F10102A1
:1067700094BF3B7301211E2AF1D100299DD1FEF760
:1067800059FC554B50221A7000225A7007229A70F9
:106790000122DA7003F8042F203415F8012F03F8D2
:1067A000012FAC42F9D14D4B00221A7007225A70CA
:1067B00001229A70DA70474A1278D2B21A72494AA4
:1067C0001278D2B25A721E22DA72FFF749F92321E7
:1067D000FBE6072D7FF671AF0022404802341146D8
:1067E00014F8013F303BDBB2092B98BF851802F14A
:1067F000010294BF2B730121082AF1D100297FF4F3
:106800005CAFFEF789FC344B50221A7007229A7055
:1068100000210122DA70597003F8042F2F4A501812
:106820000131007B082900F1300003F8010FF6D197
:10683000002313700723537001239370D370254BEB
:106840001B78DBB21372274B1B78DBB25372D17209
:10685000FFF706F90D21B8E60021B6E6412B7FF4DB
:10686000B5AC6378432B7FF4B1AC162D7FF4AEAC9E
:106870001D4D621C002312F8011FE9540133142B33
:10688000F9D1FEF707FB194B5B7D012B1DD1134995
:106890000023EA5CC8180133D2B2142B80F82C20F4
:1068A000F7D1104B00221A701B78DBB24B72FFF746
:1068B000D7F8094A631E153413F8011F02F8011BAB
:1068C000A342F9D1044A162163E4064B02221A704E
:1068D000EFE700BF3E000020B01E0020B500002002
:1068E00000010020DC1C0020361F0020840700204F
:1068F00037B504460D46002939D022480EF0B2FDC6
:106900002B78A3B39CB36068237880B3032B0DD09E
:10691000112B2ED0022B2AD16178012927D00B060A
:1069200025D403B0BDE83040FFF7E8BB6378012B06
:1069300007D10078012802D0022800D008B905F05C
:10694000D7F800240DF107008DF8074005F016F97F
:106950000D4A4C231370072393709DF80730547031
:10696000012041330521D0701371FFF733F803B0D4
:1069700030BD6378012BFAD10378044A03F0010398
:106980001370F4E75C1D0020B01E00208C1D002059
:10699000034B0022C3E902220122C3E9002270470F
:1069A0004C1F0020004870474C1F00204FF0B043A0
:1069B00082B0DA6C0243DA64DB6C03400193019B22
:1069C00002B070472DE9F04186B000240220154D39
:1069D0000594FFF7EBFF0420FFF7E8FF124F039445
:1069E0004FF4807601230DEB0001CDE901632846C9
:1069F000032304934FF4005801F04AF801A93846E4
:106A0000CDF8048001F044F822464146384601F0B2
:106A100065F928462246314601F060F9204606B065
:106A2000BDE8F0810004004800080048032810B5C4
:106A30000ED8012810D868B902460B484FF480716F
:106A400001F04CF9002209484FF4005101F046F9D9
:106A5000002010BD0122F0E7002203484FF48071AE
:106A600001F03CF90122EEE700040048000800486C
:106A7000022070470020704701207047002814BF93
:106A800016200F20704700000D48854600F025F8BD
:106A90000C480D490D4A002302E0D458C450043379
:106AA000C4188C42F9D30A4A0A4C002301E013604F
:106AB0000432A242FBD328F01DF8FCF721FBFEE7CD
:106AC0000000012000000020A005002098C8030855
:106AD000A0050020783F0020FEE7704710B5032096
:106AE00000F06EFC01F07CFA064B18600F20FDF7F9
:106AF00045F8044618B9FCF779FC204610BD01247E
:106B0000FBE700BF040100204FF0E022136923F0EF
:106B10000203136170474FF0E022136943F0020350
:106B200013617047014BD3F8900570470070FF1F49
:106B3000014BD3F8940570470070FF1F014BD3F849
:106B4000980570470070FF1F024A536823F0010345
:106B500053607047002004E0024A536823F00203A8
:106B600053607047002004E0024A536823F0040396
:106B700053607047002004E08068C0F380007047D5
:106B8000F7B5002301930446002800F0E980856DE5
:106B900025B9FBF73FFFE56584F8545023689A68F0
:106BA000D00040F1A1809A68D10000F1B480A26DBC
:106BB00042F01002A265E26D42F00102E265012599
:106BC0001846FFF7D9FFA26D02F01002024340F011
:106BD000C980A26D206922F4817242F00202A2658E
:106BE0009A68D2075DD4226BA67E94F82CC0003A36
:106BF00018BF01221703D4E902120A43217E42EA98
:106C00008132617E42EAC13242EA4632002842EADB
:106C10004C02B4BF20F000414FF400113A430A4344
:106C200094F82010012903D1002E76D142F480324D
:106C3000616A21B1A66A01F4E07131430A43D9685F
:106C4000E66C21F4FE3121F4FF711143D96094F810
:106C50003C206168012A01F0404C4CEA060609D14B
:106C6000D4E910273A433243A66C324342EA0C027D
:106C700042F001061F693E4A3A4032431A6121F050
:106C80000042B2F1804F0CD0B1F1004F09D0394E23
:106C9000D6F8082701F4701122F470120A43C6F8DE
:106CA00008275A69666BA16B22F0070232435A61CA
:106CB0005A6922F0700242EA01125A61002835D165
:106CC0009A6A62F00F029A625B6903F007039E42C0
:106CD0003CD10023E365A36D23F0030343F00103DC
:106CE000A365284603B0F0BD9A68234922F01042FC
:106CF00022F0170242F080529A60204A1268B2FBDA
:106D0000F1F2013252000192019A002A3FF44BAF96
:106D1000019A013AF7E7002552E7A16D41F0200101
:106D2000A165E16D41F00101E16581E7B0F5001F6A
:106D3000CAD19A6AE269013A92006FF00F0102F03B
:106D40001C0201FA02F2216E0A43BCE7A36D23F094
:106D5000120343F01003A365E36D43F00103E36501
:106D60000125BEE7A36D43F01003A365F8E700BF5C
:106D700002FCFF1F00200140400D03000401002021
:106D8000F8B54569082D04460E460AD00368DB684D
:106D9000D80705D5A36D43F02003A3650120F8BDF6
:106DA0000425FCF7EDFE074623681A682A4220D026
:106DB000A26D42F40072A265DA6812F4406F14D139
:106DC000A27E92B91A6812070FD51846FFF7D4FEB3
:106DD00020BB5A6822F00C025A60A26D22F4807225
:106DE00022F0010242F00102A265227EFAB10020E7
:106DF000D5E7711CD9D0FCF7C3FEC01BB04201D847
:106E0000002ED1D123681B682B40CDD1A26D84F810
:106E1000543042F00402A2650320C0E7A26D42F0A4
:106E20002002A265E26D42F00102E265DDE70C227C
:106E30001A60DCE70368186C70470000F7B50023A0
:106E4000019390F85430012B044600F0C08005688F
:106E50000269012380F854302846FFF78DFE002890
:106E600040F0AF80D1E90030022822F004027ED049
:106E7000B2F1004FC3F3110E35D1AA6A42EA0E02F5
:106E8000AA628A68686902EA032222F07C4222F040
:106E9000FF0220EA03210A43002B6A611DDA4D4AF2
:106EA0004D4DD2F80817AB4201F0E07043D10D020E
:106EB00013D4D2F8083723F0E073034343F40003FC
:106EC000C2F80837454B1A68454BB2FBF3F20C2366
:106ED00002FB03330193019B53BB0020002384F882
:106EE000543003B0F0BD226E00F01F074FF00F0CBE
:106EF0000CFA07FC6FEA0C0622EA0C0CBEF1000F3C
:106F000011D1C3F38462BA4042EA0C0222668008BF
:106F1000E26901309042B4D8A86AC3F38362BA40F0
:106F200006403243ACE793FAA3F2B2FA82F2EAE700
:106F3000019B013BCEE72B4DAB420BD1C901CCD419
:106F4000D2F8083723F0E073034343F08073C2F8AC
:106F50000837C2E7244DAB42BFD14B02BDD4D2F8B3
:106F6000083723F0E073034343F48003EFE7B2F103
:106F7000004F01BFAA6AC3F311018A43AA62002B22
:106F8000ABDA154813498342D1F8082709D1D1F863
:106F9000083702F0A07223F0E0731A43C1F8082703
:106FA0009BE71048834204D1D1F8083702F440022D
:106FB000F1E70D48834290D1D1F8083702F0C07252
:106FC000E9E7A26D42F02002A265184686E702209A
:106FD00087E700BF00200140001000B0040100203E
:106FE000400D0300004000B8002000B4026838B52E
:106FF00004461046FFF7C0FD08B9002038BD93686D
:10700000990707D4936823F0004323F0170343F054
:1070100010039360FCF7B4FD054623689B685B078B
:10702000EBD5FCF7ADFD401B0228F6D923689B6821
:107030005A07F2D5A36D43F01003A365E36D43F047
:107040000103E3650120D9E773B5002302680193CA
:107050009368DD07044602D5002002B070BD916838
:10706000214B194209D0A36D43F01003A365E36DD2
:1070700043F00103E3650120EFE7936823F0004349
:1070800023F0170343F001039360184BD3F808373C
:1070900018021CD4637E012BDED0FCF771FD144E68
:1070A000054622681368DB07D6D49368D9075FBF0B
:1070B0009368334043F001039360FCF761FD401B8C
:1070C0000228EED923681B68DA07EAD4CBE7094B1C
:1070D000094A1B68B3FBF2F301330193019B002BB8
:1070E000D8D0019B013BF8E7170000800020014049
:1070F000E8FFFF7F04010020400D030038B504467F
:107100000068FFF739FD054620BB94F85430012B89
:1071100020D0012384F854302046FFF795FFB0B902
:10712000A36D226823F4706323F0010343F480739A
:10713000A3651C23E065136084F85400936823F072
:10714000004323F0170343F00403936038BD84F831
:107150005450FBE70220F9E7026838B5936891685C
:107160000446C80701D4002038BD9907FBD49368B2
:1071700003F00503012B19D1936823F0004323F09A
:10718000170343F00203936003231360FCF7F8FC3A
:10719000054623689B68DB07E5D5FCF7F1FC401B3F
:1071A0000228F6D923689B68DA07F2D5A36D43F06D
:1071B0001003A365E36D43F00103E3650120D3E70A
:1071C00070B5044600284BD0836D43F002038365FD
:1071D000FFF70CFF054668B92046FFF7BDFF0546DF
:1071E00008B90123A3652268936823F0104323F0B4
:1071F0001703936023685A6822F4677222F003022F
:107200005A6040F29F321A60D968164A0A40DA6022
:107210001A6922F040421A615A6922F007025A6143
:107220001A6A02F0F0221A625A6A02F0F0225A62D6
:10723000DA6A02F0F022DA629A6A0B4A00269E624B
:10724000D2F8083723F0FE73C2F808372046FBF760
:10725000F5FBE6652666A66584F85460284670BD91
:107260000125FBE700023E830020014010B590F8A5
:107270005430012B044615D0012380F85430FFF719
:10728000B5FE58B92046FFF767FF38B9A36D23F460
:10729000807323F0010343F00103A365002384F806
:1072A000543010BD0220FCE7F7B50023019390F89D
:1072B0005430012B04467FD0012380F85430FFF76F
:1072C0004BFF23689A6812F00102054607D0A36DB0
:1072D00043F01003A365002384F854302DE0A16D22
:1072E000364F21F4817141F00201A165DE68D96851
:1072F00026F4FF4626F07C0621F40041360421F0F6
:107300000301360CD96008209968394041F00041EA
:1073100099609968002913DA019901310191019965
:10732000B1F52E3FF5D3A36D23F0120343F0100304
:10733000A365002384F854300125284603B0F0BD2E
:10734000D3F8B410013801F07F010A44DCD1996808
:107350001A48014041F001019960D3F8B41021F0BE
:107360007F0141EAD202C3F8B4209A68024042F099
:1073700002029A60FCF704FC074623689A68D20769
:1073800008D4DA683243DA60A36D23F0030343F0D4
:1073900001039FE7FCF7F4FBC01B0228EDD923682B
:1073A0009B68D907E9D5A36D43F01003A365E36D8E
:1073B00043F00103E365BFE70225BEE7E8FFFF7F77
:1073C0000749CA6822F4E0620302120403F4E0638E
:1073D000120C134343F0BF6343F40033CB60704798
:1073E00000ED00E0164B30B5DC68C4F30224C4F1B4
:1073F0000703251D042B28BF0423062D4FF0FF355E
:107400008CBF033C002405FA03F321EA0303A540E3
:1074100022EA0502A340002843EA0203ACBF00F1C0
:107420006040084A4FEA0313B8BF00F00F00DBB218
:10743000AABF00F56140135480F8003330BD00BF8F
:1074400000ED00E014ED00E0002807DB044A4109EC
:10745000012300F01F00834042F82130704700BF35
:1074600000E100E000280CDB4309064900F01F00A2
:1074700020330122824041F82320BFF34F8FBFF316
:107480006F8F704700E100E070B5D0E9134565608B
:10749000446D14B1D0E916456560D0E9105404F08C
:1074A0001C060124B4406C60046863608368102B80
:1074B0000BBFA260A160E160E26070BD0268416C38
:1074C000D3B210B5083B1424B3FBF4F30B4CA24227
:1074D00088BF0B4A21F0030199BF01F1804202F5F8
:1074E0000232521807338264064AC26403F01F0353
:1074F000012202FA03F3036510BD00BF0704024036
:107500001C0802408008024038B500285CD00268A0
:107510002E4B9A424FF014014AD82D4B1344B3FB23
:10752000F1F32C499B00C0E91013022380F82530A9
:107530001368056923F4FF4323F070031360D0E957
:10754000024323432B43456911682B4385692B4331
:10755000C5692B43056A2B430B431360FFF7AEFF4E
:10756000B4F5804F04BF002343604368816C03F08F
:107570007F020A60D0E91314013B032B4C601ED834
:10758000154B1649816513449B000121013A01FA0C
:1075900002F200214365C2651960114B5A64002351
:1075A0000122C36380F8243080F82520184638BDB6
:1075B0000C4B1344B3FBF1F30B499B00B3E70023DF
:1075C000C0E91533C365EAE70120F0E7070402408C
:1075D000F8FFFDBF000002403F820010400902405A
:1075E00000090240F8FBFDBF0004024038B5002846
:1075F00041D00268136823F0010313601F4B9A42C5
:107600004FF0140130D81E4B1344B3FBF1F31D4966
:107610009B00C0E91013012403F01C0304FA03F3D8
:10762000002515604B60FFF749FF836C41681D60C2
:10763000D0E913325A604A1E032A06D8124B0B4473
:107640009B0094401D60114B5C640023C363C0E940
:107650001533C0E90B33C0E90D33C36580F825301D
:1076600080F82430184638BD094B1344B3FBF1F3BE
:1076700008499B00CDE70120F5E700BF0704024061
:10768000F8FFFDBF000002403F82001000090240E9
:10769000F8FBFDBF0004024070B590F82450012DA6
:1076A00004463BD090F825600125AE4280F8245076
:1076B0004FF000062CD1022580F825500568C663DE
:1076C0002E6826F001062E60FFF7DEFE036BBBB1CD
:1076D0002B6843F00E032B60A36C1A68D20342BFE1
:1076E0001A6842F480721A60636D1BB11A6842F422
:1076F00080721A602B6843F001032B60002070BD7C
:107700002B6823F004032B602B6843F00A03E2E7A5
:107710008023C36380F824602846F0E70220EEE768
:10772000034640B190F82520022A06D00422C26305
:10773000002280F82420012070470268806C1168C4
:1077400021F00E011160016821F48071016011685F
:1077500021F001011160D3E9100202F01C010122A5
:107760008A404260D3E9132151605A6D32B11168E9
:1077700021F480711160D3E91621516001220020AB
:1077800083F8252083F82400704708B590F8253049
:10779000022B03D00423C363012008BD03681A68C9
:1077A00022F00E021A601A6822F001021A60826C3E
:1077B000136823F480731360D0E9101303F01C02E4
:1077C000012393404B60D0E913325A60436D33B1CB
:1077D0001A6822F480721A60D0E916325A600123C6
:1077E00080F82530002380F82430836B03B198475C
:1077F0000020D2E770B4426C046C036826681D68F0
:1078000002F01C020421914031420FD015F0040F08
:107810000CD01A6892065EBF1A6822F004021A6041
:10782000036B6160002B33D070BC1847022191407C
:10783000314217D015F0020F14D01A68940606D4FE
:107840001A6822F00A021A60012280F82520114AE3
:1078500093428CBF104B114B5960002380F82430A9
:10786000C36ADFE708219140314211D029070FD5C3
:10787000196821F00E011960012303FA02F2626017
:10788000C36380F82530002380F82430436BC9E7B8
:1078900070BC7047800002400004024000000240BB
:1078A0000A4A536943F4802330B55361EFF31084DF
:1078B00072B60023CD58C5500433B3F5807FF9D19B
:1078C0001369DB03FCD484F3108830BD00400058FA
:1078D000064B5A69002ABFBF054A9A6002F18832F6
:1078E0009A60BABF5869C00F002070470040005826
:1078F00023016745044B5A6942F000425A615869B6
:10790000C043C00F704700BF0040005870B5054627
:10791000FCF736F9124E04463369D90313D43369A0
:10792000DA0744BF012232614CF2FA32134011D11E
:107930000B4E306910F480200BD0FCF721F9001BAE
:10794000A842F6D304E0FCF71BF9001BA842E3D3DE
:10795000032070BD024A1361024A01205360F8E718
:10796000004000585C1F00202DE9F041184D98465A
:107970002B78012B06460C46174626D001232B7088
:107980004FF47A7000236B60FFF7C0FFA0B9012E9F
:1079900016D1104A536943F0010353612760BFF3C6
:1079A0006F8FC4F804804FF47A70FFF7AFFF094A75
:1079B000536923EA0603536100232B70BDE8F0816D
:1079C00039462046FFF76CFFEDE70220F6E700BFDF
:1079D0005C1F002000400058054A536923F47E7361
:1079E00043EAC00040F4803040F00200506170472C
:1079F000004000582DE9F041234F3B78012B05460C
:107A000088463FD001233B704FF47A7000237B609F
:107A1000FFF77CFF044688B92B68042B13D11B4A5F
:107A2000536943F4803343F0040353614FF47A7095
:107A3000FFF76CFF0446154B1A681B6800233B7068
:107A40002046BDE8F0814FF0FF33C8F800306E6883
:107A5000D5E901321344B3420AD93046FFF7BCFFDF
:107A60004FF47A70FFF752FF50B1C8F80060044637
:107A7000064A536923F47E7323F002035361DAE765
:107A80000136E5E70224DBE75C1F002000400058D8
:107A90002DE9F04F524C00234FF00F090A6832FADB
:107AA00003F501D1BDE8F08F012505FA03F818EAC6
:107AB000020200F08E804E68032706F003054FEAAD
:107AC000430E07FA0EFC6F1E012F6FEA0C0C32D822
:107AD000876807EA0C0ACF6807FA0EF747EA0A0731
:107AE0008760476827EA0808C6F300179F4047EAFF
:107AF00008074760C76807EA0C088F6807FA0EF79F
:107B000047EA0807022DC76017D14FEAD30800EBF8
:107B1000880803F0070AD8F820704FEA8A0A09FAA1
:107B20000AFB27EA0B0B0F6907FA0AF747EA0B076C
:107B3000C8F8207001E0032DDCD1076805FA0EF5C6
:107B400007EA0C073D4316F4403F056041D023F09F
:107B5000030707F1804707F5803703F0030CBD6882
:107B60004FEA8C0C4FF0070E0EFA0CFEB0F1904F5E
:107B700025EA0E0E2FD01B4DA8422ED005F58065AC
:107B8000A84214BF0725022505FA0CF545EA0E05A3
:107B9000BD602568D74316F4801F0CBF3D401543D8
:107BA0002560656816F4001F0CBF3D4015436560F5
:107BB000D4F8805016F4803F0CBF3D401543C4F804
:107BC0008050D4F88450B60354BF3D401543C4F8E8
:107BD0008450013362E70025D6E70125D4E700BFD2
:107BE0000008005800040048374A2DE9F04F0023F0
:107BF0004FF0010A4FF0070B4FF00F0931FA03F471
:107C000001D1BDE8F08F0AFA03FC1CEA010654D04A
:107C100023F0030404F1804404F5803403F00307E7
:107C2000A568BF000BFA07F8B0F1904F08EA050EFF
:107C300045D0264DA84244D005F58065A8420CBF2A
:107C400002250725BD40754517D1D2F8805025EA99
:107C50000605C2F88050D2F8845025EA0605C2F81D
:107C60008450156825EA06051560556825EA06055D
:107C70005560A56825EA0805A560056803265C002F
:107C800006FA04F423FA06F6254300EB860605609F
:107C900003F00705376AAD0009FA05F527EA05077D
:107CA0003762856825EA04058560456825EA0C0584
:107CB0004560C56825EA0404C46001339EE70025D9
:107CC000C0E70125BEE700BF0008005800040048D7
:107CD0000369194214BF0120002070470AB1816175
:107CE000704781627047436901EA030221EA030198
:107CF00041EA024181617047044AD168014208B5F6
:107D000002D0D060FDF728FE08BD00BF0008005873
:107D1000024A136843F480731360704700040058EC
:107D20000D4B10B55B690C4628B99A0507D500F0D4
:107D300027F820B110BD9B0501D400F019F8074ABF
:107D40001369012C23F00403136101D130BFF1E763
:107D500040BF20BF20BFEDE70004005800ED00E069
:107D6000024B186800F4C060704700BF0004005860
:107D7000024A136843F480431360704700040058BC
:107D80000C4A136823F4804313600B4B1B683221A9
:107D90004B430A49B3FBF1F35169890500D533B967
:107DA000536913F4007F14BF032000207047013B88
:107DB000F2E700BF000400580401002040420F0019
:107DC0000B4A136823F0070343F002031360094BC7
:107DD0001A69012842F004021A6105D130BF1A69FC
:107DE00022F004021A61704740BF20BF20BFF6E7AF
:107DF0000004005800ED00E04FF0B0431868C0F3F5
:107E0000404070474FF0B0431868C0F340007047DF
:107E10004FF0B042536823F47F4343EA002353609A
:107E200070474FF0B0431868C0F3406070470000DF
:107E30007FB54FF0B0432C4AD3F80831C0F303109C
:107E400003F00F0352F82040284A52F82330B4FBC5
:107E5000F3F4FFF785FF264B054693E80700B5F5D9
:107E6000007F04AB03E9070010D0224B9C4218D3DB
:107E700003F5B70303F67F539C4229D903F5741326
:107E800003F510639C4225D802230BE01A4B9C4259
:107E900007D91A4B9C421BD903F5370303F5D85376
:107EA000F0E7002304AA02EB830353F80C4C144DB3
:107EB0002B6823F0070323432B60FBF761FE064684
:107EC0002B6803F007039C4206D1002004B070BD6C
:107ED0000123E7E70024EAE7FBF752FE801B0228B4
:107EE000EED90320F2E700BF48620308A862030846
:107EF00010200308C0CF6A00BFEA21013F9334027B
:107F0000004000584FF0B04310B59A68D96812F09D
:107F10000C0205D00C2A4AD101F00303012B51D1E8
:107F20004FF0B0412B480B6813F0080306D00B68E4
:107F300013F0080337D1D1F8941007E00C68240738
:107F400056BFD1F894300968C3F3032350F82330A7
:107F5000002A0CBF184600204FF0B0418A6802F09A
:107F60000C020C2A1ED1CA6802F00302022A2ED08B
:107F7000032A06D10B68184A13F4801F174B18BF49
:107F800013464FF0B042D068D168D268C0F30620E3
:107F90005843C1F302130133B0FBF3F0530F013325
:107FA000B0FBF3F010BD0B68C3F30313CEE7042A54
:107FB00005D0082A06D11B6813F4801305D00648A3
:107FC0000023C9E700231846C6E70448C4E7024B6C
:107FD000D7E700BF486203080024F4000048E80126
:107FE00008B5FFF78FFF4FF0B043044A9B68C3F317
:107FF000031352F82330B0FBF3F008BDA862030866
:108000002DE9F0410446002853D04FF0B0439D685D
:10801000DE6803689B0605F00C0506F0030668D5CC
:10802000026A1DB10C2D46D1012E44D1002A40D048
:108030004FF0B043A16A1A68170756BFD3F89430BF
:108040001B681B0903F0F00399421FD90846FFF78C
:10805000EFFE00282DD14FF0B042136843F0080323
:1080600013601368A16A23F0F0030B431360606A86
:10807000FFF7CEFEFFF7B4FFAB4B1860AB4B1868B1
:10808000FBF77CFD002834D0BDE8F0814FF0B04212
:10809000136843F008031360136823F0F0030B43E5
:1080A0001360606AFFF7B4FE0846FFF7C1FE0028C0
:1080B000E0D00120E8E74FF0B043002A54D01A681E
:1080C00042F001021A60FBF75BFD0746FFF79AFEDC
:1080D000002842D04FF0B042136843F00803136009
:1080E0001368A16A23F0F0030B431360606AFFF783
:1080F0008FFE2368D80748D42368990700F18C8045
:1081000023681E0740F1FA80A3694FF0B046002BA8
:1081100000F0E180D6F89430E16903F0100291425A
:1081200000F0C48003F00302022AC2D0D80740F155
:10813000B380D6F8943023F00103C6F89430FBF7EF
:108140001FFD0746D6F89430990740F1A580FBF74C
:1081500017FDC31B112BF5D904E0FBF711FDC01B64
:108160000228B3D903208FE71A6822F001021A60AF
:10817000FBF706FD0746FFF745FE0028B9D0FBF7E1
:10818000FFFCC01B0228F6D9ECE7082D03D00C2D0C
:1081900005D1032E03D16368002BADD189E74FF0E1
:1081A000B043A1681A6822F480120A431A60626818
:1081B000B2F5803F10D11A6842F480321A60FBF7A2
:1081C000DFFC0746FFF718FE002895D1FBF7D8FC27
:1081D000C01B6428F6D9C5E7B2F5041F04D11A689C
:1081E00042F400121A60E6E7196821F48031196040
:1081F000196821F400111960002AE0D1FBF7C0FCD6
:108200000746FFF7F9FD00283FF476AFFBF7B8FC0F
:10821000C01B6428F5D9A5E7042D236903D00C2DD4
:108220000ED1022E0CD1002B3FF443AF4FF0B042E1
:108230006169536823F0FE4343EA016353605FE7DB
:108240004FF0B046BBB1336843F480733360FBF743
:1082500097FC074633685A0505D4FBF791FCC31B0E
:10826000022BF7D97EE77368626923F0FE4343EA85
:108270000263736044E7336823F480733360FBF771
:108280007FFC074633685B057FF53AAFFBF778FC68
:10829000C31B022BF6D965E74FF0B042E169D2F873
:1082A000943023F010030B43C2F894304FF0B047E2
:1082B000D7F8943043F00103C7F89430FBF760FC23
:1082C0000646D7F894309A0718D4FBF759FC831B5D
:1082D000112BF6D946E7D6F8943023F00103C6F8FF
:1082E0009430FBF74DFC0746D6F894309B0705D534
:1082F000FBF746FCC31B112BF6D933E7236858075D
:1083000054D50B4F3B68D90514D4FFF701FDFBF79B
:1083100037FC06463B68DA050CD4FBF731FC831BBF
:10832000022BF7D91EE700BF04010020080100203E
:1083300000040058E3684FF0B046002B58D023F0FB
:108340008003052B02BFD6F8903043F00403C6F833
:1083500090304FF0B046FBF713FCD6F8903043F066
:1083600001030746C6F8903041F28838D6F89030BD
:108370009B0705D4FBF704FCC31B4345F6D9F1E684
:10838000E36823F00403812B1BD1FBF7F9FBD6F83C
:10839000903043F08003C6F8903007464FF0B04667
:1083A00041F28838D6F89030180504D5E36A002BDE
:1083B0004AD1002068E6FBF7E3FBC01B4045F1D93A
:1083C000D0E6FBF7DDFBD6F8903023F08003C6F84B
:1083D000903007464FF0B04641F28838D6F89030DA
:1083E0001905E3D5FBF7CCFBC01B4045F6D9B9E630
:1083F000FBF7C6FBD6F8903023F080030746C6F89B
:10840000903041F28838D6F890301A0516D4FBF730
:10841000B7FBD6F8903023F00103C6F8903007463A
:108420004FF0B04841F28836D8F890309B07BDD560
:10843000FBF7A6FBC31BB342F6D993E6FBF7A0FB01
:10844000C01B4045DFD98DE60C2D4ED0022B4FF0DE
:10845000B0431A6822F080721A6033D1FBF790FBA8
:108460000546FFF7DEFC38BBD4E90C314FF0B042D3
:108470000B43D0682D4901400B43E16B0B43216C4A
:108480000B43616C0B43A16B43EA0123D360136878
:1084900043F080731360D36843F08053D360FBF7DD
:1084A0006FFB0446FFF7BDFC002882D1FBF768FB99
:1084B000001B0A28F6D955E6FBF762FB401B0A2889
:1084C000CFD94FE6FBF75CFB0446FFF7AAFC30B9B7
:1084D0004FF0B042164BD1680B40D36069E7FBF711
:1084E0004FFB001B0A28F0D93CE6012B3FF4E1AD1D
:1084F0004FF0B043D868236B00F003029A427FF438
:10850000D8AD626B00F0700393427FF4D2ADA26BE2
:1085100000F4FE43B3EB022F7FF4CBAD636C00F0AD
:108520006040C01A18BF0120AEE500BF8C80C111A9
:10853000FCFFFEEE2DE9F0410D46044610B9012086
:10854000BDE8F081684E336803F007038B4216D311
:1085500023689A0727D54FF0B047A268BB6823F07D
:10856000F0031343BB60FBF70BFB0646BB68DB0362
:1085700019D4FBF705FB831B022BF7D911E03368F5
:1085800023F007030B433360FBF7FAFA074633681F
:1085900003F00703AB42DBD0FBF7F2FAC01B022863
:1085A000F5D90320CCE72368580617D54FF0B0471C
:1085B0006269D7F8083123F00F0343EA1213C7F8B2
:1085C0000831FBF7DDFA0646D7F80831D90305D4A0
:1085D000FBF7D6FA831B022BF6D9E2E723685A078A
:1085E00013D54FF0B047E268BB6823F4E063134350
:1085F000BB60FBF7C5FA0646BB689B0305D4FBF7D7
:10860000BFFA831B022BF7D9CBE72368180714D5D1
:108610004FF0B0472269BB6823F4605343EAC203BA
:10862000BB60FBF7ADFA0646BB68590305D4FBF700
:10863000A7FA831B022BF7D9B3E72368DA070FD415
:10864000294C236803F00703AB4239D8FFF7C8FC75
:10865000264B1860264BBDE8F0411868FBF78EBA30
:108660006268022A1DD1FFF7C7FB00283FF467AFFD
:108670004FF0B04641F28838B36823F00303134348
:10868000B360FBF77DFA0746B368626803F00C033A
:10869000B3EB820FD4D0FBF773FAC01B4045F3D97C
:1086A0007FE7032A02D1FFF7BCFBDEE712B9FFF731
:1086B000A9FBDAE74FF0B0431B685B05D8D43EE76F
:1086C000236823F007032B432360FBF759FA064680
:1086D000236803F00703AB42B8D0FBF751FA801BC5
:1086E0000228F5D95DE700BF0040005804010020D2
:1086F0000801002008B5FFF773FC4FF0B043044AAF
:108700009B68C3F3022352F82330D84008BD00BF52
:108710008862030808B5FFF763FC4FF0B043044AD2
:108720009B68C3F3C22352F82330D84008BD00BF72
:10873000886203084FF0B043D3F89000C0F34000C4
:1087400070474FF0B0410209D1F8883002F47F221F
:10875000000123EA020300F47F200343C1F88830BC
:1087600070474FF0B041020CD1F88830120423EA70
:10877000020343EA0040C1F8880070470368DA0347
:1087800070B5044639D5FFF7C3FAFBF7F9F9614E26
:1087900005463368DB0532D54FF0B043616BD3F843
:1087A000902002F4407291421DD0D3F89010D3F87B
:1087B000902042F48032C3F89020D3F8902021F426
:1087C000407022F480328D07C3F89020C3F89000E7
:1087D00009D5FBF7D5F941F288360546FFF7AAFF20
:1087E000012840F090804FF0B042616BD2F8903099
:1087F00023F440730B43C2F89030002605E0FBF7EA
:10880000BFF9401B0228C4D903262568E8070AD50A
:108810004FF0B0416268D1F8883023EA124392B237
:108820001343C1F88830A9070AD54FF0B041A268B8
:10883000D1F8883023EA124392B21343C1F888304A
:10884000AA0609D54FF0B0422169D2F8883023F446
:1088500040630B43C2F88830AB0502D5206AFFF7AE
:1088600080FF680502D5606AFFF77BFF290502D506
:10887000A06AFFF776FF6A0602D56069FFF761FF1D
:108880002B0602D5A069FFF75CFFE80502D5E06979
:10889000FFF757FFE90610D54FF0B042E168D2F874
:1088A000883023F440730B43C2F88830B1F5807FE1
:1088B00002BFD36843F08073D3602A040ED54FF013
:1088C000B042216BD2F8883023F040430B43C2F80A
:1088D000883019B9D36843F08073D3606B0410D526
:1088E0004FF0B042E16AD2F8883023F040530B4396
:1088F000B1F1005FC2F8883003D1D36843F480330C
:10890000D360304670BDFBF73BF9401BB0427FF6A9
:1089100065AF79E70004005830B590F82C30012B92
:1089200002464FF0020022D0174B82F82D00CA24D5
:10893000012582F82C505C6253245C62B1F5807F83
:10894000146B996914D121F488519961596C24F000
:10895000010421F0004159641463DD650A4BFF21D5
:1089600059620020012382F82D3082F82C0030BD9E
:1089700021F408519961D96C24F0020421F00041DE
:10898000D9641463D865E9E70028004070B50B4E40
:10899000036B756D1D40EA07044603D50123F3659B
:1089A000FBF777FBAB0704D50223F365204600F005
:1089B000C9F9012384F82D3070BD00BF00280040A4
:1089C00038B50A4CE36823F02003E360FBF7D8F8DE
:1089D0000546E3689B0601D5002038BDFBF7D0F8BB
:1089E000401BB0F57A7FF4D90320F6E70028004059
:1089F000F8B5114DEC6814F0400406461AD1EB6846
:108A000043F08003EB60FBF7BBF823460746EC68B6
:108A100014F0400401D1032B01D11846F8BDFBF737
:108A2000AFF8C01BB0F57A7F234684BF032386F8D6
:108A30002D30ECE70023F0E70028004038B50F4C5C
:108A4000E36823F08003E360A3699B06054606D430
:108A5000FFF7B6FF10B1032085F82D0038BDA369DC
:108A600023F02003A361FFF7ABFF10B1032085F8CB
:108A70002D00A36943F02003A361EFE70028004025
:108A800038B5044600284BD090F82D3003F0FF0293
:108A90001BB980F82C20FAF78DFB0223214D84F8B6
:108AA0002D30EB68DB0636D4CA236B6253236B622E
:108AB0002046FFF79DFF10B1FF236B6238BDAB6905
:108AC00023F08E6323F04003AB6121696368AA69D8
:108AD0000B431343A2691343AB61D4E9022343EA76
:108AE00002432B61D4E90931EA680B4322F4F852BE
:108AF0001343EB602046FFF7A1FF0028DCD1D4E947
:108B00000713AA690B4322F06042134362691343BF
:108B1000AB61FF236B62012384F82D300020CDE789
:108B20000120CBE7002800400023092803D840EAB1
:108B30000310C0B270470A380133C0B2F5E7000035
:108B40002DE9F04790F82C30012B05464FF002003C
:108B500069D0012385F82C304E4B85F82D00DE6856
:108B600006F44076B6F5807F78D04C69087891F8A5
:108B7000019091F802A091F82470002A55D19B69C8
:108B800013F0400308BFCB70FFF7CEFF8046484686
:108B9000FFF7CAFF02465046FFF7C6FF8146384638
:108BA000FFF7C2FF0B6ACF78234343EA875343EAB8
:108BB000090343EA084343EA022343EA0063354AD0
:108BC000CA205062532050628C6A8869B4F5807F55
:108BD000946945D124F4885494610124D465B6F590
:108BE000807F09BFCB6913640343536418BF50648B
:108BF000284B4A681A672A6B42F001022A639A6975
:108C000042F488529A61244AD2F8803043F4003307
:108C1000C2F880301F4BFF225A620020012385F8E2
:108C20002D3085F82C00BDE8F087B4F1803F07D0E7
:108C3000B4F5000F04D09B6913F0400308BFCB705C
:108C40000B6ACA781C4344EA0A0444EA004343EA34
:108C5000092343EA825343EA0763B0E70023AEE700
:108C600024F4085494610224D465B6F5807F09BFCA
:108C7000CB6993640343D36418BFD064054B4A683F
:108C80005A672A6B42F002022A639A6942F4085238
:108C9000B8E700BF002800400008005890F82C20DA
:108CA000012A03464FF0020012D00A4A83F82D0031
:108CB000CA21516253215162916941F020019161B1
:108CC000FF2151620020012283F82D2083F82C001F
:108CD000704700BF0028004090F82C20012A03466E
:108CE0004FF0020019D00D4A83F82D00CA215162BD
:108CF0005321516291690A4841F080019161D0F895
:108D0000801041F48021C0F88010FF2151620020C2
:108D1000012283F82D2083F82C00704700280040A2
:108D200000080058064B5A6D520610B5044603D58C
:108D30004022DA65FBF7B0F9012384F82D3010BD2D
:108D4000002800407047890001F1804101F5314160
:108D50000A607047890001F1804101F531410868DE
:108D6000704700002DE9F3471F46894690460446A8
:108D7000FAF706FF0A9D3D442D1AFAF701FF264B2C
:108D80001E68C6F3CB366E4382460196226893680E
:108D900039EA03030CBF01230023434501D100201E
:108DA0002EE07B1CF3D0FAF7EBFEA0EB0A00A84202
:108DB00029D323685A6822F0E0025A606268B2F54B
:108DC000827F0AD1A268B2F5004F02D0B2F5806F5F
:108DD00003D11A6822F040021A60A26AB2F5005F5D
:108DE00007D11A6822F400521A601A6842F400523D
:108DF0001A60012384F85D30002384F85C3003207E
:108E000002B0BDE8F087019A019B002A03F1FF330D
:108E1000019308BF1546B9E7040100202DE9F74F7B
:108E2000994600238DF80330044688461746FAF722
:108E3000A7FE0C9D4D442D1AFAF7A2FE2C4BD4F838
:108E400000B01E6823235E43360D6E4382460196B2
:108E50002268936803EA0803BB4201D100203AE08C
:108E6000B8F5C06F07D137B99BF80C30DBB28DF87D
:108E700003309DF80330B9F1FF3FEAD0FAF780FEE6
:108E8000A0EB0A00A84229D323685A6822F0E00226
:108E90005A606268B2F5827F0AD1A268B2F5004FCB
:108EA00002D0B2F5806F03D11A6822F040021A6036
:108EB000A26AB2F5005F07D11A6822F400521A6064
:108EC0001A6842F400521A60012384F85D300023CE
:108ED00084F85C30032003B0BDE8F08F019A019B59
:108EE000002A03F1FF33019308BF1546B0E700BF26
:108EF0000401002073B50B4600920D4616464FF450
:108F0000C05100220446FFF789FF024630B1236EAC
:108F100043F020032366032002B070BD00962B4669
:108F200080212046FFF71EFF02460028EFD1009661
:108F30002B464FF4C0612046FFF770FF0028EBD0AE
:108F4000E5E74368B3F5827FF7B504460E4617465A
:108F50000BD18368B3F5004F02D0B3F5806F04D115
:108F60002268136823F04003136000973346002201
:108F700080212046FFF7F6FE054628B1236E43F018
:108F800020032366032514E06368B3F5827F10D1C4
:108F9000A368B3F5004F02D0B3F5806F09D10097F5
:108FA000334600224FF4C0612046FFF737FF002808
:108FB000E4D1284603B0F0BDF8B5044600287ED0C1
:108FC000436A002B50D14268B2F5827F00D0C36162
:108FD00094F85D3003F0FF0223B984F85C2020464A
:108FE000FAF74EF92268E068022384F85D301368CE
:108FF000B0F5E06F23F0400313604FF0000337D962
:109000001D46B0F5706F18BFA362A7686368A169B9
:10901000A66A07F4044703F482733B43276907F009
:1090200002073B43676907F001073B4301F4007700
:109030003B43E76907F038073B43276A07F080079F
:109040003B4306F400573B43B6F5005F136014D171
:10905000236B8BBBB0F5E06F0DD90223236313683C
:1090600043F40063136008E00023C0E90433AFE772
:109070004FF48055C7E701232363636A676B03F0EE
:10908000100307F0080700F470603B43090C03432A
:1090900001F004010B432B43B6F5005F536004BF9E
:1090A000A38D1361D36923F40063D36100200123EE
:1090B000206684F85D30F8BD022BDED1CFE70120B9
:1090C000F9E7000070B5044690F85C00012800F054
:1090D000CF80012084F85C0094F85D006668012868
:1090E000C5B20AD0B6F5827F40F0C080A0680028E3
:1090F00040F0BC80042D40F0B980002951D0002AF6
:109100004FD0002B4DD094F85D00A16304281CBF04
:10911000052084F85D0000202066C4E91300A06AE1
:10912000E387B0F5005F2168A3872264A4F8443088
:10913000A4F8463007D1086820F400500860086899
:1091400040F400500860486820F4C0404860E0687F
:10915000B0F5E06FA06D29D94B6823F480534B60C4
:1091600094F85D30434E444D042B444B18BF1D46CC
:10917000434B18BF3346C0E90B35424B43630023D2
:109180008363B4F846300C319BB2FEF785FA034690
:10919000002848D0236E43F010032366012384F88F
:1091A0005D300120002384F85C3070BD4D6845F4CB
:1091B00080554D60656DAD69B5F5806F0AD113F0CE
:1091C000010F4B681ED123F480434B60E38FC3F340
:1091D0004E03E3878369B3F5806FC1D14B6823F4F5
:1091E00080534B60B4F8463013F0010F4B6811D137
:1091F00023F400534B60B4F84630C3F34E03A4F895
:109200004630ADE743F480434B60E38FC3F34E0336
:109210000133DEE743F400534B60B4F84630C3F348
:109220004E030133EBE72268606D516841F00101A4
:109230005160C0E90B33C0E90D33E38FA16B9BB2E2
:109240000C32FEF729FA0028A4D123681A685206C6
:109250005EBF1A6842F040021A605A6842F020026B
:109260005A605A6842F002025A609BE7022099E76E
:1092700002209AE7BD9300088D9200089992000899
:10928000C7920008A59200087047704708B5806A29
:10929000FFF7FBFF08BD704708B5806AFFF7FBFFCB
:1092A00008BD7047806A026808B5536823F003035D
:1092B0005360036E43F010030366012380F85D30B2
:1092C000FFF7EFFF08BD7FB5064600230393846ACE
:1092D0008DF80B30FAF754FC33681B689A06054684
:1092E00068D42268536823F020035360A36AB3F55F
:1092F000005F13D101220090642311462046FFF73E
:1093000031FD18B1236E43F002032366E36826683B
:10931000B3F5E06F2ED9F3680393039BA26823682B
:10932000002A43D16268B2F5827F3FD15A6822F0A9
:1093300003025A6064212A462046FFF702FE08B164
:10934000202323660023A4F846302268012384F8F2
:109350005D309368DB0606D5236E43F00203236677
:109360004FF6EF739360236E23B32046FFF799FF08
:1093700004B070BD337BDBB28DF80B309DF80B3041
:10938000236B022BCAD1012200956423114620468B
:10939000FFF7E8FC18B1236E43F002032366337B2A
:1093A000DBB28DF80B309DF80B30B7E75A6822F02E
:1093B0000102BEE72046FFF767FFD9E77FB5064603
:1093C00000230393846A8DF80B30FAF7D9FB3368D6
:1093D0001B68990605465ED42268536823F0200373
:1093E0005360A36AB3F5005F1BD1E368B3F5E06F88
:1093F0003ED1236B012B3BD1009064234FF40072CC
:109400004FF4C0612046FFF709FD18B1236E43F009
:109410000203236623681B7BDBB28DF80B309DF8BB
:109420000B302A4664212046FFF764FD18B1236EF5
:1094300043F02003236623685A6822F003025A602F
:109440000022E287A4F84620012284F85D209A6871
:10945000D20606D5226E42F0020222664FF6EF7265
:109460009A60236EBBB12046FFF71BFF04B070BDAE
:10947000009564234FF480624FF4C0612046FFF7EB
:10948000CDFC18B1236E43F0020323662368DB682A
:109490000393039BC5E72046F9F70EFAE6E70000C1
:1094A000036830B559689A6802F04105012D85B00E
:1094B000044606D14D0604D5C36C05B0BDE8304066
:1094C0001847950704D5080602D5236D2046F4E712
:1094D00012F4B07F59D08D0657D550060FD594F8A9
:1094E0005D0003284FF0000549D0206E40F00400D5
:1094F00020660095D86800909868009000989506BE
:109500000CD5206E40F00100206600200290986883
:109510000290186820F0400018600298D00508D525
:10952000226E42F008022266002203929A68039299
:10953000039A226E4AB35A6822F0E0025A6001226E
:1095400084F85D208A0722D05A68A06D22F00302B9
:109550005A6040B1104B8363FEF717F918B1236EC0
:1095600043F040032366606D78B10B4B8363FEF7D5
:109570000CF950B1236E43F04003236605E00195DA
:10958000DA6801929B680193019B05B030BD2046CB
:10959000FFF787FEF9E700BF9D95000808B5806AD0
:1095A0000023A0F84630C387FFF77BFE08BD00000C
:1095B000034AD2F8903043F40043C2F89030704729
:1095C00000040058034AD2F8903023F40043C2F854
:1095D0009030704700040058074B1A6822F0400290
:1095E0001A6040F441704FF4B85218605A601A681B
:1095F00042F040021A6070470000015837B5054636
:1096000000284ED0837903F0FF046BB1032C0BD0FC
:10961000254B4FF400629A612868FFF7DDFF0024B4
:1096200001232B71AC602FE000236B712846FAF701
:10963000BBF91E4AD2F8903043F48053C2F8903000
:10964000002CE5D102234FF0B042AB71D2F8943038
:1096500023F40043C2F89430154B1B681C214B4384
:10966000DB0C64214B430193019B93B90124AC6053
:10967000FFF79EFF0C4B9A6842F400629A604FF429
:1096800000629A61002CC7D00123AB71204603B061
:1096900030BD019B013B0193D2F894305B04E3D4CD
:1096A000E6E70124F2E700BF000400580008005874
:1096B0000401002037B5174D2B6802461C20434398
:1096C000DB0C6420434314480193019B93B90120B0
:1096D0009060114C21732B681C214B43DB0C6421DF
:1096E0004B430193019B6BB9012090600A4BDB68EF
:1096F00003B030BD019B013B019383689C07E4D517
:109700000020E6E7019B013B0193A368DB07E9D555
:10971000ECE700BF040100200000015837B5184DE8
:109720002B6802461C204343DB0C6420434315484E
:109730000193019BA3B901209060124CFF23237376
:109740002B681C256B43DB0C64256B430193019B49
:1097500073B9012090600B4BDB680B7003B030BD18
:10976000019B013B019383689C07E2D50020E4E75D
:10977000019B013B0193A368DB07E8D5EBE700BF42
:1097800004010020000001580E4B0F491B681822ED
:10979000534382B01B0D6422534301934B69019ADA
:1097A000C3F3800322B902238360012002B0704713
:1097B000019A013A01924A69920701D5002BEDD135
:1097C0000020F3E7040100200004005807B50379E6
:1097D000012B0FD10A4B1B68182253431B0C01931A
:1097E000FFF7F0FE019B013B0193019B002BF9D198
:1097F000FFF7DEFE03B05DF804EBFFF7C5BF00BF67
:1098000004010020F8B51E468379012B1546044655
:109810000F46DAB22DD14379012B2AD002234271AF
:109820008371FFF7D3FF0D212046FFF7CBFEFFF733
:1098300041FF390A2046FFF73DFFF9B22046FFF706
:1098400039FF2E44B5420ED12046FFF7B1FEFFF797
:109850009BFFA06801230038A3714FF0000318BFDD
:1098600001206371F8BD15F8011B2046FFF722FFA8
:10987000E8E70220F6E7F8B51E468379012B154686
:1098800004460F46DAB22FD14379012B2CD0427116
:10989000FFF79CFF1D212046FFF794FEFFF70AFF0C
:1098A000390A2046FFF706FFF9B22046FFF702FF0C
:1098B00000212046FFF7FEFE2E44B5420ED1204681
:1098C000FFF776FEFFF760FFA06801230038A37161
:1098D0004FF0000318BF01206371F8BD29462046F0
:1098E000FFF71CFF0135E8E70220F6E7F8B51F4651
:1098F0008379012B154604460E46DAB22CD1437902
:10990000012B29D04271FFF761FF06F0EF03A3F1AD
:10991000840253425341237131462046FFF752FEE1
:10992000FFF7C8FE2F44AF4210D1FFF741FE842E4F
:1099300002D02046FFF728FFA06801230038A3715A
:109940004FF0000318BF01206371F8BD15F8011B2B
:109950002046FFF7AFFEE6E70220F6E7F8B51E4621
:109960008379012B154604460F46DAB227D1437995
:10997000012B24D04271FFF729FF39462046FFF71B
:1099800021FEFFF797FE00212046FFF793FE2E44AD
:10999000B5420ED12046FFF70BFEFFF7F5FEA0689B
:1099A00001230038A3714FF0000318BF0120637139
:1099B000F8BD29462046FFF7B1FE0135E8E7022051
:1099C000F6E737B50023ADF8043001AA02231221CF
:1099D0000546FFF7C3FFBDF80440022364BA01AA9D
:1099E000A4B219462846FFF781FFE20702D52846B0
:1099F0000AF094FFA30702D528460AF095FF6007F6
:109A000002D528460AF0BAFF210702D528460AF0F7
:109A1000BBFFE20602D528460AF0BCFFA30602D52A
:109A200028460AF0A5FF600602D528460AF082FF04
:109A3000210606D514F4807118BF012128460AF0CA
:109A40007FFFA20502D528460AF08AFF630402D5EB
:109A500028460AF0A5FF03B030BDF8B51E4683794D
:109A6000012B154604460F46DAB227D14379012B64
:109A700024D04271FFF7AAFE0E212046FFF7A2FD77
:109A8000FFF718FE39462046FFF714FE2E44B54274
:109A90000ED12046FFF78CFDFFF776FEA06801236C
:109AA0000038A3714FF0000318BF01206371F8BDA7
:109AB00015F8011B2046FFF7FDFDE8E70220F6E759
:109AC000F8B51E468379012B154604460F46DAB2D7
:109AD0002BD14379012B28D04271FFF777FE1E214D
:109AE0002046FFF76FFDFFF7E5FD39462046FFF7FB
:109AF000E1FD00212046FFF7DDFD2E44B5420ED1E9
:109B00002046FFF755FDFFF73FFEA0680123003810
:109B1000A3714FF0000318BF01206371F8BD2946FF
:109B20002046FFF7FBFD0135E8E70220F6E70000DD
:109B3000036A23F001030362036A70B54468826913
:109B40000D6822F4803222F073022A438D6823F0DC
:109B500002032B43124DA84206D0124EB04203D04E
:109B6000A6F58066B04214D1CE6823F008033343D3
:109B7000A84223F0040306D00B4DA84203D005F5FC
:109B80008065A84205D124F44075D1E905463443E7
:109B90002C43446082614A684263036270BD00BF27
:109BA000002C01400048014000440140036A23F4B6
:109BB00080730362036A426870B5C4690D6824F457
:109BC000803424F073042C438D6823F4007343EA3B
:109BD00005230F4DA8420ED1CD6823F4006343EA5C
:109BE000052323F48063D1E9055622F4405235431E
:109BF00042EA051206E0074DA842F4D005F580655B
:109C0000A842F0D042604A68C461C263036270BD7A
:109C1000002C014000440140036A23F48053036296
:109C2000026A30B54468C3690D6823F0807323F479
:109C3000E64343EA05238D6822F4005242EA0532E6
:109C40000A4DA84207D005F5C055A84203D005F536
:109C50008065A84204D14D6924F4804444EA851407
:109C60004460C3614B680364026230BD002C014054
:109C7000036A23F480330362026A30B54468436D9B
:109C80000D6823F4803323F070032B438D6822F496
:109C9000003242EA05420B4DA84207D005F5C055F7
:109CA000A84203D005F58065A84204D14D6924F48B
:109CB000803444EA0524446043654B68836502624E
:109CC00030BD00BF002C0140036A23F480130362FF
:109CD000026A30B54468436D0D6823F0807323F445
:109CE000E04343EA05238D6822F4001242EA05525C
:109CF0000A4DA84207D005F5C055A84203D005F586
:109D00008065A84204D14D6924F4802444EA852466
:109D1000446043654B68C365026230BD002C01405E
:109D2000704710B5846A626A82420BD1012323779F
:109D3000D2690AB984F83E302046F9F709FE0023BB
:109D4000237710BDA36A834208D102222277DB6900
:109D5000002BF1D1012384F83F30EDE7E36A834221
:109D600008D104222277DB69002BE5D1012384F896
:109D70004030E1E7236B8342DED108222277DB69A2
:109D8000002BD9D1012384F84130D5E7704710B5B5
:109D9000846A636A834207D1012323772046FFF751
:109DA000F5FF0023237710BDA36A834201D102236C
:109DB000F3E7E36A834201D10423EEE7236B834296
:109DC000ECD10823E9E7704710B5846A636A8342DF
:109DD00009D10123237784F83E302046FFF7F3FFB3
:109DE0000023237710BDA36A834205D10223237782
:109DF000012384F83F30F0E7E36A83424FF0010328
:109E000004D10422227784F84030E6E7226B8242B4
:109E100003BF0822227784F8413084F83D30DCE724
:109E20001A4A0368904210B502D0B0F1804F09D1B0
:109E30004C6823F07003904243EA040309D0B0F168
:109E4000804F06D0124A904203D002F580629042C1
:109E500003D1CA6823F4407313434A6923F0800393
:109E6000134303608B68C3620B688362074B98429D
:109E700007D003F5C053984203D003F5806398429E
:109E800001D10B6903630123436110BD002C014024
:109E90000044014010B5044650B390F83D3003F043
:109EA000FF021BB980F83C20F9F738FF0223206835
:109EB00084F83D30211DFFF7B3FF012384F84830BB
:109EC000002084F83E3084F83F3084F8403084F835
:109ED000413084F8423084F8433084F8443084F8C8
:109EE000453084F8463084F8473084F83D3010BD62
:109EF0000120FCE710B5044650B390F83D3003F064
:109F0000FF021BB980F83C20FFF70AFF02232068FC
:109F100084F83D30211DFFF783FF012384F848308A
:109F2000002084F83E3084F83F3084F8403084F8D4
:109F3000413084F8423084F8433084F8443084F867
:109F4000453084F8463084F8473084F83D3010BD01
:109F50000120FCE7036A23F010030362036A4268EE
:109F600070B584690D6824F0807424F4E64444EAF2
:109F700005248D6823F0200343EA05130F4DA84202
:109F80000ED1CD6823F0800343EA051323F040038C
:109F9000D1E9055622F44062354342EA850206E0E3
:109FA000074DA842F4D005F58065A842F0D0426084
:109FB0004A6884618263036270BD00BF002C014067
:109FC0000044014038B590F83C30012B044673D072
:109FD00001200C2A84F83C004ED008D8042A2BD04B
:109FE000082A39D0BAB1002384F83C3038BD102A91
:109FF00052D0142AF7D12068FFF766FE436D0A6934
:10A0000043F400634365436D23F480634365436D0C
:10A0100043EA02234EE02068FFF78AFD83690A695C
:10A0200043F008038361836923F004038361836938
:10A03000134383610020D6E72068FFF78BFF836915
:10A040000A6943F400638361836923F48063836155
:10A05000836943EA0223ECE72068FFF7A7FDC369A1
:10A060000A6943F00803C361C36923F00403C361B1
:10A07000C3691343C361DDE72068FFF7CDFDC36902
:10A080000A6943F40063C361C36923F48063C36155
:10A09000C36943EA0223EDE72068FFF7E9FD436D5A
:10A0A0000A6943F008034365436D23F004034365E5
:10A0B000436D13434365BDE7022097E710B58468FD
:10A0C0000A4324F47F4442EA03222243826010BD03
:10A0D00038B590F83C30012B04464FF0020000F0F8
:10A0E000958084F83D000122206884F83C20856832
:10A0F000474B2B4083600B68602B54D037D8402BE4
:10A100006BD019D8202B0DD00AD833F0100109D00C
:10A11000012384F83D30002384F83C30104638BDDC
:10A12000302BF5D1826822F4401222F070021A43DB
:10A1300042F0070282602BE0502BE9D14A68CD68DB
:10A14000016A036A23F001030362836921F00A01B3
:10A1500023F0F00343EA05130A4383610262836834
:10A1600023F4401323F0700343F057030FE0B3F5DB
:10A17000805F0DD0B3F5005F0CD0702BC8D1CB68D9
:10A18000D1E90121FFF79AFF836843F077038360E9
:10A190000022BDE7CB68D1E90121FFF78FFF83687B
:10A1A00043F48043F3E7036A4D68C96823F0100362
:10A1B00003628269036A22F4704223F0A00343EA37
:10A1C000051342EA013282610362836823F440137B
:10A1D00023F0700343F06703D9E74A68CD68016A4A
:10A1E000036A23F001030362836921F00A0123F06B
:10A1F000F00343EA05130A4383610262836823F490
:10A20000401323F0700343F04703C0E7024685E79D
:10A210008800CEFF036A01F01F0110B501248C40B5
:10A2200023EA04030362036A8A401A43026210BDF0
:10A2300038B50D46082D044611461BD005D85DB132
:10A24000042D14D094F8430008E00C2D15D0102DE7
:10A25000F8D190F8420001E090F83E00A0F1020C25
:10A26000DCF1000040EB0C0050B1022076E090F8E9
:10A270003F00F3E790F84000F0E790F84100EDE789
:10A28000082D1AD007D86DB1042D13D094F84320AF
:10A29000012A19D00CE00C2D27D0102DF6D194F8FE
:10A2A00042000CE094F83E20501E424242415AB90E
:10A2B000012053E094F83F20F6E794F84000421E56
:10A2C000504250410028F3D00029F1D0002BEFD0AC
:10A2D000082D4FF0020256D00AD885B1042D3ED089
:10A2E000042D84F84320E3D13BE094F84100E6E7F5
:10A2F0000C2D5CD0102DF3D184F84220D8E7606A91
:10A3000084F83E203A4AC2623A4A02633A4A4263B9
:10A3100022683432FDF7C0F90028C9D12268D36819
:10A3200043F400732068D36029460122FFF772FFCF
:10A33000324A904250D0324B98424DD003F5806360
:10A34000984249D0B0F1804F4DD182682D4B1340D7
:10A35000062B02D0B3F5803F45D1002038BD84F8EC
:10A360003F20A06A224AC262224A0263224A426312
:10A3700022683832FDF790F9002899D12268D36815
:10A3800043F48063CEE7E06A84F84020184AC26252
:10A39000184A0263184A426322683C32FDF77CF98E
:10A3A000002885D12268D36843F40063BAE7206BA4
:10A3B00084F841200E4AC2620E4A02630E4A42638A
:10A3C00022684032FDF768F900287FF471AF2268F7
:10A3D000D36843F48053A5E7436C904243F40043B1
:10A3E0004364B2D0AEE7036843F001030360B4E70F
:10A3F000239D00088F9D0008C99D0008002C014086
:10A400000044014007000100FFF712BF082938B5DA
:10A4100004460D464FD004D861B1042944D0012030
:10A4200038BD0C29FBD10268006BD36823F480533C
:10A43000D36005E00268406AD36823F40073D360F8
:10A44000FDF7A3F9206800222946FFF7E3FE2A4B17
:10A45000984207D003F5C053984203D003F58063B8
:10A4600098420DD1026A41F211131A4208D1026AD0
:10A4700040F244431A4202BF436C23F40043436456
:10A48000026A41F211131A4208D1026A40F24443AF
:10A490001A4202BF036823F00103036001238DB950
:10A4A00084F83E300020BBE70268806AD36823F45A
:10A4B0008063D360C4E70268C06AD36823F4006392
:10A4C000D360BDE70C2D13D007D8042D0AD0082D7A
:10A4D0000BD0012384F84330E4E7102DF9D184F840
:10A4E0004230DFE784F83F30DCE784F84030D9E7DA
:10A4F00084F84130D6E700BF002C0140FFF786BF4B
:10A5000070B590F83C30012B02464FF0020020D08D
:10A5100082F83D000F4D106843688468A84202BF6E
:10A520004E6823F4700333430E6823F07003334303
:10A53000A842436002D0B0F1804F04D1896824F072
:10A5400080030B4383600123002082F83D3082F8B2
:10A550003C0070BD002C014010B590F83C30012B40
:10A5600002463BD0CB6888681D4C23F440730343FC
:10A57000486823F480630343086823F400630343BB
:10A58000086923F480530343486923F400530343C9
:10A59000086B23F480430343886923F4702343EA60
:10A5A00000431068A04214D1CC6923F080532343A8
:10A5B0008C6A23F4700343EA04530C6A23F080731B
:10A5C00023434C6AC96A23F00073234323F00053EA
:10A5D0000B434364002082F83C0010BD0220FCE7DE
:10A5E000002C0140026852E8003F23F0C00342E81B
:10A5F000003102680029F5D102F1080353E8003F59
:10A6000023F4000302F1080C4CE800310029F3D1D7
:10A610002023C0F88830704710B5026852E8003F28
:10A6200023F4907342E8003102680029F5D10F4C01
:10A6300002F1080353E8003F234002F1080C4CE804
:10A6400000310029F4D1C36E012B07D152E8003F3D
:10A6500023F0100342E800310029F7D12023C0F88D
:10A660008C300023C366436710BD00BFFEFFFFEFC1
:10A67000F8B504461346D4F88850202D32D1F1B1F4
:10A68000EAB1E06FA4F85620A4F854200026212255
:10A69000C4F890602165C4F88820226888B1124F00
:10A6A000C762124F0763124F2832C0E90D76FCF7DC
:10A6B000F3FF30B11023C4F89030C4F88850012063
:10A6C000F8BD236840221A62226802F1080353E8A9
:10A6D000003F43F0800302F1080141E80030002808
:10A6E000F3D1EDE70220EBE7F5A600083DA700084F
:10A6F00049A7000808B50346806A1B681B6813F069
:10A70000200317D1A0F85630026802F1080353E87D
:10A71000003F23F08003083242E80031026800293C
:10A72000F2D152E8003F43F0400342E800310029F3
:10A73000F7D108BDF9F7E4FDFBE7704708B5806A7B
:10A74000FFF7FBFF08BD7047806A38B50468D0F892
:10A750008830D0F88C50A268120606D5212B04D17F
:10A760000023A0F85630FFF73DFFA3685B0606D52F
:10A77000222D04D10023A0F85E30FFF74DFFD0F862
:10A78000903043F01003C0F89030FFF7DCFF38BD85
:10A7900008B5806A0023A0F85E30A0F85630FFF7B5
:10A7A000D2FF08BD704700000368D9691A682DE917
:10A7B000F04140F60F0631429D68044610D18E06E6
:10A7C00040F1978002F0200605F080573E4300F0EC
:10A7D0009080436F002B00F08580BDE8F041184762
:10A7E000AB4EAC482E401040304300F08280CF0783
:10A7F00009D5D00507D501201862D4F8900040F0A3
:10A800000100C4F890008F0709D5E80707D502209A
:10A810001862D4F8900040F00400C4F890004F078C
:10A8200009D5E80707D504201862D4F8900040F055
:10A830000200C4F890000F070BD502F0200030434F
:10A8400007D008201862D4F8900040F00800C4F83F
:10A8500090000E050AD5500108D54FF4006018622B
:10A86000D4F8903043F02003C4F89030D4F89030FE
:10A87000002B37D08B0609D502F0200205F0805559
:10A880002A4303D0636F0BB1204698472668D4F85B
:10A890009020B36802F0280203F0400353EA020557
:10A8A000204621D0FFF7B8FEB3685F0617D52268AF
:10A8B00002F1080353E8003F23F04003083242E866
:10A8C00000310029F3D1D4F8800040B1724B83638A
:10A8D000FCF75BFF30B1D4F88000836B7DE7204646
:10A8E000FFF731FFBDE8F081FFF72DFFC4F890506E
:10A8F000F8E7E06E012840F08980CE0640F18680BE
:10A90000D00640F1838010221A629A6851064BD516
:10A91000D4F8802011684A6892B2002AE2D0B4F8D4
:10A920005C009042DED9A4F85E200A6892062FD41B
:10A9300053E8002F22F4807243E800210029F7D168
:10A9400003F1080252E8002F22F0010203F108008F
:10A9500040E800210029F3D103F1080252E8002F5A
:10A9600022F0400203F1080040E800210029F3D161
:10A970002022C4F88C20E16653E8002F22F0100258
:10A9800043E800210029F7D1D4F88000FCF7C8FE85
:10A9900002232367B4F85E30B4F85C10C91A89B298
:10A9A0002046FFF7FFFE9DE7B4F85E20B4F85E0096
:10A9B000B4F85C1080B292B2002893D0891A89B2A0
:10A9C00000298FD053E8002F22F4907243E8002032
:10A9D0000028F7D1314D03F1080252E8002F2A4038
:10A9E00003F1080646E800200028F4D12022C4F82C
:10A9F0008C206067E06653E8002F22F0100243E8E5
:10AA000000200028F7D102232367C9E7CF0209D528
:10AA10006E0207D54FF4801220461A62BDE8F0415D
:10AA200000F0A0BD08060BD502F0800005F400057B
:10AA3000284305D0A36F002B3FF454AF2046CCE64B
:10AA40004F0611D556060FD553E8002F22F04002CD
:10AA500043E800210029F7D12023C4F88830A167FA
:10AA60002046F9F74DFC3DE70D0206D5500004D510
:10AA70002046BDE8F04100F077BDCB017FF532AF55
:10AA8000002ABFF62FAF2046BDE8F04100F06BBDB5
:10AA9000010000102001000491A70008FEFFFFEF55
:10AAA000D0F88C20B0F86010222A08B5036855D180
:10AAB0005B6A826D0B401370836D01338365B0F860
:10AAC0005E30013B9BB2A0F85E30B0F85E309BB2C6
:10AAD000002B42D1026852E8003F23F4907342E811
:10AAE000003103680029F5D103F1080252E8002F74
:10AAF00022F0010203F1080C4CE800210029F3D1F7
:10AB00002022C0F88C20184A41679342016705D182
:10AB1000C26E012A0ED0F9F701FC1EE05A6811023C
:10AB2000F6D553E8002F22F0806243E80021002987
:10AB3000F7D1EDE70022C26653E8002F22F01002A1
:10AB400043E800210029F7D1DA69B0F85C10D20699
:10AB500044BF10221A62FFF725FE08BD9A6942F031
:10AB600008029A61F9E700BF00800040D0F88C200D
:10AB7000B0F86010222A08B5036852D15A6A114011
:10AB8000826D22F8021B8265B0F85E20013A92B213
:10AB9000A0F85E20B0F85E2092B2002A40D153E8BF
:10ABA000002F22F4907243E800210029F7D103F12D
:10ABB000080252E8002F22F0010203F1080C4CE8D1
:10ABC00000210029F3D12022C0F88C20174A4167C8
:10ABD0009342016705D1C26E012A0ED0F9F79EFBA0
:10ABE0001EE05A681102F6D553E8002F22F0806269
:10ABF00043E800210029F7D1EDE70022C26653E8BF
:10AC0000002F22F0100243E800210029F7D1DA6971
:10AC1000B0F85C10D20644BF10221A62FFF7C2FDE2
:10AC200008BD9A6942F008029A61F9E70080004085
:10AC30002DE9F84F0368B0F86060D3F81CB01F68C6
:10AC40009D68D0F88C20222A044640F0B980B0F8E4
:10AC5000683043B1DFF87491DFF874A14FF0000859
:10AC60001BF0200F20D1B4F85E309BB2D3B1B4F802
:10AC700068209A4216D9226802F1080353E8003F7F
:10AC800023F08053083242E8003122680029F2D1D3
:10AC9000504B636752E8003F43F0200342E8003125
:10ACA0000029F7D1BDE8F88F2368A26D5B6A3340B5
:10ACB0001370A36D0133A365B4F85E30013B9BB202
:10ACC000A4F85E302368D3F81CB01BF0070F2ED019
:10ACD0001BF0010F09D0F90507D501221A62D4F83B
:10ACE000902042F00102C4F890201BF0020F09D01E
:10ACF000EA0707D502221A62D4F8902042F0040233
:10AD0000C4F890201BF0040F09D0E80707D50422EF
:10AD10001A62D4F8903043F00203C4F89030D4F8AB
:10AD2000903023B12046FFF70EFDC4F89080B4F8B0
:10AD30005E309BB2002B93D1226852E8003F23F48F
:10AD4000807342E8003123680029F5D103F108023D
:10AD500052E8002F02EA090203F1080040E800214E
:10AD60000029F3D120225345C4F88C206167216764
:10AD70000AD05A68110207D553E8002F22F08062EA
:10AD800043E800210029F7D1E26E012A14D1002204
:10AD9000E26653E8002F22F0100243E80021002968
:10ADA000F7D1DA69B4F85C10D20644BF10221A62F7
:10ADB0002046FFF7F7FC53E72046F9F7AFFA4FE7D5
:10ADC0009A6942F008029A616CE700BFFEFFFFEF4C
:10ADD00000800040A1AA00082DE9F84F0368B0F8F0
:10ADE0006060D3F81CB01F689D68D0F88C20222AC0
:10ADF000044640F0B780B0F8683043B1DFF8709196
:10AE0000DFF870A14FF000081BF0200F20D1B4F83C
:10AE10005E309BB2D3B1B4F868209A4216D922684A
:10AE200002F1080353E8003F23F08053083242E860
:10AE3000003122680029F2D14F4B636752E8003F8E
:10AE400043F0200342E800310029F7D1BDE8F88F34
:10AE50002368A26D596A314022F8021BA265B4F83A
:10AE60005E20013A92B2A4F85E20D3F81CB01BF029
:10AE7000070F2ED01BF0010F09D0F90507D50122CD
:10AE80001A62D4F8902042F00102C4F890201BF01E
:10AE9000020F09D0EA0707D502221A62D4F89020DF
:10AEA00042F00402C4F890201BF0040F09D0E80718
:10AEB00007D504221A62D4F8903043F00203C4F894
:10AEC0009030D4F8903023B12046FFF73CFCC4F812
:10AED0009080B4F85E309BB2002B95D1226852E886
:10AEE000003F23F4807342E8003123680029F5D144
:10AEF00003F1080252E8002F02EA090203F10800F8
:10AF000040E800210029F3D120225345C4F88C20C9
:10AF1000616721670AD05A68110207D553E8002FEC
:10AF200022F0806243E800210029F7D1E26E012A75
:10AF300014D10022E26653E8002F22F0100243E809
:10AF400000210029F7D1DA69B4F85C10D20644BFB9
:10AF500010221A622046FFF725FC55E72046F9F734
:10AF6000DDF951E79A6942F008029A616EE700BF85
:10AF7000FEFFFFEF008000406DAB000838B50446CF
:10AF800003682169A2681D68C0690A4361690A43B0
:10AF90007749024329400A431A605A68E16822F45B
:10AFA00040520A435A60734AA16993421CBF226A05
:10AFB00011439A6822F06E4222F430620A439A608A
:10AFC000DA6A616A22F00F020A43DA626A4A93423D
:10AFD00019D14FF0B043694AD3F8883003F0030326
:10AFE00043F44033934200F0B480B3F1031F24D004
:10AFF000013A934240F0B580B0F5004F40F08F80A9
:10B00000FCF780FF6EE05E4A93421CD14FF0B043E4
:10B010005C49D3F8883003F00C0343F440228A42A1
:10B0200000F0978006D8002B7CD0574B9A42E3D093
:10B03000012026E0B2F10C1FFAD1B0F5004F53D039
:10B040004FF4004075E04B4A9342F1D14FF0B043CA
:10B05000D3F8883003F44063B3F5006F18D006D8F6
:10B060005BB1B3F5806FE3D1FCF74CFF07E0B3F5BC
:10B07000406FDDD14FF400400BE0FDF73BFB40B9E2
:10B0800000204FF00113A3660023C4E91D3338BD2F
:10B090003E4865683E4B626A05EB450133F8122075
:10B0A000B0FBF2F39942C3D8B3EB053FC0D80023FD
:10B0B0001946F7F7F9F9090241EA10616B08000235
:10B0C000C0182A464FF0000341F10001F7F7ECF9F0
:10B0D000304BA0F540729A42AAD82368D860CFE7D7
:10B0E000FDF708FB0028CBD06168294B626A33F872
:10B0F0001220B0FBF2F24B0803EB42034FF6EF7263
:10B10000B3FBF1F3A3F11001914291D823F00F02A8
:10B11000216892B2C3F342031343CB60B0E7FCF75C
:10B12000F1FE04E0B0F5004FDAD0FDF7E3FA0028B5
:10B13000A6D06368616A164A32F81120B0FBF2F0BB
:10B1400000EB5300B0FBF3F04FF6EF73A0F11002E9
:10B15000C1E7B0F5004F0D48EBD1C5E7FDF7DAFACE
:10B16000C0E7B0F5004FF9D0FDF7D4FADFE700BF34
:10B17000F369FFCF00800040003801400200030067
:10B180000044004008000C0004000C000024F400FF
:10B19000E8620308FFFC0F00836ADA0710B506D5E2
:10B1A0000168C46A4A6822F4003222434A609C075C
:10B1B00006D50168046B4A6822F4803222434A6053
:10B1C000590706D50168446B4A6822F4802222435D
:10B1D0004A601A0706D50168846B4A6822F4004267
:10B1E00022434A60DC0606D50168C46B8A6822F4F3
:10B1F000805222438A60990606D50168046C8A68E9
:10B2000022F4005222438A605A060FD50168446C2A
:10B210004A6822F480122243B4F5801F4A6005D1A7
:10B220004A68846C22F4C00222434A601B0606D599
:10B230000268C16C536823F400230B43536010BDB4
:10B240002DE9F843DDF8209005460F46164698464E
:10B250002A68D36937EA03030CBF01230023B342F2
:10B2600001D0002029E0B9F1FF3FF2D0F8F788FCC7
:10B27000A0EB080048452C6802D8B9F1000F1ED198
:10B2800054E8003F23F4D07344E80032002AF7D199
:10B2900004F1080353E8003F23F0010304F108011F
:10B2A00041E80032002AF3D12023C5F88830C5F8E0
:10B2B0008C30002385F884300320BDE8F8832368B0
:10B2C0005A07C5D5E3691B05C2D54FF40063236255
:10B2D00054E8003F23F4D07344E80032002AF7D149
:10B2E00004F1080353E8003F23F0010304F10801CF
:10B2F00041E80032002AF3D12023C5F88830C5F890
:10B300008C30C5F89030D4E773B504460026C0F8F9
:10B310009060F8F735FC23681B681A07054619D4B6
:10B3200023681B685B070AD56FF07E4300930022F9
:10B330002B464FF480012046FFF782FFB0B9002072
:10B340002023C4F8883084F88400C4F88C30E06688
:10B3500020670CE06FF07E430093324603464FF4C3
:10B3600000112046FFF76CFF0028D9D0032002B05F
:10B3700070BD10B5044650B3D0F888301BB980F8C2
:10B380008430F8F7CBFE22682423C4F88830136891
:10B3900023F0010313602046FFF7F0FD012816D0CB
:10B3A000A36A13B12046FFF7F7FE23685A6822F418
:10B3B00090425A609A6822F02A029A601A6842F013
:10B3C000010220461A60BDE81040FFF79DBF012032
:10B3D00010BD000030B581658168A0F85C200023B5
:10B3E000B1F5805FA0F85E20436735D10369002B7B
:10B3F00040F2FF1318BFFF23A0F860300023C0F80D
:10B4000090302223C0F88C30016801F1080353E822
:10B41000003F43F00103083141E800340368002C89
:10B42000F2D1456E84680169B5F1005F32D1B0F8A0
:10B43000685095422ED8B4F5805F244A03D1244C3D
:10B44000002908BF22464267B1B153E8002F42F4F9
:10B45000807243E80021F7E729B90369002B14BF84
:10B460007F23FF23C8E7B1F1805FC5D10369002BBB
:10B4700014BF3F237F23BFE703F1080252E8002FE8
:10B4800042F0805203F1080040E800210029F3D186
:10B49000002030BDB4F5805F0E4A03D10E4C002968
:10B4A00008BF2246426741B153E8002F42F4907230
:10B4B00043E800210029F7D1EAE753E8002F42F0E2
:10B4C000200243E800210029F7D1E1E731AC000870
:10B4D000D9AD0008A1AA00086DAB0008D0F88C30E7
:10B4E000202B30B415D1B9B1B2B100230468C366C2
:10B4F0000A4B9C420AD063681B0207D554E8003F00
:10B5000043F0806344E80035002DF7D130BCFFF7ED
:10B5100061BF022030BC70470120FBE70080004083
:10B52000436E30B52BB90123A0F86A30A0F868301B
:10B5300030BD0368094D9A689968094C490FC2F3F8
:10B5400042626B5C615CDB00B3FBF1F3A0F86A3034
:10B55000AB5CA25CDB00B3FBF2F3E7E70863030834
:10B56000006303087047704770471FB504AB03E9D9
:10B57000060090F88430012B04463AD0012380F86D
:10B5800084302423C0F8883003681A6822F001024E
:10B590001A609A6822F440120A439A6071B95A6894
:10B5A000BDF80C009DF80E1022F0100202435A6004
:10B5B0005A6822F07F4242EA01625A601A6842F0F9
:10B5C00001021A60F8F7DCFA6FF07E42034600923F
:10B5D0004FF4800100222046FFF732FE38B92023C5
:10B5E000C4F88830002384F8843004B010BD0320F0
:10B5F000F8E70220F9E790F88430012B0FD00123FF
:10B6000080F88430016851E8002F42F0020241E8DE
:10B610000023002BF6D180F88430184670470220B2
:10B62000704710B590F88430012B044617D02423BE
:10B63000C0F8883003681A68196821F001011960A0
:10B6400042F000524FF0005141661A60FFF768FF68
:10B650002023C0F88830002084F8840010BD022028
:10B66000FCE770B590F88430012B044617D00568CC
:10B670002423C0F888302E682B6823F001032B6048
:10B68000AB6823F060431943A960FFF749FF20230B
:10B690002E60C0F88830002084F8840070BD02203D
:10B6A000FCE770B590F88430012B044617D005688C
:10B6B0002423C0F888302E682B6823F001032B6008
:10B6C000AB6823F060631943A960FFF729FF2023CB
:10B6D0002E60C0F88830002084F8840070BD0220FD
:10B6E000FCE7000038B5084D052455F8043B2BB99C
:10B6F000013C14F0FF04F8D1204638BDDB689847C0
:10B700000028F5D0F9E700BFB0200020034BD87027
:10B71000034B1B681B6C03B118477047982000202F
:10B7200094200020034B1874034B1B685B6C03B11F
:10B73000184770479820002094200020F0B5314D24
:10B74000314B95F90420314E91B00C46012795F903
:10B7500005108DF8047002288DF809208DF80A1064
:10B7600010D18DF80800D8711C7203F075FB337886
:10B7700003B114B101A804F0A5F8254B059A1A608D
:10B7800011B0F0BD59714FF480711A71D9801C72DB
:10B7900033788DF8087053BB1F2306A88DF81C2042
:10B7A0008DF8183003F036FD20238DF8183006A8E8
:10B7B0002B798DF81C3003F02DFD22238DF81830E5
:10B7C00006A86B798DF81C3003F024FD21238DF839
:10B7D000183006A86B798DF81C3003F01BFD292367
:10B7E0008DF8183006A80B4B079303F013FD03F0F8
:10B7F00033FB012306A88DF818308DF81C3003F0B8
:10B8000009FDB4E7982000203C010020741F0020AF
:10B8100068200020000400017FB5092301A88DF8ED
:10B82000043004F04FF80038044B059A1A6018BF32
:10B830000120404207B05DF804FB00BF68200020F3
:10B8400070B504460B46144962784A700020A2780D
:10B850000A7208701A884A729A788A72DB780B74B6
:10B860006368CB600D4B1B68DA6A2AB1237803F05A
:10B87000FB030A2B00D09047094E002556F8043BE5
:10B880001BB15B6A0BB1204698470135EBB2052B23
:10B890006DB2F3D170BD00BF0C01002094200020D8
:10B8A000B020002070B5044611480123037063786E
:10B8B0004370A3788372E368C360E37803762369F7
:10B8C0004376237943720B4B1B689B6A03B19847FD
:10B8D000094E002556F8043B1BB19B690BB120466D
:10B8E00098470135EBB2052B6DB2F3D170BD00BFA7
:10B8F0002001002094200020B0200020014B186877
:10B90000704700BF6820002000B58BB00123684657
:10B910008DF8003003F058FB38B99DF8040000386A
:10B9200018BF01200BB05DF804FB0020FAE700000F
:10B9300008B502F049FC40B9FFF7E6FF012806D040
:10B94000054B197AD879FFF7F9FE012008BDBDE84B
:10B950000840FFF7C7BE00BF3C0100202DE9F041C1
:10B9600086B005460E46174602F02EFC002873D11D
:10B9700002F042FC044640B9FFF7C6FF01280AD096
:10B980003D4B197AD879FFF7D9FE6FF002042046B3
:10B9900006B0BDE8F081DFF8E48088F80860003E7A
:10B9A00018BF01268DF80460354E687833798DF81C
:10B9B0001230694603F0A6FA00283FD08DF8044003
:10B9C0000394ADF810406FF0060495E803002D4B8A
:10B9D00083E80300337988F80A30394601A804F077
:10B9E00075F8294B059A1A6011283FD801A353F81E
:10B9F00020F000BF5FBA000859BA00086DBA00080D
:10BA00006DBA00086DBA00086DBA00086DBA00087A
:10BA10008BB900086DBA00086DBA00086DBA00084D
:10BA200053BA00086DBA00086DBA000859BA000888
:10BA300059BA000859BA000873BA00082B788DF873
:10BA400008306B78ADF810306B6803934FF0FF341B
:10BA5000BBE76FF005049AE76FF0010497E70B4B23
:10BA600000221A70E31D18BF144690E74FF0FF3410
:10BA70008DE76FF004048AE73C01002020010020DC
:10BA8000982000203001002068200020672000203E
:10BA900037B502F0BBFB134D052455F8043B4BB101
:10BAA0001A693AB19B682BB1984718B155F8043C14
:10BAB0001B699847013C14F0FF04EED1FFF712FE1A
:10BAC00068B9094D2B7853B1084BADF80040D978CF
:10BAD000019422466846FFF741FF00B92C7003B07D
:10BAE00030BD00BFB020002067200020982000203B
:10BAF00030B58BB0044602F067FB0546002835D10F
:10BB0000FFF702FF012834D168468DF8005003F09A
:10BB10005BFA40BB9DF80430A34204D0012C22D034
:10BB2000022C12D014B100200BB030BD002BFAD083
:10BB300068468DF8044003F06DFBA0B90E4B1B68FE
:10BB40001B6B002BEFD09847EDE763B968468DF883
:10BB5000044003F05FFB30B9074B1B681B6B002BE5
:10BB6000E1D02046EFE74FF0FF30DDE76FF0010056
:10BB7000DAE76FF00200D7E79420002010B5044602
:10BB80008AB018B94FF0FF300AB010BD00236846E4
:10BB90008DF8003003F018FA0028F3D19DF8043036
:10BBA0002370F1E77FB500220B4620498DF807206E
:10BBB00001220A7042784A700446002A33D1027981
:10BBC0000A721A884A729A788A72DB780B7403694F
:10BBD000CB60C378164D8DF80830037B8DF80930A3
:10BBE000836803932B68DB6A0BB102A898472B6824
:10BBF0009B6B13B1227E02B198470E4E052556F875
:10BC0000043B1BB1DB690BB120469847013D15F0A1
:10BC1000FF05F4D10DF10700FFF7B0FF637913B111
:10BC2000054B01221A7004B070BD00BF0C0100204A
:10BC300094200020B02000206720002010B504468A
:10BC40008AB018B94FF0FF300AB010BD2023684603
:10BC50008DF8003003F0B8F90028F3D1024A9DF9BD
:10BC6000043023701371EFE79820002000B58BB0EB
:10BC70002323019068468DF8003003F0CBFA00389A
:10BC800018BF012040420BB05DF804FB70B5654C55
:10BC900001468EB01822204606F0BCFF624B0022FF
:10BCA0001A70FAF77FFE23784068012202FA03F146
:10BCB000014004D15D4B084608F098FFFEE75C495F
:10BCC0005C481A4602F00AFF18B14FF0FF300EB080
:10BCD00070BD272304A88DF8103003F09BFA564E50
:10BCE000564D002870D1012333702B68DB690BB1EE
:10BCF00000209847272304A88DF8103003F064F93A
:10BD0000059B93F84820227093F8182193F81A3174
:10BD10006270A370464BD3E9020106F06BFE054644
:10BD20000028D2D1464E062304A88DF8103003F027
:10BD30004BF9059B736104A803F06CFA022304A875
:10BD40008DF81030059603F03FF90836032304A858
:10BD50008DF81030059603F037F90F2606F010FF26
:10BD6000012304A88DF814308DF8106003F052FA06
:10BD700010230DEB03008DF810308DF8145003F0F4
:10BD800049FA04238DF8103004A8A3788DF81430F4
:10BD900003F040FA3A238DF8103004A86369059344
:10BDA00003F038FA02A920788DF8086004F0CCFF7F
:10BDB000003818BF0120E0711420FFF757FFE07929
:10BDC00004F046F8284682E728238DF810302B68C7
:10BDD0001B6943B104A803F0F7F82B6805981B69A9
:10BDE00040F2C4519847272304A88DF8103003F07F
:10BDF00011FA50B9012304A88DF8103003F0E4F8CB
:10BE00009DF81430002B7FF46EAF3378002B7FF455
:10BE10006CAF052204A88DF81020059303F0FAF901
:10BE200078E700BF982000206720002010630308F7
:10BE30006C20002084200020741F0020942000200B
:10BE4000D420002037B500230D4601930446D0B915
:10BE500000F07CFD0190019BD3B10F4A42F82430E1
:10BE60000E4A9A620E4A1268916B1963916C59637B
:10BE700092690C49D9625A6128465B680A49F222E4
:10BE80009847002006E001A900F076FD0028E2D0E6
:10BE90004FF0FF3003B030BDB02000203DB70008A8
:10BEA0009420002019B80008751F0020194B07B511
:10BEB0001860194B194A1A60194A5A60194A9A604F
:10BEC000194ADA60194B02681A6042685A6082683F
:10BED0009A60C268DA60164A1A6182695A61154B23
:10BEE000C26B5A60144A019119609A601946134A4C
:10BEF000DA600020FFF7A6FF48B901A800F02AFD8C
:10BF0000003818BF0120404203B05DF804FB4FF039
:10BF1000FF30F9E79420002084200020A5B8000815
:10BF2000A5BB0008E5BF000841B800086C20002050
:10BF3000F90C0108C42000200DB7000825B700083F
:10BF400049B118B1012804D000207047034B0B60A1
:10BF5000FAE7034BFBE74FF0FF30704700040001A6
:10BF60000100010208B503F08FFF002814BF6FF035
:10BF70000100002008BD08B502F096FF002814BF9C
:10BF80006FF00100002008BD20B1044BDB79037085
:10BF9000002070474FF0FF30704700BF982000200E
:10BFA00008B5034BD87103F053FF002008BD00BF54
:10BFB0009820002010B504468AB018B94FF0FF3021
:10BFC0000AB010BD212368468DF8003002F0FCFF56
:10BFD0000028F3D1024A9DF9043023705371EFE732
:10BFE000982000202DE9F0412F4D304F00232B7079
:10BFF00043786B703B689B6A8AB004460BB1284655
:10C000009847DFF8AC80002658F8043B1BB11B6A48
:10C010000BB1204698470136F3B2052B76B2F3D127
:10C020002378052B2FD00B2B35D0012B25D1214C7C
:10C03000062368468DF8003002F0C6FF0199E079CA
:10C0400006F01EFD10B91C4B019A5A611B48FFF700
:10C05000F5FD1B48FFF7AEFF6B788BB9A371194B49
:10C060005878FFF745FD3B685B6A0BB1114898476C
:10C070006B7813B9E07906F095FD0AB0BDE8F08160
:10C08000FF23A371EFE7104B01225A74227A9A74AE
:10C09000627ADA74F1E76378002BEED00AB0BDE87B
:10C0A000F041FFF7B9BB00BF200100209420002021
:10C0B000B02000203C010020D420002040010020BE
:10C0C00041010020982000200C01002030B58BB0E9
:10C0D000FFF751FF0446F0B904F016FE831C1DD093
:10C0E000F8B9134D2B685B69DBB1272368468DF8DF
:10C0F000003002F069FF2B6801985B694FF4B96169
:10C10000984704F013FE78B92CB9094B1B68DB691A
:10C110000BB10120984720460BB030BD6FF00704EB
:10C12000EFE74FF0FF34ECE74FF0FF34F3E700BFE9
:10C1300094200020014B1878704700BF0421002094
:10C14000014B5878704700BF04210020064B074878
:10C1500010B501225A7309F085F9054B5B6913B1DB
:10C16000BDE81040184710BD04210020EC2000203D
:10C170004801002013B50A4C79B1A27001230022B6
:10C18000616023700748084B00924FF0FF3109F0BF
:10C19000BDF80023637002B010BD2170F9E700BF45
:10C1A00004210020EC2000204DC100082DE9FF47AC
:10C1B000C378CA2B804600F0BE8004B0BDE8F0878B
:10C1C000D8F808305A5D6E1CF6B2032A0FD8DFE8A3
:10C1D00002F0022E6CAB7A6800231355611CA31C7D
:10C1E000DBB2C9B2012050540334D054E4B2354616
:10C1F00098F80C30AB42E3D8002CDED0CA238DF87F
:10C200000830504B8DF809405B6803930DF107002F
:10C21000FFF7BAFE0020FFF7C3FE0122002102A8AB
:10C22000FFF79CFB9DF80700FFF7BAFEC5E7002269
:10C230007A7398F818204AB96A1DD2B2397A9A5C92
:10C2400001F00F0102F00F02914202D0AE1DF6B2D2
:10C25000CDE7AA1CD2B29E5D9A5C06EB0226EA1CD0
:10C26000D2B20DF1080A9A5C06EB02462A1DD2B240
:10C2700050469B5C06EB036608F022FF029B3344AA
:10C2800002939AE8030008F0F3FE3B7AC3F303023B
:10C29000013262F303033B722B4B1B6B002BD5D097
:10C2A0000136022ED2D89847D0E7EE1C0235EDB207
:10C2B0001E215B5D002003F00F0380259D4006F0EA
:10C2C0008DFC7A680223135504EB030A631CDBB26E
:10C2D0000021D154054402A808F0F2FE029B7A68BE
:10C2E0004B4504F1030188BFA3EB09035FFA8AFA07
:10C2F000C9B2180A02F80A305054611D201DC9B293
:10C30000C0B24FEA134C1B0E02F800C053544FF456
:10C310007A7169430D4809F0DFF806340B48F6B22C
:10C32000E4B209F09FF862E79B5D023503F0070372
:10C330007B73EEB25BE70024024FDFF814902546D2
:10C3400056E700BF0421002048010020EC20002017
:10C35000803DD51210B5114C637A8AB0E3B1042345
:10C360008DF800306846A37A8DF8043002F052FF51
:10C3700018238DF800306846E37A8DF8043002F017
:10C3800049FF20238DF800306846237B8DF8043068
:10C3900002F040FF002363720AB010BD04210020A8
:10C3A000004870474801002030B58FB0FFF7C0FA51
:10C3B000002861D1324C657A4DBB042304A88DF866
:10C3C000103002F001FE9DF81430A37204A88DF81D
:10C3D000145002F01FFF182304A88DF8103002F04B
:10C3E000F3FD9DF81430E37204A801238DF8143096
:10C3F00002F010FF202304A88DF8103002F0E4FDB5
:10C400009DF8143023731F4BDB6A03B1984702A8D1
:10C4100008F056FE029A1C4B1C4913448B4288BFFD
:10C420001B4B616888BF9B181A0A4B708A701A0CE4
:10C430001B0E0B71237ACA7001256FF304134B7125
:10C440000D7023720DF1070040F2CA63ADF8103091
:10C4500005916572FFF798FD0020FFF7A1FD2A46C0
:10C46000002104A8FFF77AFA04469DF80700FFF7B9
:10C4700097FD20460FB030BD4FF0FF34F9E700BF05
:10C48000042100204801002080C22AED803DD51201
:10C49000008555DA10B5054C637B2BB1FFF784FF9F
:10C4A00010B9637B013B637310BD00BF0421002002
:10C4B000014B1878704700BF30210020014B58789D
:10C4C000704700BF3021002070470000044B9A7A6B
:10C4D0000AB101225A70034B5B6903B118477047D8
:10C4E000302100208001002073B5224C6378002B9E
:10C4F00033D008F025FF66680546FFF7FFF90644CC
:10C50000AE4214D2A37A93B1E0228DF800208DF8C8
:10C510000130217AE368019301226846FFF71EFA91
:10C5200008B1073010D100236370A372656094F8DE
:10C530003430EBB1002384F834300F4B5B6BBBB16C
:10C5400002B0BDE87040184740F2DC510B4808F0DB
:10C55000C3FF0A4808F086FFE8E794F83520002A70
:10C56000E5D094F8360084F83530FFF7C1FADEE7FD
:10C5700002B070BD30210020800100201421002075
:10C5800037B5104D104CC8B1C1B162720123002201
:10C590002860E16023700D480D4B00924FF0FF3191
:10C5A00008F0B4FE00250B4825822022294606F01B
:10C5B00045FB6570A574A58603B030BD00232B60D4
:10C5C0002370EFE72C2100203021002014210020CF
:10C5D000CDC40008442100202DE9F0478E4C23787B
:10C5E0008CB0002B56D0C2780AB9837B13B1238A52
:10C5F00001332382437B002B4CD0E02A4AD1002315
:10C60000A372876897F80080B8F1220F27D8B8F195
:10C61000220F30D8DFE818F04100FB0052005A002A
:10C6200061006E0075008E009D00B400C7002F00F1
:10C630002F002F002F002F002F002F002F002F0082
:10C640002F002F002F002F002F002F002F002F0072
:10C650002F002F002F002F00C900D000D400B8F108
:10C660007E0F00F0CC80B8F17F0F00F0DF80B8F1D2
:10C670007D0F00F0AB80A57A002D00F05B81674C48
:10C68000637A3BB94FF47A71204608F025FF2046C3
:10C6900008F0E8FE0CB0BDE8F087E3680122002155
:10C6A000A2721970A37AE1689818A0720620C85483
:10C6B000A37AE1689818A072CA54DCE7584B9B6AC9
:10C6C000002BD8D0012102209847D4E77B7884F84A
:10C6D0003630012384F83530CDE704238DF804305B
:10C6E0007B78003B18BF012301A88DF8083002F0C9
:10C6F00091FDC0E77878003818BF012003F0A8FB4F
:10C70000B9E7484E0FCE01AD0FC50FCE0FC596E865
:10C71000070085E807007B780A2BACD8424A1268EC
:10C720005268002AA7D00CA901EB830353F82C0C04
:10C730009047A0E77878431E012B9CD83A4B0138EC
:10C740001B6818BF012020729B68002B93D098476C
:10C7500091E7E26801230821A3721170627A057BD8
:10C76000A17AAA4228BF2A46934284D285685A1CDD
:10C77000EB5CE56801334E1CA6726B54D3B2EDE757
:10C78000E3680122A27209221A70A37AE268218A60
:10C79000581CA072D154A27A238AE1681B0A501C4B
:10C7A000A0728B5467E7238265E705238DF8043078
:10C7B00001A803F087F85EE7194BDB6A98475AE750
:10C7C000194B78781B686075DB68BEE7037B072B25
:10C7D0007FF451AF06238DF80430B7F80130ADF87F
:10C7E00008307B793A791B0443EA0223FA78134331
:10C7F000642253430393BB798DF81030D8E73B2272
:10C8000001A88DF804208DF8083002F003FD012303
:10C8100084F834302FE700BF30210020142100209D
:10C82000800100201C2003082C2100202A2301A8BD
:10C830008DF8043002F0C8FB94F80A90E6689DF881
:10C8400008009DF809509DF80A709DF80BC09DF8EE
:10C850000D309DF80E209DF80F109DF80CE009F1A9
:10C86000010A84F80AA006F80980354E94F80A9067
:10C870003668D4F80C8009F1010A84F80AA096F809
:10C8800003A008F809A094F80A90D4F80C8009F1E4
:10C89000010A84F80AA096F802A008F809A094F802
:10C8A0000A90D4F80C8009F1010A84F80AA096F8DD
:10C8B00001A008F809A094F80A9009F1010A84F887
:10C8C0000AA096F80080E66806F8098094F80A80C5
:10C8D000E66808F1010984F80A9006F808C094F89F
:10C8E0000AC0E6680CF1010884F80A8006F80C70AA
:10C8F000A77AE66807F1010C84F80AC0F555A57A15
:10C90000E6686F1CA7727055A07AE568461CA6728F
:10C910002954A17AE0684D1CA5724254A27AE168BC
:10C92000501CA0728B54A37AE268591CA17202F8C1
:10C9300003E0A0E6034808F047FD6570AAE600BFE3
:10C940002C2100201421002070470000004870476F
:10C9500080010020002108B50120FFF773FA01468D
:10C9600038B90220FFF76EFA003818BF01204042A4
:10C9700008BD4FF0FF30FBE710B50C4661B1012850
:10C9800003D0022805D0002010BDFFF709FD20606C
:10C99000F9E700F01FFCFAE74FF0FF30F4E7000082
:10C9A000014B1878704700BFF0010020014B587808
:10C9B000704700BFF0010020F7B500208DF8070098
:10C9C000EFF3108272B62A4FBB78FD7882F310889D
:10C9D000012B08D0022B04D1264B93F82030012BD9
:10C9E0003CD103B0F0BD234E0DF10700FFF7C6F8B0
:10C9F000382303FB056393F82C00012806D19DF82A
:10CA00000730022B08D10023BB70EAE7022803D1CC
:10CA10009DF80730012BF5E7FFF76AF805EB4504B1
:10CA2000E400B0B9144BB8701C44382303FB05660E
:10CA30004FF47A7196F82830994096F82C30012BF3
:10CA400000D1C901204608F047FD204608F00AFD44
:10CA5000C7E70A4B1C444FF47A71F3E7FFF748F835
:10CA60000028D0D0044C05EB450504EBC504F2E7E3
:10CA7000F001002098210020682100208021002062
:10CA800037B50F4CD1B100250123A160227123706D
:10CA90002A460C4B0C4800954FF0FF3108F036FC4D
:10CAA0000A4B0B4800952A464FF0FF3108F02EFC48
:10CAB000084A00236370137003B030BD2170F7E79C
:10CAC000F00100200DCB000880210020D9CA000809
:10CAD000682100209821002010B5084808F074FC57
:10CAE000074B002283F82020064B02225A80064B77
:10CAF0005B6913B1BDE81040184710BD68210020E4
:10CB000098210020F0010020B801002010B508484D
:10CB100008F05AFC074A012382F82030064A538065
:10CB2000064B5B6913B1BDE81040184710BD00BF4C
:10CB30008021002098210020F0010020B801002071
:10CB40002DE9F04FC378C82B8FB0824600F02983BF
:10CB50000FB0BDE8F08FDAF80820D05C591CC9B2DC
:10CB6000052816D8DFE810F00600AA00F000AE0194
:10CB7000E1018B02BA680023601C1355C0B2A31CEC
:10CB8000DBB24FF0020C02F800C001200334D05495
:10CB9000E4B20B469AF80C209A42DCD8002CD7D08D
:10CBA000C8238DF81430B74B8DF815409B68069359
:10CBB0000DF11300FFF7E8F90020FFF7F1F901226A
:10CBC000002105A8FEF7CAFE9DF81300FFF7E8F95B
:10CBD000002DBDD1AC4CAD4F637803F003032A4662
:10CBE000294600930220AA4B08F000F82646636805
:10CBF00000932A462946A74B022007F0F7FF16F8B4
:10CC0000083F00932A462946A34B022007F0EEFF77
:10CC1000012516F8013F009300223B4611460220F1
:10CC2000013507F0E3FF102DF3D1002211469B4B95
:10CC3000022007F0DBFFA369009300221146984B06
:10CC4000022007F0D3FFE369009300221146954BC1
:10CC5000022007F0CBFF636A009300221146924B3B
:10CC6000022007F0C3FF94F82820012393400022FC
:10CC70001146009302208D4B07F0B8FF94F82C303A
:10CC80000022012B236B00931146894B4FF00200C9
:10CC900040F08D8207F0AAFF94F93430009300220F
:10CCA000844B1146022007F0A1FFE38E0093824BD4
:10CCB00000221146022007F099FF49E7BD6812F8EB
:10CCC00001C001222A55023300220234DBB2E4B251
:10CCD000114696460CF0010C96F80080BEF1000F4C
:10CCE00007D0120102F0700211436970054619461F
:10CCF0004FE7B8F1000FF4D0BCF1000F21D005F8D8
:10CD000004E004F1010E5FFA8EFE716805F80E1062
:10CD100004F1020E71685FFA8EFE090A05F80E1022
:10CD200004F1030E5FFA8EFEB6F8068005F80E8059
:10CD3000211DC9B296F807E005F801E00534E4B218
:10CD4000614601328646C7E7555C382105F0030588
:10CD500001FB056103F1020B5FFA8BFB4D70002DA7
:10CD600040F08E80D81C12F80B107160C0B203F135
:10CD7000050C105C01EB0021181DC0B27160105C45
:10CD80005FFA8CFC01EB0041716012F80CC0981D39
:10CD900001EB0C6903F11601DFF820C1C6F804901D
:10CDA000C0B2C9B286460130C0B212F80EE00CF82B
:10CDB00001EF8842F6D1115CB16103F11700C0B2F6
:10CDC00003F11E0B105C01EB002103F11800C0B24F
:10CDD000B161105C01EB004103F11900C0B2B16117
:10CDE000105C01EB006803F11A01C9B2C6F81880A3
:10CDF00003F11B00515CF161C0B25FFA8BFB105C68
:10CE000001EB002103F11C00C0B2F161105C1D3385
:10CE100001EB0041DBB2F161D35C0DF1170001EBD6
:10CE2000036321220021F361039321F0FBFD40F213
:10CE30000112ADF814207278039B0A93C2F3010229
:10CE40008DF8162005A81E4ACDF818900792CDF847
:10CE5000248002F065FC012390B93370B968022385
:10CE60000B55621C1C44382303FB0563D2B25B786C
:10CE7000C3F3010343EA80008854E4B2594688E6CC
:10CE80000120EBE7F001002098210020AF630308A8
:10CE900074630308876303089C630308116B03082A
:10CEA000B5630308C8630308DB630308EE63030884
:10CEB00003640308166403082C6403089F21002000
:10CEC000A0210020555C382005F00305023300FB4B
:10CED00005FB5FFA83F906EB0B034FF000081846D9
:10CEE00010224146083083F80180C3F80480039380
:10CEF00005F0A4FE039BC3E90688BB68032204F186
:10CF000001081A5528465FFA88F802F051FC40B132
:10CF100045F00403BA68023402F80830E4B2494626
:10CF200037E606F80B002B46F4E74FF0000B8DF8C0
:10CF300013B0555C03F1020815F003055FFA88F899
:10CF400040F09680DFF874B24FF002098BF82C9015
:10CF5000D81C12F80810CBF82410C0B203F10B084B
:10CF6000105C01EB0021181DC0B2CBF82410105C3E
:10CF700001EB0041581DC0B2CBF82410105C01EB4E
:10CF800000618F480844991DC9B2CBF82400515C58
:10CF900001F00F018BF82810D91DC9B203F1080068
:10CFA000515CCBF83010C0B25FFA88F8105C41EAEF
:10CFB000002103F10900C0B2CBF83010105C0A3335
:10CFC00041EA004164204143DBB2CBF83010D35C2E
:10CFD0008BF834300DF113020BF12C01284602F0CE
:10CFE00013FC002849D105A808F06AF8DBF82420D2
:10CFF000059BA2EB030BBBF1000F31DD4FF47A71FF
:10D0000001FB0BF16F48039108F066FA6D4808F0D8
:10D0100029FA039900916C4B29462A46484607F0A5
:10D02000E5FD0121BA6804231355601CC0B29DF8C8
:10D0300013C002F800C0A31CDBB271B102F803B048
:10D04000E31CDBB24FEA2B21D154631D0434E4B25C
:10D050004FEA2B4B02F804B0DBB21C46414698E580
:10D060009DF8133043F010038DF813302946D9E7AB
:10D0700010238DF813305946D4E7AB46F6E74FF04E
:10D08000000B8DF813B0555C03F1020815F0030591
:10D090005FFA88F87ED1DFF824B14FF001098BF8F0
:10D0A0002C90D81C12F80810CBF82410C0B203F151
:10D0B0000B08105C01EB0021181DC0B2CBF8241046
:10D0C000105C01EB0041581DC0B2CBF82410105C7D
:10D0D00001EB00613A480844991DC9B2CBF824001D
:10D0E000505CC0F30210ABF83600515C01F00F0148
:10D0F0008BF82810D91DC9B203F10800515CCBF898
:10D100003010C0B25FFA88F8105C41EA002103F1E8
:10D110000900C0B2CBF83010105C0A3341EA00417C
:10D1200064204143DBB2CBF83010D35C8BF8343051
:10D130000DF113020BF12C01284602F065FB70BBC8
:10D1400005A807F0BDFFDBF82420059BA2EB030B2D
:10D15000BBF1000F16DD4FF47A7101FB0BF119489A
:10D16000039108F0B9F9174808F07CF90399009188
:10D17000154B29462A46022007F038FD4946BA6871
:10D18000052351E79DF8133043F010038DF8133059
:10D190002946F4E710238DF813305946EFE7AB46E4
:10D1A000F6E70024094F054EFF252346F2E407F079
:10D1B0001DFD94F934300093054B79E5982100204A
:10D1C000803DD5128021002059630308F001002022
:10D1D0001664030800487047B8010020044B054A54
:10D1E00093F81831022B18BF062382F89034704749
:10D1F0003C280020002E0020034BD3F8483313B105
:10D200005B6903B118477047002E0020034A13786A
:10D2100043F004031370FFF7EFBF00BFE4210020C9
:10D220001FB50A4B8DF8090093F87C208DF80A2071
:10D2300093F88C2093F848000D3202A98DF808204D
:10D2400003F082FDC0B205B05DF804FB3C2800206D
:10D2500008B5074808F0B8F8064B93F81A2412B13D
:10D26000012283F81924BDE80840FFF7C5BF00BFBD
:10D2700000320020002E002010B50C4CD4F84033B2
:10D2800043F08003C4F8403394F81A3413B10020FB
:10D29000FFF7DEFF94F8913423F0120343F01203FA
:10D2A00084F89134BDE81040FFF798BF002E0020AD
:10D2B0002DE9F041DFF8AC8098F81831022B0646D2
:10D2C0000D4602D0284BDB6A984702F078FE0446F0
:10D2D00028B1022002F069FE002002F06BFE98F8EF
:10D2E0001831012B17D102F06CFE074630B1002037
:10D2F00002F05CFE002002F05EFE3C4602F063FE9F
:10D3000048B1002002F053FE002002F055FEBDE8B7
:10D31000F041FFF763BF002CF9D1144C94F890242E
:10D3200094F81A34BAB90BB184F84164304602F06B
:10D33000EBFFD8F82C0008F00DF8D4F8B43398427D
:10D34000E5D30B4808F040F894F8913443F010030B
:10D3500084F89134DBE70BB184F84154284602F09D
:10D36000D3FFF1E73C2800206C6B0308002E00205F
:10D3700098310020074A10B5137843F00203137068
:10D38000FFF73AFFBDE81040034B012200210220C5
:10D3900007F02CBCE42100203F640308074A10B5C5
:10D3A000137843F008031370FFF726FFBDE8104021
:10D3B000034B01220021022007F018BCE4210020C9
:10D3C0004F6403082DE9F0410F4616461D4680467E
:10D3D00007F0B6FF0B4A0C4C1378278123F011039A
:10D3E00043F01103C4E90008137066812573FFF749
:10D3F00003FFBDE8F041054B01220021022007F0A8
:10D40000F5BB00BFE4210020D02100205F640308A9
:10D4100013B507F095FF0D4B6C461860204607F0DA
:10D420004FFE94E803000A4A0A4B83E8030013788E
:10D4300043F020031370FFF7DFFE074B01220021AA
:10D44000022002B0BDE8104007F0D0BBE021002070
:10D45000E4210020383100206C6403082DE9F041FC
:10D4600092B0064602F0ABFD002840F05881AD4D69
:10D4700095F81831012B09D02B6BAB4C93B194F874
:10D480000431BBB1042B6FD0032003E002F099FDFF
:10D4900018B10F2012B0BDE8F08102F094FD002811
:10D4A000EAD0F6E7B5F82031D4F81C24013B534309
:10D4B0002B63E4E79D4803F07EFB002840F01281D7
:10D4C00094F80C3123802B6B0C930DF1180895F810
:10D4D00039308DF83830404695F81C318DF83A30A7
:10D4E00007F014FED5F82831009302AF98E8060043
:10D4F000D5F82431384607F09FFD97E803000FABBD
:10D5000083E80300EB6A0D9300238DF844302388F1
:10D51000ADF8463095F8303101228DF839201BB92D
:10D520008DF844208DF83930814B0093814B95F86C
:10D530004800A3F179020CA903F07BFCC0B10B28D1
:10D54000A8D1D4F8941499B1002EA3D0D4F84033C4
:10D55000794843F02003C4F8403307F0BDFF764814
:10D5600007F080FF002095E7704803F058FBA4E720
:10D5700095F8487095F9693095F9392095F87D103E
:10D580006E4E384603F062FC009641B2EB6C95F8A3
:10D5900050203846183603F0FDFB0096EB6C95F8EA
:10D5A000502095F9701095F8480003F0F3FBD4F87B
:10D5B000C413AB6DD4F8DC230B44C4F8B033EB6D6B
:10D5C0001344C4F8B43394F80431042B07D02B6E01
:10D5D0000B44C4F8B0336B6E1344C4F8B433002367
:10D5E000089395F83031002B40D100238DF813308B
:10D5F00095F839308DF8213095F838308DF8223093
:10D60000D5F880300993D5F884300A932388ADF893
:10D610002C3095F8303194F81B648DF82E3095F845
:10D620004800474B8DF820600DF1130208A903F064
:10D63000C5FB012384F8413495F8393084F842342D
:10D640009DF8133084F84334D4F81C34C4F8506483
:10D65000C4F84834C4F8583402F0B7FCC8B1D4F860
:10D660001C0402F0C4FCA0B1102013E708A802F0CB
:10D670007BFD60B995F9390094F837629DF8207008
:10D68000FFF7CEFD3E44B042AFD2082002E71320A0
:10D6900000E795F81831012B01D102F0AAFC02F045
:10D6A00097FC0023059394F8043195F9395094F8C8
:10D6B0001B649BB1042B7FF4E7AE05A802F088FF42
:10D6C00058BB94F8183413B1059B013B0593174BD5
:10D6D00005983246E9B202F0E1FF02E0134802F099
:10D6E000B1FF08B11120D5E6D4F8403394F80C11FD
:10D6F000218043F00203C4F8403394F818341148F1
:10D700000133DBB284F8183484F845340E4B00251D
:10D710009B6AC4F89854984724E71220BAE60E2072
:10D72000B8E600BF3C280020002E0020082F002073
:10D730006C2800209432002068310020B83100208D
:10D740001C320020022E00206C6B030873B5134DB1
:10D75000134E0096EB6C95F8502095F9781095F8DB
:10D76000480003F017FB95F83031337595F8480001
:10D7700040F2012306F13C023146738203F016FBAE
:10D7800050B196F83C3086F88230064B00205B6B37
:10D790009847F37C86F8A83002B070BD3C28002082
:10D7A000E83100206C6B0308F8B5324C94F818315E
:10D7B000012B05460ED0022B4ED0002B57D138B985
:10D7C000D4E91B0104F1740383E803000020F8BDD1
:10D7D000012806D102F0FEFB0028F8D184F8185188
:10D7E000F5E7022843D1244E84F8180106F5747C2D
:10D7F000BCE80F0006F57A770FC79CE8030094F8A1
:10D80000E92094F8003187E8030086F8FB53D2B191
:10D81000022B18D1D4F804316367C6F8EC3394F8BE
:10D820007D3094F8082186F8F83394F88C3084F829
:10D83000782086F8F93396F81B2486F8E82340F21E
:10D840000133A6F8FA33002386F81A340B4BDB6A4F
:10D850009847FFF77BFFB9E748B9074B84F81801F1
:10D86000062283F89024054BDB6A9847AEE7032035
:10D87000ADE700BF3C280020002E00206C6B0308A1
:10D88000F0B5504C504EB4F8DC202287D4E92D017D
:10D8900094F8B12084F8692004F16C0282E8030056
:10D8A000D4E92F0104F1740282E80300B4F8C42023
:10D8B000A4F87C2091B0D4F8CC20D4F8C810C4F8D7
:10D8C00084200025D4F8D020C4F888200123A4F8AF
:10D8D0002031C4F8801084F83051A56284F81B51BF
:10D8E00084F83A5084F81D5184F81E51C4F834511C
:10D8F000C6F89854A6F8185486F81A54A4F8385163
:10D900008DF8183004F50973039304F50A7394F83D
:10D910004800049303A92D4B84F84551C4E94F55A1
:10D92000A4F84651059303F01DFAE36EC6F8D4330C
:10D9300094F87D3086F8E03394F88C3086F8E13343
:10D940004FF48073A6F8E23386F8D05394F8303160
:10D9500086F8E43306F574770FCF06F57A740FC4B2
:10D9600097E8030040F2012384E80300A6F8FA33A5
:10D97000D6F8483386F81B54CDE901551BB15A68D7
:10D980005B6901920293124B0793A3F1480208923C
:10D99000A3F1140209920F4A0B9229330A93A2F1C0
:10D9A0009C030C93A2F198030D93131D0E9301A9F0
:10D9B00002F14C0307A802F599620F9302F0F4FA02
:10D9C00011B0F0BD3C280020002E0020E8210020EE
:10D9D0006832002020290020F8B50D4F0D4E0C466E
:10D9E00007F0F2FC3B6B98470B4A96F8480021463B
:10D9F00003F0DCF950B1094D706D95F8243485F8C9
:10DA00006A347B6B9847E37C85F89034F8BD00BF9F
:10DA10006C6B03083C28002024320020002E0020DC
:10DA20000F4890F81B3480F8B8330E4B93F86920F8
:10DA300080F8BB2393F87D2080F8C82393F88C20CE
:10DA400080F8C92393F8303180F8CC330022A0F855
:10DA5000CA2300F56E7100F56070FFF7BDBF00BF0F
:10DA6000002E00203C280020114890F89034EBB1A3
:10DA700090F81B3480F8D0330E4BDA6EC0F8D42304
:10DA800093F87D2080F8E02393F88C2080F8E12340
:10DA900093F8303180F8E4334FF48072A0F8E22339
:10DAA00000F5747100F56670FFF796BF704700BF10
:10DAB000002E00203C28002070B5344C2421204644
:10DAC00005F0BEF8636A984218BF60624FF01C010F
:10DAD0002F4814BF0125002505F0B2F8636C984269
:10DAE00018BF60644FF480712A4818BF45F00205E2
:10DAF00005F0A6F8D4F84831984218BFC4F8480198
:10DB00004FF0D401244818BF45F0040505F098F8FB
:10DB1000D4F82032984218BFC4F820024FF0000118
:10DB20001E4818BF45F0080505F08AF8D4F82432DD
:10DB3000984218BFC4F824024FF46071184818BF07
:10DB400045F0100505F07CF8D4F8A835984218BFC8
:10DB5000C4F8A8054FF01401124818BF45F020057D
:10DB600005F06EF8D4F8C03598420F4B18BFC4F8D2
:10DB7000C005D3F8483318BF45F040052BB11B69E9
:10DB80001BB12846BDE87040184770BD3C280020F6
:10DB9000642800208428002088290020602A002092
:10DBA000642A0020E82D0020002E00202DE9F04FEF
:10DBB0008FB04FF00009012B06460F4690468DF8B6
:10DBC0000D90ADF8109002D84C46BC4202D30FB075
:10DBD000BDE8F08F305D02F007FB2044B842F6DC70
:10DBE000335D651C023BEDB2112BF0D801A252F857
:10DBF00023F000BF3DDC000867DC000865DD00089D
:10DC00008DDD00080BDE000831DE000897DE00081D
:10DC1000BFDE000845DF0008CFDB0008CFDB0008CF
:10DC200099DF0008CFDB0008CFDB000841E00008E7
:10DC300069E00008A1E00008D5E00008052002F036
:10DC40007BFB70B10521002002F03CFB725DBA4BFA
:10DC5000E51C0234E4B283F85C24325D83F85D2471
:10DC6000EDB22C46B1E700238DF80E308DF80F3061
:10DC70008DF814308DF81830B9F1000F6DD1AF4C1C
:10DC80004FF0050994F87C208DF831206B1E94F834
:10DC900039208DF83320334494F838200B938DF8D5
:10DCA000342094F81A3194F868208DF83520D4F88F
:10DCB0002C218DF832300A9273B37B1C5B1BDBB2D4
:10DCC0008DF8303006AB019305AB009394F8480013
:10DCD0000DF10F030DF10E020AA903F07BF88DF888
:10DCE0000D0000F00700072813D194F939209DF9A1
:10DCF0000E3084F839309A429DF80F3084F838306D
:10DD0000B8BF01229DF81430B8BF84F81D2184F8F3
:10DD100068304FF0000A09E00523D1E701220DF138
:10DD20000D01032002F078F90AF1010A5FFA8AF284
:10DD30009DF81830B3FBF9F19142EFD82B44DDB2D6
:10DD40006B1EDBB29F420BD9F25C032A9AD0AF4222
:10DD500088BF1D464FF0010983E70534E5B2F9E7B6
:10DD60001D46F7E7735D754903F00F03012281F843
:10DD70001B31023402FA03F3A1F82031E4B200228D
:10DD800004A9042002F048F925466AE707238DF824
:10DD90000D30735DC3F3021203F00F038DF82830CA
:10DDA000E31CDBB28DF82920F25C231DDBB2651D7C
:10DDB000F35C0234E4B21B0443EA0223325D5F4C9D
:10DDC00013436422534394F848000B930AA903F0C9
:10DDD00010F800F00703072BEDB28DF80D000CD101
:10DDE0009DF8283084F8703084F878300B9BE36617
:10DDF00063679DF8293084F869308DF8100001229E
:10DE000004A9052002F008F92BE74B4BD3F848335F
:10DE100063B11B6853B1984708F03F038DF81000B9
:10DE20008DF81130022204A90620EBE7FF20F3E76A
:10DE300003238DF80D30735D8DF81C300AAB06930B
:10DE4000E31CDBB2A51DF25C231DDBB206A9F35C6B
:10DE50001B0443EA0223A21CD2B20534B25C134372
:10DE600064225343E4B20A9300230B93335D8DF88D
:10DE70003030324B93F8480002F0C1FFC3B20028A3
:10DE8000EDB28DF80D30FFF6ECAE8DF810300122BA
:10DE900004A90720B6E7735D03F00F03012B4FF4CD
:10DEA0007A7238BF01235343244A0234936503F541
:10DEB0007A73D365E4B2002204A9082062E7735D97
:10DEC0001E4DC3F340128DF8152095F84800C3F39A
:10DED000001205A903F00F038DF814208DF81630F9
:10DEE00002F093FF02340130E4B23FF44DAFBDF8CD
:10DEF0001430134AA5F87C309DF816309DF814A014
:10DF0000D05CF4F757F80223C5F880000AA995F809
:10DF100048008DF828308DF82AA002F015FF95F9F9
:10DF20003930069040B29842B8BF184685F839009B
:10DF3000002204A9092025E7002E00203C2800200B
:10DF40007964030803238DF80D30735D8DF8283054
:10DF5000E31CDBB2651DF25C231DDBB20234F35C13
:10DF6000E4B21B0443EA0223325D134364225343A9
:10DF70000B93644B0AA993F8480002F04CFFC3B21C
:10DF80000028EDB28DF80D30FFF66BAE8DF8103035
:10DF9000012204A90A2035E7092002F0CDF9DFF8B3
:10DFA00068B1002849D00921002002F08BF9002334
:10DFB000ADF81E30A31CDBB2F25CE31CDBB216F83A
:10DFC00003A0735D4FEA0A4A4AEA022A4AEA030AB0
:10DFD000231DDBB2A51D0534F35CE4B24AEA036AF3
:10DFE000335D4FF47A7253430AAC1B122046ADF8EE
:10DFF0001C3007F065F8454B53440693DBF83C337F
:10E0000000930DF1180A9AE80600DBF8383308A8E7
:10E0100007F012F8099B009394E80600089B50460D
:10E0200006F0EFFF9AE8030007F022F801F0DCFFAA
:10E030000123EDB28BF8383413E68BF8380410E680
:10E040000C2002F079F900283FF40BAE0C210020DF
:10E0500002F038F92C4B93F89034043B012B7FF6F7
:10E0600000AE01F0BDFFFCE5A31CDBB2725DF15C0C
:10E07000E31CDBB2651DF35C0434E4B21B04305DC9
:10E0800043EA012313436421594300F00F0001F0D8
:10E09000A8FFEDB28DF81000012204A91120B1E60D
:10E0A0000D2002F049F900283FF4DBAD0D210020DE
:10E0B00002F008F9A31CDBB2154AF05C735D12682C
:10E0C000251D0334E4B243EA0020315DEDB201F0D6
:10E0D0008AFFC6E5725DA31C251D0334DBB2E4B2E2
:10E0E000F15C335D1B0443EA01231343642058436E
:10E0F00001F07BFFEDB28DF81000012204A913207E
:10E1000080E600BF3C280020002E0020803DD51274
:10E11000D02100200E4B93F89124920703D593F859
:10E120008F24012A08D90B4991F81A2122B18A6A51
:10E13000501C18BF01328A620022A3F8182483F809
:10E140001A24D3F8402322F00202C3F84023704778
:10E15000002E00203C28002070B5184C1848194D9E
:10E1600007F032F9D4F84033D4F89804D5F8906029
:10E1700023F02003C4F8403338B107F0EBF88642AF
:10E1800003D2002385F83A3070BD0120FFF766F90D
:10E190000028F9D00B28F7D095F8393084F84234AC
:10E1A000092094F8183484F8453484F8410402F0C6
:10E1B000ABF8BDE87040FFF7ADBF00BF002E0020F8
:10E1C000683100203C280020094BD3F84023012A65
:10E1D0000AD008490978C90708D43AB993F89204D3
:10E1E000013818BF01207047002070470120704798
:10E1F000002E0020E4210020034BD3F84003431EEF
:10E2000058425841704700BF002E00202DE9F04FC2
:10E21000A9B0EFF3108272B6DFF8F0B20021DBF89C
:10E220000030CBF8001082F31088B94C002B00F0BE
:10E23000E180DAB29B06039264D5B64D95F81831A9
:10E24000022B02D0B44BDB6A9847EFF3108872B60A
:10E25000B24F07F075F83E68D4F8B013361A31445F
:10E26000AF4807F039F9AE4807F0FCF8D4F8B4131A
:10E27000AC48314407F030F9AA4807F0F3F888F3C6
:10E28000108894F81A34002B00F06B81152312A922
:10E2900095F848008DF8483002F056FDD4F8B413D4
:10E2A0000F900144A04807F017F99F4807F0DAF8EB
:10E2B0003B6894F81B24EB620DAF38468DF8702054
:10E2C0001D9306F023FFD5F82831009306AE97E89A
:10E2D0000600D5F82431304606F0AEFE96E803007D
:10E2E0001FAB83E80300D4F81C341E9395F830313B
:10E2F00095F84800003B18BF01231CA98DF8713028
:10E3000002F02BFD039BDF0648D5824DDFF81CA2EF
:10E31000D5F8E42004929BF80020BAF90A809AF913
:10E320000C90A4F88C84002363F300020A9384F811
:10E330004434A4F8223484F82534C4F82834A4F8EA
:10E340002C3484F82E34C4F8303484F82034C4F8E3
:10E35000343484F83834C4F83C346F4B8BF80020E4
:10E3600094F89024DB6A84F88E9484F88F24DAF889
:10E370000470BAF80860984794F88F3413B9694864
:10E3800007F022F83146384601F017FE8346002890
:10E3900000F0EA80A4F87E8484F88094039B190737
:10E3A0001AD55C4B93F81831022B02D05A4BDB6A1A
:10E3B00098470220FEF712FF84F8410401F0A4FF01
:10E3C00094F81A3413B1012384F8193494F8913471
:10E3D00043F0100384F89134039B5A0703D50621B8
:10E3E0000520FEF765FF039B9B0703D5042103204F
:10E3F000FEF75EFF01F000FE94F89124D7065FD58A
:10E40000002384F89234D4F840331E0644BF23F02E
:10E410008203C4F8403312F0050F00F0FB820B209A
:10E4200001F08AFF002800F0F58294F89134DD07AE
:10E4300000F1F082580740F10783D4F8403323F00D
:10E440000203C4F84033D4F8402382BB94F89154BB
:10E4500015F001011EBF2B4662F3000384F89134CE
:10E4600094F891345E0744BF6FF3820384F89134CB
:10E47000012384F8923421B1D4F844332C481B682A
:10E4800098476D070BD52B4801F062FF01F090FF14
:10E4900028B194F8913443F0040384F8913401F0E6
:10E4A00098FD94F891346FF3041384F891340123A8
:10E4B00084F8923494F8913443F0200384F8913432
:10E4C00094F8913418070AD56FF3C3031A4984F8F6
:10E4D0009134D4F84433A1F12400DB68984794F8D0
:10E4E000913499070AD56FF34103134984F89134A5
:10E4F000D4F84433A1F16C005B68984794F89034E9
:10E50000022B1BD1FFF722F918E000BFE421002005
:10E51000002E00203C2800206C6B0308E021002026
:10E52000803100209831002000320020D0210020CE
:10E5300040320020543200208C32002094F8913474
:10E540009A0640F1C4826FF3451384F89134D4F8ED
:10E550004033002B40F0BB8229B0BDE8F04FFFF7FD
:10E56000ABBA84F84134A3E695F81831012B0CD1ED
:10E5700001F027FD804668B1584601F017FD584666
:10E5800001F019FD042384F88F347EB9012384F847
:10E5900021344FE101F017FD0028F6D0404601F08C
:10E5A00006FD404601F008FD0523ECE73B780593A6
:10E5B0005B09013B062B00F21782DFE813F007002E
:10E5C000150295001502920015020602102EDDD9E3
:10E5D00095F830311297F6B28DF84C60002BD5D1FA
:10E5E0001CA804F03FFA12AA1CA9FF2002F072F93D
:10E5F0009DF85830C3F3030307468DF82C3095F887
:10E60000480095F87D308DF82D3007220BA902F0D7
:10E61000AEFB002F5DD100285BD09DF853309DF8F4
:10E6200052201599C5F8E4101B0443EA02239DF813
:10E63000512002201343C5F8E03004F021FA9DF880
:10E64000583095F8480085F82E71C3F30212C3F3D1
:10E65000030385F8703085F878309DF8593085F8D7
:10E660006920012B38BF01234FF47A725343AB6505
:10E670001344EB650DF15A034FF001081093113E5E
:10E6800094F81B348DF83C300FA985F868808DF81C
:10E69000446002F074FB0223404685F8303101F0FB
:10E6A0004BFE18B14146384601F00CFE94F88F3409
:10E6B000012B00F2A78194F81A34002B40F09A81C4
:10E6C00094F8913443F0100384F89134FEF786FDFA
:10E6D00064E6012001F030FE0028E7D00121072088
:10E6E000E2E7012384F8203495F87D308DF82E3050
:10E6F00094F824348DF82D3095F88C3095F8480036
:10E700000D330BA98DF82C3002F01EFBA6F10D0382
:10E710001BB2099023EAE37300B283423FF736AF9E
:10E720000B2E7FF633AFBA4B25931CA8FF231C9703
:10E730008DF874608DF8983002F0E2F907460028F1
:10E740007FF424AF95F81831012B13D101F039FC77
:10E75000002872D0384601F029FC384601F02BFC25
:10E7600004239DF87C101E9884F88F34C1F30011A7
:10E7700001F041FC9DF87C301E99C4F8341413F06C
:10E780000F0203D09DF89000002862D19DF89800F8
:10E79000002861D0002A7FF4F9AE9DF89020002A6D
:10E7A00014BF4FF003084FF0020800220A92D5F878
:10E7B000EC2095F8E900914251D100284FD0D5F8CE
:10E7C0000C1195F8EAB009680A9195F81811022918
:10E7D00002D1032184F88F14B8F1030F7FF4D6AE71
:10E7E00013F0600F7FF4D2AE0492012795F82E311A
:10E7F000BBF1000F36D0BBF1010F13D1012B33D188
:10E800006FF0090646FA08F606F00106C6F10206A0
:10E81000F6B2BDF87E100AAA304601F0E5FE38B324
:10E82000072823D0012384F821340A9BC4F830340C
:10E83000C4F86C34FEF720FDB0E501F0C4FB0028FD
:10E8400098D0384601F0B3FB384601F0B5FB0523FC
:10E8500087E74FF00008A8E74FF00108A5E74FF061
:10E86000010BC3E70426D4E70326D2E70823DAE73F
:10E870001CAB009304990A9B3246584601F076FF80
:10E8800020B1022814BF0B230A2380E60A9BC4F898
:10E890003034C4F86C349DF87C3084F82104C3F320
:10E8A000401384F82E3484F8443494F88F3484F878
:10E8B0002274012B9EBF0122A86285F81E21012F20
:10E8C000C4F8280484F82C0484F8410438D10222C6
:10E8D00084F8202495F83A20002A4AD19DF87C201B
:10E8E000D60646D4012B94F840149DF87C2005D818
:10E8F000012901D1900601D501F020FCB8F1020FE9
:10E9000094F88F3443D0B8F1030F0AD09DF87C10EF
:10E91000B8F1010F4A4601F00F0120A83BD0FFF7E4
:10E9200045F99DF8903084F82334259BC4F82834A9
:10E930009DF8983084F82C34012384F82D3430E08D
:10E94000059A02F0E002A02A1BD195F82E110122AF
:10E9500085F83A2009B927996963012B84F82024A6
:10E9600007D9D5F89020C4F83C24DAF80020C4F880
:10E97000982495F81821002AB4D1012284F825247E
:10E98000B0E7002285F83A2084F82024A6E79DF815
:10E99000981025984A46FFF709F99DF8903084F8B9
:10E9A00023349DF89020E02A08D195F81F312BB927
:10E9B00084F82324C4F82834A4F82C3494F891342F
:10E9C00043F0020384F8913470E6114D013EB2B277
:10E9D000791C284604F01EF90323A4F82034C4F857
:10E9E000285484F82C64E9E7012384F82134FEF7E5
:10E9F00043FC5BE694F84434002B3FF461AE002006
:10EA0000FEF726FC94F88F34022B3FF45FAE57E6F6
:10EA10003830002094F89134590715D5012001F0C1
:10EA20008BFC60B1012001F05FFC08B984F8180488
:10EA3000D4F8403323F00203C4F8403304E0062046
:10EA400001F07AFC0028F3D194F89134DA077FF5CD
:10EA5000FAAC94F840240AB1032A18D11D4A94F85C
:10EA6000181492F86820914205D29B0723D594F898
:10EA70008F34012B1FD8184806F0A6FCD4F8403379
:10EA800023F02003C4F84033FFF744FBDBE4012A02
:10EA900011D194F81924002A3FF4D5AC0D4A94F80A
:10EAA000181492F868209142E5D29F0703D594F894
:10EAB0004434002BDFD194F8913400206FF3041319
:10EAC00084F8913484F81904FFF746FBBBE429B0BD
:10EAD000BDE8F08F3C280020683100202DE9F04F80
:10EAE00089468DB090460746002800F08F810029A6
:10EAF00000F08C810368002B00F088814368002BB4
:10EB000000F084818368002B00F08081C368002BB3
:10EB100000F07C81104602F013F9002800F07881A3
:10EB2000BD4CBE4D384601F083FB40F2C45200217B
:10EB3000204604F083F840F21C520021284604F0DD
:10EB40007DF8B74BC4F82C3104F50973089304F52C
:10EB50000A7300264046099308A9B24B84F84880FE
:10EB60000A9384F8186184F88C608DF82C6002F0A8
:10EB7000F9F80F2306A994F848008DF8183002F030
:10EB8000E3F8801B18BF01204FF00A0B84F81C012A
:10EB900006A994F848008DF818B002F0D5F84FF0A7
:10EBA000060A84F8DC0006A994F848008DF818A03D
:10EBB00002F0CAF8102384F8DD0006A994F8480092
:10EBC0008DF8183002F0C0F81123C4F89C0006A993
:10EBD00094F848008DF8183002F0B6F81223C4F803
:10EBE000A00006A994F848008DF8183002F0ACF89F
:10EBF0001323C4F8A40006A994F848008DF818302F
:10EC000002F0A2F81423C4F8A80006A994F848005A
:10EC10008DF8183002F098F81623C4F8AC0006A955
:10EC200094F848008DF8183002F08EF8172384F815
:10EC3000B10006A994F848008DF8183002F084F865
:10EC400018230DEB0301C4F8B400C4F8BC0094F819
:10EC500048008DF8183002F077F8C0B21D2384F810
:10EC6000B80084F8C00006A994F848008DF8183060
:10EC700002F06AF81E2384F8C40006A994F848003C
:10EC80008DF8183002F060F81F2384F8C50006A93B
:10EC900094F848008DF8183002F056F82023C4F894
:10ECA000C80006A994F848008DF8183002F04CF816
:10ECB0000B23C4F8CC0006A994F848008DF818304E
:10ECC00002F042F80C2306A9A4F8D00094F84800FA
:10ECD0008DF8183002F038F8D4F89C306365D4F819
:10ECE000A030A365D4F8A430E365D4F8A830236637
:10ECF0004FF00108D4F8AC300590A4F8D200636658
:10ED000084F8B080C4F894B084F898A0C4F84CB0EB
:10ED100084F850A084F8688084F81F81C5F848936F
:10ED2000FEF7AEFDC5F84473C4E90B663E4B84F8AC
:10ED3000198185F89164C5F8408332464FF0FF3160
:10ED4000009605F55A7006F0E1FA384B0096324607
:10ED50004FF0FF3105F5607006F0D8FA344B00969D
:10ED600032464FF0FF3105F5667006F0CFFA02AF7C
:10ED7000304B009632464FF0FF3105F5806006F0CB
:10ED8000C5FA384606F0C2F997E8030004F5927315
:10ED900083E80300284B294F1E60294BC5F84C33EC
:10EDA000284BC5F85433284BC5F85C33274BC5F8BE
:10EDB0005033274BC5F8583305F553703B689847D7
:10EDC00004F5A67003F06AFC20B1112630460DB0A0
:10EDD000BDE8F08F204601F0D7FB0028F5D101F007
:10EDE0000DF9B8B91B4801F021FC06460028ECD10A
:10EDF0007B69984703F0ECFEBB6D94F819019847C6
:10EE0000FB6A9847012385F89234DFE70326DDE7A4
:10EE10000926DBE71326D9E73C280020002E002036
:10EE200000040001E821002059E1000821DA00086F
:10EE300069DA000851D20008E42100206C6B030855
:10EE400011D40008C5D300080DD200089DD30008D6
:10EE500075D300082429002008B5034B0020C3F80F
:10EE60004003FEF7BBF908BD002E002010B5FFF7E8
:10EE7000ABF90A4C60B90A4B93F81831022B02D156
:10EE8000084BDB6A98470123C4F84033002010BDCB
:10EE9000D4F84003013818BF0120F8E7002E002005
:10EEA0003C2800206C6B030838B5124C204606F055
:10EEB0008BFA04F1180006F087FA04F1300006F02E
:10EEC00083FA04F1980006F07FFA01F081F80A4B0A
:10EED0000025DB6A984744F8285CFEF7EDFD0749FA
:10EEE000074840F2C45203F095FE012344F8283C41
:10EEF000284638BD683100206C6B03083C28002090
:10EF00007822002070B52E4B8AB0054693F8DD00BC
:10EF10008DF8090093F8DC008DF80A0029489A6AF8
:10EF200090F81804039200268DF80B0004960C4606
:10EF3000002940D00692D3F8882007921A8F93F8C0
:10EF40001A118DF8151052BAADF8202093F87C20D4
:10EF500093F848308DF8243003AB8DF822008DF8FB
:10EF6000232000930DF10A020DF10B030DF10901AD
:10EF700005A88DF8146000F0A9FF9DF90900FEF7BF
:10EF80004FF9607004A801F0EFF8B0B9049A0F2AA5
:10EF90000DD863789A420AD81544AB42A3EB02011C
:10EFA0002CBF002001202170C0000AB070BD0023DA
:10EFB00023700820F9E70320F7E71320F5E700BFE7
:10EFC0003C280020002E00201FB50446002800F039
:10EFD00010810378412B00F20781DFE813F0420033
:10EFE00049004D005100550059005E000501050122
:10EFF000050105010501050105010501650069001F
:10F000006D0078007F00820085008A0088008C00F7
:10F0100090009300960099009C009F00AE00B20003
:10F02000BA00B600BE00C100C500CE00CA00CC00C8
:10F030000501D200050105010501050105010501D4
:10F040000501050105010501050105010501050190
:10F050000501DA00DE00E200E700EB00EF00F3005C
:10F06000FC00664B93F818312371002004B010BDEA
:10F07000624B93F83031F7E7406803F0ADFCF4E7FA
:10F08000406803F0EFFCF0E75C4B93F81A31EBE7D4
:10F090005A4BD3F8E0306360E7E7584B011D93F813
:10F0A000300103F0F7FCE0E7544B93F81931DBE74C
:10F0B000524B93F88C30D7E71C238DF808304F4B18
:10F0C00002A993F8480001F03FFE6060CDE74C4B89
:10F0D000043493E8030084E80300C6E7494B043492
:10F0E000F7E7494B0434F4E7484B0434F1E71A23BB
:10F0F000E3E71923E1E7414B93F86830B4E73F4B6E
:10F100005B6DC8E73D4B9B6DC5E73C4BDB6DC2E7D4
:10F110003A4B1B6EBFE7394B5B6EBCE702238DF8A1
:10F120000830364B02A993F87C2093F848008DF8FC
:10F130000A2001F009FE207197E7304B93F8DD308B
:10F1400092E72E4B93F839308EE72C4B93F8DC3056
:10F150008AE72A4B93F8383086E7284BDB6C9AE72E
:10F16000264B93F850307FE7244BD3F8843063600C
:10F170007BE7224B8FE7264B8DE7204BD3F8CC3033
:10F18000F5E71E4BD3F82C31436001F06BFEA06015
:10F190006BE71A4BD3F890307DE7184B93F81F318B
:10F1A00062E7164BB3F88830A3805EE7134BB3F8E1
:10F1B0008A30F9E7114BB3F8D030F5E70F4BB3F8CD
:10F1C000D230F1E70D4B93F848200AB1062A12D14C
:10F1D000B3F8A035E8E7094B93F848200AB1062AAE
:10F1E00009D1D3F8A43556E704B0BDE8104000F0CB
:10F1F000F3BE03203AE7182038E700BF3C28002080
:10F20000A8280020F0280020B0280020F82800209E
:10F21000782200207FB5044610B9032004B070BDE9
:10F22000A34DD5F840339A0700F16F820278412A46
:10F2300000F26882DFE812F04200470055005B00F0
:10F240005F00640069007600810087008D009300F4
:10F2500099009F00A500AB00B5006602BA00DC0073
:10F26000EF0016013801290142014B014F01530102
:10F2700057015B0166025F01710199018701AB01D2
:10F28000B101B801BD01C201660228026602660230
:10F29000660266026602660266026602660266022E
:10F2A000660266026602660266026602340239027D
:10F2B0003E02430248024D0252025C020079FEF710
:10F2C00073FA30B1AAE70379022BA6D0794A82F803
:10F2D000303195F8913443F0200385F891340020C3
:10F2E0009CE7406803F06AFB0028F2D095E740688D
:10F2F00003F0A8FBF8E76F4B027983F81A21E8E7DF
:10F300006C4B4268C3F8E020E3E76A4E416896F828
:10F31000300103F0B5FB00287FF47FAF6368C6F8C7
:10F32000E430D6E7416800293FF477AF002001F0D0
:10F33000B1FA0028CDD0112070E7416800293FF4D0
:10F340006CAF0120F3E7416800293FF466AF082065
:10F35000EDE7416800293FF460AF0920E7E7416825
:10F3600000293FF45AAF0C20E1E7416800293FF43F
:10F3700054AF0D20DBE7416800293FF44EAF0E206B
:10F38000D5E7416800293FF448AF0F20CFE74A4C4A
:10F39000484B007983F81901A36D9847E36A9847B1
:10F3A00097E7444B027983F88C2092E7414E037A29
:10F3B0008DF8043096F8480096F87D308DF80530C9
:10F3C000072201A901F0D3FC00283FF426AF6368AF
:10F3D00096F848000193002201A901F0C8FC00281A
:10F3E0003FF41BAF6C36D4E9010186E8030070E7F7
:10F3F000304E037A8DF8043096F8480096F87D3048
:10F400008DF80530072201A901F0B1FC00283FF476
:10F4100004AFB436E7E7274E037A8DF8043096F848
:10F42000480096F87D308DF80530072201A901F0DB
:10F430009EFC00283FF4F1AED4E9010106F174030B
:10F4400083E8030096F81831022B7FF442AF96F858
:10F450003031002B3FF43DAF174BDB6A9847FEF786
:10F4600075F936E7134E037A8DF8043096F84800A4
:10F4700096F87D308DF80530072201A901F077FC60
:10F4800000283FF4CAAEBC36ADE7436802930123BF
:10F490008DF80C30074B02A993F8480001F074FC7A
:10F4A00000287FF416AFB8E6436802930023EFE725
:10F4B000002E00203C2800206C6B030803795A1EA4
:10F4C0000E2A3FF6AAAE934A82F8683001E7914BC4
:10F4D00042685A65FDE68F4B42689A65F9E68D4BA6
:10F4E0004268DA65F5E68B4B42681A66F1E6894BAD
:10F4F00042685A66EDE6874C037994F848008DF827
:10F500000430062201A901F032FC00283FF485AE48
:10F510009DF8043084F8DD30DBE67E4C03798DF80D
:10F52000043094F8480094F87C308DF806300522B9
:10F5300001A901F01CFC00283FF46FAE9DF80430D7
:10F5400084F83930C5E6734C037994F848008DF897
:10F5500004300A2201A901F00AFC00283FF45DAE44
:10F560009DF8043084F8DC30B3E66A4C037994F8F3
:10F5700048008DF80430092201A901F0F8FB0028A9
:10F580003FF44BAE9DF8043084F83830A1E6614B6F
:10F590004268C3F89420DA649BE65E4B027983F8F4
:10F5A000982083F8502094E65A4B4268C3F8842090
:10F5B0008FE6584B4268C3F8CC208AE6012B40F016
:10F5C000A480554C2421204603F03AFB636A9842FC
:10F5D00001D0172022E61C2104F1280003F030FBA3
:10F5E000636C9842F5D14FF4807104F1480003F048
:10F5F00027FBD4F848319842EBD1D42104F5A6700A
:10F6000003F01EFBD4F820329842E2D1002104F529
:10F61000097003F015FBD4F824329842D9D14FF485
:10F62000607104F50A7003F00BFBD4F8A83598421A
:10F63000CFD1142104F2AC5003F002FBD4F8C03552
:10F640009842C6D1334E2146304640F2C45203F0B0
:10F65000E1FA204640F2C452002103F0EFFA95F897
:10F660001B3485F8E833736FC5F8EC3396F87D30BA
:10F6700085F8F83340F20123A5F8FA33274B96F8C2
:10F6800019019B6D984724E68379012B3FF6C5ADA0
:10F69000204B42684068C3F82C2100F091FF48E6F7
:10F6A0001C4B4268C3F8902013E61A4B027983F88A
:10F6B0001F210EE6174B8288A3F8882009E6154B18
:10F6C0008288A3F88A2004E6124B8288A3F8D0200F
:10F6D000FFE5104B8288A3F8D220FAE50D4B93F892
:10F6E00048200AB1062A12D1A288A3F8A025F0E585
:10F6F000084B93F848200AB1062A08D16268C3F87B
:10F70000A425E6E500F06AFCDBE5012086E518208B
:10F7100084E500BF3C280020782200206C6B0308A1
:10F72000DFF880C0F8B5DCF840339B07064635D4D7
:10F730008778002F34D105460FCD1B4C0FC40FCD59
:10F740000FC42B6823609CF89134B16843F0200308
:10F750008CF891343378BBB10D2001F09BF810B1D7
:10F7600011273846F8BD7168B07801F031F90028EA
:10F77000F6D1B2780D4B302101FB02334FF0FF324E
:10F78000D3F80C311A60ECE70E2001F083F8002862
:10F79000E6D1F1680F2001F07DF8E8E70127E0E706
:10F7A0001627DEE7002E0020242900203C28002018
:10F7B000F0B5134FD7F840339B078BB006461AD4E9
:10F7C000D8B9104C94F8E930BBB10146242201A805
:10F7D00001AD03F033FA0FCDE8340FC40FCD0FC4E1
:10F7E0002B68236097F8913443F0200387F8913415
:10F7F00030460BB0F0BD0126FAE71626F8E700BF49
:10F80000002E00203C28002000F00303F7B51C3335
:10F81000294F13701546D7F8402392070C4647D45A
:10F820000A78013A012A03D90325284603B0F0BD1E
:10F8300000283FD1214E96F8E920002A3AD003F063
:10F840000F032B7091F908308DF8043096F84800BA
:10F8500096F87D308DF80530072201A901F087FA6E
:10F8600018B12B7823F004032B70636896F84800D6
:10F870000193002201A901F07AFA18B12B7823F044
:10F8800008032B702D78002DCED194E807000C4B87
:10F8900083E8070097F8912442F0200287F891242A
:10F8A0002278012AC1D1A3F1180000F0A3FBBCE724
:10F8B0000125BAE71625B8E7002E00203C280020D5
:10F8C0003C2900202DE9F04387B00023ADF800303B
:10F8D0000646002800F0EE800361FEF775FC20B1BB
:10F8E0000124204607B0BDE8F08300F067FD002842
:10F8F000F6D100F05DFD014618B96F48142203F0FF
:10F900009DF96E4D95F89134012243F0040385F87A
:10F91000552485F8913433788DF804300021013B6B
:10F920008DF80520ADF806100C2B00F2BB80DFE847
:10F9300003F007B9B9B97982B9B990B9AD9AA900FC
:10F94000D5F8407317F02007CAD196F80480B8F1B3
:10F95000020F46D1DFF868815A4CFDF791FF96F906
:10F96000051098F848003A4601F05BFA88F839002B
:10F97000B37988F83830384607238DF80530FDF71D
:10F9800013FFFF2304F58670A5F80C31C5F8084174
:10F9900085F8047103F066F804F58A7003F01CF82A
:10F9A0003846FDF75BFD0446002839D096F905106E
:10F9B00098F84800012201F034FA88F83900D5F8A7
:10F9C00094343361002C71D000F0F2FC002888D10F
:10F9D00095F8913485F81A0460F3820385F8913420
:10F9E0007FE7B8F1010F4FF00204E8D1DFF8D090C3
:10F9F0008DF8144099F8480089F81D7102A901F0AA
:10FA0000B1F9337989F830318DF805708DF80680B9
:10FA1000FDF7F2FB95F8913443F0100385F891342B
:10FA20000024CCE700226946022000F0F5FA002805
:10FA3000F6D01324C3E7244BB288DB6B96F90C1085
:10FA4000B0689847D5F8403343F00203C5F8403317
:10FA5000E6E702A90D2000F055FB0028E0D00022C7
:10FA600069460D20E1E7164B93F81831D3B9347984
:10FA700004F0070000F0ABFA8DF80040012269465F
:10FA80001020D2E7002269461220CEE78DF8072029
:10FA900000F08EFA044638B900F087FA204600F0EC
:10FAA00089FABDE702248AE7012488E701A800F06B
:10FAB000D3FB16E7032414E754320020002E002065
:10FAC0003C280020022E00206C6B03082DE9F04F2B
:10FAD00099B08046059118B9032019B0BDE8F08FA0
:10FAE00000230361FEF770FB0446002840F0A58068
:10FAF00046460FCE0EAD0FC51422524898F800A00E
:10FB0000B8F80C7098F90EB04F4E214603F096F8F5
:10FB10004E4B012283F8412496F83021022A2546D3
:10FB20000BD196F81821022A07D196F81E2122B986
:10FB3000BAF1010F38BF4FF0010ABAF1010F2BD013
:10FB4000BAF1030F2AD0BAF1000F33D102229DF887
:10FB50003C30DDF84090029362F34715012496F89B
:10FB60007C108DF8321002220CA996F848008DF80E
:10FB7000302001F0E9F896F81A3196F830C196F87D
:10FB80001D1140B2002B63D0BCF1010F57D10029E9
:10FB900055D1002C61D153E00422D8E70023DDF8D1
:10FBA0003C90BDF840709DF942B0029365F01F058E
:10FBB0000124D4E74FF0000BD946CDF808B0CEE7CA
:10FBC0004FF0010084F81A04D2E005F29A420BA922
:10FBD00000F0D6FA002800F015811320049B33872B
:10FBE0001A4B002283F81A2423E105F29A452A468B
:10FBF0000BA900F0C5FA0028EFD10B9B84F828016F
:10FC0000C4F82C5184F83031FCE0B9F1000F00F059
:10FC1000F980002A00F0F6804946E01C02F0FAFF65
:10FC200094F8373201332380ECE01220D6E702202B
:10FC3000D4E70720D4E71320D2E701204DE7FCB931
:10FC40000220F6E0403200203C280020002E002058
:10FC5000002CF5D05845B8BF584696F87C308DF842
:10FC60002000052296F848008DF8223008A901F0FE
:10FC70007EF800283FF430AF9DF8203086F8393008
:10FC80006F4A704BD2F89804D3F8904038B105F021
:10FC900061FB6C4B84423CBF002283F83A20198FF1
:10FCA0001A8F93F830010491996A099152BA002889
:10FCB000BFD093F81B0100B9186393F81801ADF891
:10FCC0005820013893F87C2093F81A411491D0F110
:10FCD000000BD3F888108DF85B204BEB000B93F8EA
:10FCE000482093F83A0093F868308DF85A3009AB01
:10FCF0000093554B03904FF001008DF84C00159187
:10FD00008DF85C20A3F12F01A3F1300213A88DF828
:10FD10004D4000F0DBF8039B4FEA0B1B4BEA431B03
:10FD200000264BEA801B4BEAC413B145444C0393B5
:10FD300008BF37463A46494604F59C70CDE90A6645
:10FD40009B46268084F81A6402F064FFE9B2A5702D
:10FD5000C5F34215FAB2042D3A4E039B84F83722BC
:10FD60003FF42EAF072D3FF450AF022D7FF45FAF6D
:10FD7000364D84F80D110420029984F80401FF2007
:10FD800084F80C0184F8281184F81431D6F8E410B2
:10FD9000C4F8085105F59B730AA8C4F8101184F83B
:10FDA0003021C4F82C3100F013FC00287FF43DAF63
:10FDB0000A9BA4F844040BA8A4F81631C4F84C34E8
:10FDC00000F0D2F900287FF408AF0B9BD3B196F96D
:10FDD0003900FDF725FA94F83732002B3FF405AFD0
:10FDE0000B9B0F2B3FF6F1AE05F58B720BA90F2085
:10FDF00000F0C6F900287FF4F0AE0B9B63F3030B11
:10FE000084F814B10598FDF729FB00287FF4E6AECD
:10FE1000099B86F83A00B36200F082F900287FF46B
:10FE20000AAF94F8913484F840A443F0010384F8B5
:10FE30009134034BD3F89434C8F810304DE600BF2A
:10FE4000002E00203C280020A4280020022E0020A4
:10FE500037B50B4D8DF8040004460F2295F8480085
:10FE600001A900F084FF40B1064A85F81C4192F8D0
:10FE7000913443F0200382F8913403B030BD00BFC9
:10FE80003C280020002E002010B5FEF7EFFF0446AE
:10FE900088B90A4805F098FA094805F095FA094822
:10FEA00005F092FA00F094F8FDF7EAFC064BDB6AE5
:10FEB0009847204610BD0124FBE700BF68310020B1
:10FEC00080310020983100206C6B03082DE9F04F41
:10FED0008BB047780093149B90F90C8090F90D60DB
:10FEE00090F80EB08A464168196004469146002F8A
:10FEF00058D002238DF8103004A9C37B007C8DF804
:10FF0000123000F021FFB4F808C0618943B2606884
:10FF1000984545466144B8BF1D46604534BF00273B
:10FF20000127884209D30A218DF81010207C019303
:10FF300004A900F009FF019B46B2B4F808C060892B
:10FF400061680CEB400E714519D3A1EB0C01B1FBBC
:10FF5000F0FC00FB1C1191B9984503DC2378CBB968
:10FF60004FF0010B21238DF81030207CE37B8DF8BE
:10FF7000115004A98DF8123000F0E6FE45B2009B46
:10FF80008AF80050384689F8006083F800B00BB05A
:10FF9000BDE8F08F0223207C8DF8243006A900F004
:10FFA000E1FEDDE74546EAE7704770477047704776
:10FFB000002070477047704770470020704700204E
:10FFC000704700207047002070470020704770473E
:10FFD0007047704702207047022070470220704728
:10FFE000704700207047704770470020704700201E
:10FFF00070477047704770477047000010B5054C58
:020000040801F1
:100000004FF403722046002102F018FE0020C4E9DC
:10001000000010BD1C3300202DE9F84381469046B6
:1000200000293CD01F4C2023224604F1100012F876
:10003000017F6FBB8242FAD11B4E3368013403B992
:100040003460736803B11C6000252560C4F8088023
:1000500074601FFA88F284F80490601D02F0DAFDE3
:10006000B9F1110F4FF0000398BF104D6373D6F82C
:10007000083298BF25FA09F503F1010398BF05F08E
:10008000010543442573C6F808323846BDE8F883B5
:10009000013B13F0FF030446C6D10227F5E7012711
:1000A000F3E700BF233300201C33002020070200A9
:1000B00010B518B3124A1368984204D1036813604C
:1000C000002305E00B46002BFAD019688842F9D1CD
:1000D0005168884208BF53600BB101681960D2F8BB
:1000E00008328168013B00245B1A04602146C2F893
:1000F0000832102202F0A2FD204610BD0120FCE7CC
:100100001C330020054B1B6813B11A798242FAD1C7
:10011000002B0B600CBF0320002070471C33002015
:1001200010B5054B186800B910BD037B04680BB906
:10013000FFF7BEFF2046F6E71C33002038B5084B1A
:10014000084C186800B938BD03790568112B05D82B
:1001500024FA03F3DB0701D5FFF7AAFF2846F1E7EE
:100160001C3300202007020028B1044BD3F80832CA
:100170000360002070470120704700BF1C3300203F
:100180002DE9F04107460E46154642B339B3154BEB
:100190001C6800232CB93046FFF7E6FF0020BDE8BD
:1001A000F081A268F91A0132914215D32279EA54FA
:1001B000581C22895FFA80F8611D55FA80F002F020
:1001C00029FDA368246898445FFA88F3E2E7204693
:1001D0002568FFF76DFF2C46002CF8D1DBE70120E6
:1001E000DDE700BF1C3300200238C0B211289ABFDF
:1001F000014B185C002070478964030830B50B4B35
:1002000093F820200446084672B100211C3305787B
:10021000A54208D001319842CDB214BF0430103845
:10022000AA42F4D8002030BD1046FCE72835002053
:1002300010B5084C00232060142204F10C00FF21AB
:1002400084F82030C4E9010002F0F8FC012384F8AE
:10025000213010BD2835002010B50E4A92F820102C
:10026000042915D8936804781C7044785C70C478AD
:10027000807898700131DC7082F8201002F11C0146
:100280008B4214BF043302F10C039360012010BDB4
:100290000020FCE728350020094B93F8200068B1C6
:1002A0005A6803F11C018A4200F1FF3014BF043286
:1002B00003F10C0283F820005A600120704700BF50
:1002C0002835002010B5074B93F820200446084637
:1002D00032B15968FFF792FF10B101234470837067
:1002E00010BD00BF2835002008B5064B93F820202C
:1002F0002AB15968FFF782FF08B1407808BD012094
:10030000FCE700BF2835002030B50A4A92F82010DB
:10031000536882F8210061B1916801241C32DD78B4
:10032000587005B99C70934214BF0433103B994236
:10033000F5D130BD2835002008B5044B5968FFF7CA
:100340005DFF003818BF012008BD00BF2835002020
:10035000F7B50422154E044600210DEB020096F875
:10036000207002F06BFC0025EBB29F4201D803B075
:10037000F0BD7368197821705A786270987838B136
:10038000336820469B689847FFF786FF0135EBE707
:10039000DB788DF804108DF805208DF80730FFF715
:1003A0007BFF01A8FFF758FFF0E700BF28350020CA
:1003B000014B93F82000704728350020034B93F839
:1003C0002000042894BF0020012070472835002019
:1003D0001FB50024CDE90244C41F8DF800408DF8FC
:1003E00001100C0AADF80420090C120C8DF8031052
:1003F0008DF806208DF8073002461B0A0121684659
:100400008DF802408DF8083002F073FA002818BF0A
:100410000E2004B010BD2DE9F04188B090460D4685
:100420000F9A0746002847D000240121CDE9044453
:100430008DF810109DF838108DF81510ADF81630A5
:10044000190CCDE900441B0ECDE902448DF819309A
:10045000ADF81A20130C120E07948DF818108DF8B1
:100460001C308DF81D20E3B21E01002DF6B203DC16
:10047000002008B0BDE8F081013310218DF81F3055
:1004800042466B460DEB010002F0C9F90346A8B9DC
:10049000102D28463E44A8BF10206946327811F836
:1004A00001CB013382EA0C02984206F8012BF5DCFD
:1004B000103D2DB20134D6E70920DAE70E20D8E747
:1004C0000138032815D8DFE800F002080C100A4BA9
:1004D0001B681B690B6000207047074B1B685B693A
:1004E000F8E7054B1B689B69F4E7034B1B68DB6966
:1004F000F0E70520704700BF4C3500202DE9F041A2
:10050000C4B00C464A9E17461D468046B8B3B1F5A6
:10051000807F36D84FF488720021684602F08EFB47
:10052000492300934FF48073ADF804302B0C8DF801
:100530000830330CADF80650ADF80A608DF80C3079
:1005400022460023414604A82D0E360E8DF80E30AB
:100550008DF809508DF80D608DF80F4002F05AFBB0
:1005600004F110014B9A3B4689B2684602F041F90A
:1005700010B1012818BF0E2044B0BDE8F081092059
:10058000FAE70D20F8E7000010B590B10A4C2822D8
:100590000021206002F052FB2368084A1A60002004
:1005A0004FF0FF32C3E90302C3E90522C3E9072282
:1005B00010BD0820FCE700BF4C3500200001010100
:1005C000024B1B6818600020704700BF4C350020AC
:1005D00030B1044B1B68DB680133036000207047B7
:1005E000092070474C35002013B500230C460193B9
:1005F000CAB101A9FFF764FF18B9019B591C02D1C8
:10060000146002B010BD99B2611A002901DD5C18B6
:10061000F6E702D113600720F3E71B0C1B0403F578
:1006200080331C44ECE70920EBE7000028B1044BC1
:100630001B681C334362002070470920704700BFCD
:100640004C3500201FB5044600B3002303A80393D4
:1006500002F0A6F9104ABDF80C30126820469380CB
:10066000E38200F0A8FA98B904F118030093216816
:100670000123132202F0B2F860B9204600F09BFA81
:10068000003818BF0120000104B010BD0920FBE7AD
:100690001020F9E70E20F7E74C350020F0B50546AD
:1006A00087B01C4613B9092007B0F0BD2E4E336841
:1006B000DB68834255D894F82020002A0CBF08221A
:1006C0000922834205D3204600F0A9FA68B1102020
:1006D000EAE7002301900093A36894F82810606A69
:1006E000FFF799FE0028EED0DEE723792168B4F801
:1006F00008C0A768043B9AB20029D4D0B2F5807F25
:100700002DD8ADF80EC08DF817304FEA174C04F114
:100710002C033F0E8DF8117000932F0C08234FF01F
:10072000490EADF80C008DF814708DF816002F0EE0
:100730000DEB0300CDF808E08DF810C0ADF81250B5
:100740008DF8157002F04AF808B10E20ACE720468B
:1007500000F065FA0028BAD13368DD60A4E70D2007
:10076000A2E70620A0E700BF4C3500202DE9FF419D
:100770000A9D80460F4616461C46002D5AD000237F
:1007800003A910460393FFF79BFE18B1062004B09F
:10079000BDE8F081039B9C4201D80133F6D1284685
:1007A00000F0AEF9002847D1264B1A78424503D015
:1007B0001A79424542D10120AA68BA4240D103EBDE
:1007C0008002EB6A92F801802979CDE9004304396F
:1007D000927828683B4689B2FFF790FE0028D6D170
:1007E00095F820300194002B4FF00103009314BFC3
:1007F0004246082295F82810686A3B46FFF70BFE30
:100800000028C4D1013E032EC1D8DFE806F002075C
:100810000B0F0D4B1B681C611C62B8E70A4B1B6871
:100820005C61F9E7084B1B689C61F5E7064B1B68A8
:10083000DC61ACE70920AAE70F20A8E70B20A6E7B8
:100840000220A4E7FC0100204C3500201FB50B2935
:100850004FF00003CDE90033CDE902330A4607D05B
:100860000C2914D00A2910D00A2005B05DF804FB29
:10087000012802D120238DF800300021684602F0C3
:1008800038F8002818BF0E20EFE73023F3E70B21DC
:10089000F4E7000038B5054602F026F8044610B12A
:1008A0000E24204638BD002DFBD1094B1B680B21BF
:1008B0009878FFF7CBFF0028F2D10C21FFF7C6FF95
:1008C0000028EDD10A21FFF7C1FF0028E9D0E7E7B2
:1008D0004C3500202DE9F04380468FB00C4617467A
:1008E000002A6BD0002969D0002529461D2206A8C0
:1008F00005951EF097F88DF81350344D2B680DF1C7
:1009000014099E88CDF804900DF1130302933B79EE
:1009100000933B6832462146404602F006F8002824
:100920004ED138683A79494602F074F9384600F0F9
:1009300099F8002846D13C7AFA79BB79240444EA34
:1009400002241C432B689A6894423DD99C609DF810
:1009500013000B21FFF77AFF034658BB0C21FFF76A
:1009600075FF034630BB0A21FFF770FF034608BB43
:100970007B7ABA7AFF7A3F0447EA02271F433A4656
:10098000334621460920FFF723FD034690B933463D
:100990003A4621460820FFF71BFD034650B92A6856
:1009A0009DF8131091700021D1604FF0FF31C2E922
:1009B0000411916118460FB0BDE8F0830923F9E7EF
:1009C0000E23F7E70F23F5E70323F3E74C35002069
:1009D00070B588B000293FD0214C2378834231D0B4
:1009E000237983423AD101220023CDE90133CDE9B5
:1009F000053304EB8204039307930123C1F307201B
:100A0000CDB28DF80030C1F30743090E8DF8020016
:100A10008DF8041002268DF812008DF814106278FB
:100A2000E1788DF8015068468DF803308DF810603C
:100A30008DF811508DF8133001F05BFF20B10E20BE
:100A400008B070BD0022CFE7A278E17804A801F0D9
:100A500050FF0028F4D0F2E70920F1E70B20EFE780
:100A6000FC01002010B50446002845D0016800298B
:100A700042D011F8013B43710322063002F0CAF85C
:100A80002046032250F8091B043102F0C3F8216804
:100A9000CB79E3600A7A43EA0223E3604A7A43EAC5
:100AA0000243E3608A7A43EA0263E360CB7A237409
:100AB0000B7B63742379212B1AD110220D3104F1A1
:100AC000120002F0A7F81D222168501C8B5C6362A3
:100AD000085C43EA0023901C6362085C033243EA2B
:100AE000004363628A5C43EA02636362002010BDD4
:100AF000112B03DC0D22E7E70220F8E70120F6E7DF
:100B000010B50446002854D00168002951D00B7854
:100B100043714B7883608A7843EA02238360CA7802
:100B200043EA024383600A7943EA026383604B79B4
:100B300003738B79C381CA7943EA0223027BC381A1
:100B400002F00F020831103002F064F8237B00221B
:100B500003F00F0384F8202084F82820227903F181
:100B60000800111A04290DDD21680933043AD21A4C
:100B7000085C84F82000D2B2606A84F82820194406
:100B800002F048F8237922681A44002012F8043C45
:100B9000E36212F8031C43EA0123E36212F8021C29
:100BA00043EA0143E36212F8012C43EA0263E36281
:100BB00010BD0220FCE710B5044660B3036853B3D0
:100BC0000279162A29D942791A700146082251F869
:100BD000060B013002F028F82146082251F80E0BCE
:100BE000093002F021F82368E28A5A74E38A226805
:100BF0001B0A93742368A269DA74A36922681B0A2A
:100C000013752368628B5A752368E27E9A751723E1
:100C10002371002010BD0120FCE70220FAE738B55F
:100C20000446002863D00168002960D0037B90F857
:100C3000282003F00F03002A57D10833207904320B
:100C40001344984255D363790B702368A2685A7095
:100C5000A36822681B0A937023686289DA7023688C
:100C6000E27A1A712368227B5A712368E2899A71A9
:100C7000E38922681B0A2146D371227B51F8100BAD
:100C800002F00F02083001F0C5FF237B94F8282002
:100C900003F00F0303F108052AB1226894F820102D
:100CA000515503F10905206894F82820616A284409
:100CB00001F0B0FF94F828302268E16A2B44D15447
:100CC0005A1CE16A206892B2090A81549A1C216870
:100CD000E08D92B28854DA1C216894F82F0092B209
:100CE000043388542371002038BD0933A6E701205E
:100CF000FAE70220F8E70000024B1A881043188038
:100D0000704700BF5035002008B5074B1B883BB12A
:100D1000FEF7ACF8002814BF6FF00200002008BDF9
:100D20006FF00100FBE700BF5035002010B5034B0A
:100D300000241C80FEF790F8204610BD503500209E
:100D4000B0FA80F04009704782B018B9084602B086
:100D500000F0CAB8002002B0704710B9084600F091
:100D600079B9704710B9084600F090B9704703464A
:100D7000084611460BB900F0DDB90020704710B9E4
:100D8000084600F039BD704710B9084600F0FEB9BA
:100D90000020704710B40446084611461A46019BCD
:100DA00014B910BC00F00CBA10BC704703460846DA
:100DB00011460BB900F036BA0020704710B4044653
:100DC000084611461A4614B910BC00F0A3BA002018
:100DD00010BC704730B40546084611461A46DDE996
:100DE00002341DB9029430BC00F022BB002030BC9C
:100DF000704710B9084600F0D3BB0020704710B907
:100E0000084600F037BD0020704710B9084600F0D2
:100E1000E2BB0020704710B9084600F0DFBB00209D
:100E200070470346084611460BB900F0F9BB002095
:100E3000704710B40446084611461A46019B14B97F
:100E400010BC00F0EFBB092010BC704710B4044682
:100E5000084611461A4614B910BC00F02DBDC8B2A0
:100E600010BC70470048704701000102064B10B5E6
:100E70001B6A0446984730B10448054B2044984209
:100E80008CBF0020012010BD6C6B0308403576C973
:100E9000405DC600F0B5114B85B00C4610491F5699
:100EA000054601F017F80F4BE4B25E6A072D4FF0CC
:100EB0000103CDE9024301460AD105220023CDE911
:100EC00000234FF47A727A431846B04705B0F0BD5C
:100ED00008220020CDE900203A46F5E754650308D2
:100EE000346503086C6B03081FB500230093037877
:100EF000013B372B21D8DFE803F01C242020201EE3
:100F0000202020204143454E2055585B5E616420DF
:100F10006C1E6E73787A7D207F832620202020200F
:100F2000202020202020202085878C2020858C20B8
:100F30008E92C3780BB102230093009805B05DF840
:100F400004FB8378F6E743788DF8043007238DF8A7
:100F500005308378003B18BF01235B008DF8063015
:100F600010238DF80730314B1B6801A803F5587228
:100F7000CDE9022300F08EFF0090DEE74023DBE79F
:100F80002023D9E7827890F9013012B9284AD35C3E
:100F9000D2E7284AFBE7827890F90130002AF8D19D
:100FA000254AF4E740F6B833C6E74FF47A73C3E74F
:100FB0004FF4FA63C0E741F28833BDE741F2707342
:100FC000BAE71E484FF47A7101F008FE00F5FA60A6
:100FD000D2E71B4BB0E7154B1B6803F55873ABE723
:100FE000124B1B6803F55B73A6E71023A4E70F4BB6
:100FF0001B68A1E701239FE74FF0834300939CE721
:10100000104BFBE7104B97E740F21113ADF800309F
:1010100093E7032390E790F901300C4AB7E70C49B6
:1010200090F9010000F056FFA6E700BF58350020F8
:101030002B6503081B6503082365030818FCFFFFE5
:1010400000EA06379A99094040F7093754650308C2
:101050003465030837B50B4B02781B680C2101FB84
:1010600002335B7A03EB4304074B1D68036900936B
:10107000C3684278816805EBC40000F0A7FC03B0A8
:1010800030BD00BF583500205435002030B587B042
:10109000027B6423ADF80030012A4FF00003CDE954
:1010A0000133CDE903338DF802308DF8143028D0A8
:1010B000022A2FD01ABB03680BB34368FBB11A4C4A
:1010C00080682360194B18226946186001F0A2FD60
:1010D000174B246893E807000C3384E8070093E873
:1010E000070004F10C05032385E80700A4F86C331E
:1010F000012204F55B7104F5587000F058FC07B04C
:1011000030BD094908684360036100F55B7100F573
:101110005870F2E7044B1B68B3F86023B3F86C1304
:101120000A43A3F86023EAE758350020543500202D
:101130004820030808B503460A2924D8DFE801F04F
:1011400006232323230B161B23212100BDE808407F
:101150000068FFF78BBE90F900009978072271B9FB
:1011600000F0E5FB003818BF012008BD052293F907
:1011700000000021F4E790F900005978EEE7022121
:10118000EEE70722F3E70020EFE7000008B5027959
:101190001AB1012A0BD0002008BD084B01681B685A
:1011A000012203F5587000F002FC0120F4E7034B24
:1011B00001681B6803F55B70F5E700BF5835002038
:1011C000F7B50728144D1C46A8BF072058700E46D7
:1011D0002946174600F07EFE94F90130A070072BD7
:1011E00013D1322000F076FD0C4BDB6D054698479D
:1011F00004F10C0208340346019200943A46314649
:10120000284600F06CFD03B0F0BD054A55F82310E8
:10121000D05C00F057FDE7E7346503086C6B03080A
:10122000546503082DE9F04F344F90F901607B6855
:10123000D0F804908BB004468846984705460028AD
:1012400059D1E37C73B92E4A2378126803EB430328
:10125000990002EB8303D3F80490B9F1000F01D198
:1012600052F80190274B484613F906B0FB6898479F
:10127000A37C2289D7F818A00993072E28D1002330
:101280000121CDE90223204A0693CDE90431CDE9BD
:1012900007330521CDE900214FF47A7202FB0BF2EE
:1012A0004CF250311846D047637C13B3174B995D0D
:1012B0007B6D0D31C9B228469847E07C32464946DD
:1012C00000F01AFE88F8006001200BB0BDE8F08F36
:1012D000002101250823CDE90013CDE90715CDE94B
:1012E0000511CDE903110292A1782B465A462846F2
:1012F000D9E7074BDBE70020E7E700BF6C6B03088B
:10130000583500205465030885450100236503080E
:101310002B6503082DE9F04F8DB090F90130DFF80F
:10132000FCA0DFF8FC90CDE90A123E4A12F903B0A6
:101330000278DAF800300C2505FB02333A4A5B7A72
:10134000126803EB430302EBC303044693F9021054
:1013500090F9020000F0B9FD3449064694F9010005
:1013600000F0B8FDA26861688046304600F0DFFCFE
:101370002178DAF80020D9F80C3069430746505834
:101380009847D9F81C309C4694F901300025072B6A
:101390004FF47A63CDE90753CDE905552DD10123EB
:1013A000CDE903530523CDE901534FF47A7303FBD1
:1013B0000BF300933946434646F2A8122846674687
:1013C000B8472378DAF800200C214B4394F9011038
:1013D000D05800F0B3FDA18994F90100FFF75AFD40
:1013E0000B9B217B1860D9F85430284698470A9BFC
:1013F00001201E700DB0BDE8F08F01200823CDE95B
:101400000350CDE901032A46CDF800B065464346B6
:101410003946A84701200546D3E700BF58350020CC
:101420006C6B0308546503085435002034650308C9
:101430002DE9F04F8FB0002405468A469146984624
:101440000494ADF81440ADF8024007264FF0010BAC
:101450002B7AA34206D9686804A9204400F0CAFB8D
:1014600000285DD102238DF8083002A86B7A8DF830
:101470000A30FFF739FDAB7A8DF81D309DF8113039
:101480008DF81E309DF812308DF81F309DF8103009
:101490008DF82030EB7A8DF821302B7B8DF82230BF
:1014A0006B7B8DF8233010238DF81C608DF8243071
:1014B0003A4E8DF82C000DF102030A93072332688F
:1014C0008DF82D30ADF834302B680C9206930DF169
:1014D000120204AB0DF1110106A800F0A5FB0728CC
:1014E00005460BD130680C22002100F5587001F040
:1014F000A5FB3368BDF80220A3F860239DF81130E6
:101500008AF800309DF8123089F800309DF81030CC
:1015100088F80030189B28461C700FB0BDE8F08F8B
:101520009DF81330BDF81470ADF802702044C4B2B9
:10153000F3B917B3194A00201168072602464FF085
:101540000C0C062B1BD10CFB00FE51F80EE0BEF17B
:10155000000F04D00BFA00F23A4397B20122013097
:101560001028EED1002A3FF473AFADF802706FE798
:101570005A1E042A01D9062BDCD0062668E747FA52
:1015800000FE1EF0010FEAD00CFB00FE51F80EE049
:10159000BEF1000F08BF0626E1E700BF5835002066
:1015A00038B505464068FFF761FC0722841D00211D
:1015B00095F90000E4B200F0BAF908B904F0FD04AE
:1015C00095F901000722002100F0B1F908B904F0F3
:1015D000FB04204638BD00207047000010B503789A
:1015E0000F2B044618D84068FFF740FC22780B49BF
:1015F00002EB42020968831C01EB820051F82220B1
:10160000DBB21AB903F0FD0358B210BD032B06BFBD
:10161000626842600223F7E70020F6E758350020B1
:10162000022070472DE9F0413A4D0446286896B0F3
:101630000E46904600211F460122032300F55870F4
:10164000CDE90411CDE906118DF80C108DF80D10BF
:10165000ADF80E3000F08DF930B92A68B2F8603379
:1016600043F00303A2F860332A68637A8DF82030D0
:1016700002F55871CDE90912274A94F90830126829
:101680000B921022ADF830200DF10E020D9222685F
:101690000E9262680F92D4E90301A27A8DF840207D
:1016A00001228DF8412011AA82E80300227DE18AFF
:1016B0008DF8213018468DF84C20FFF7EBFB08AB76
:1016C00015930DF10D0314900093CDF8048003AB36
:1016D00004AA39460EA800F099FB044678B99DF893
:1016E0000C10013901F07AFA00F158030DEB0300F8
:1016F00010F8483C3370204616B0BDE8F0810C2845
:1017000001BF2A68B2F8603343F00303A2F86033E4
:10171000F1E700BF5835002054350020F8B50679B0
:10172000012E054648D90F2E48D80368187A40F391
:1017300003000722002140B200F0F9F82B680446AC
:10174000187A40F303100722002140B200F0EFF8AE
:10175000B8B1B4FA84F4640929680B7A086843F3D1
:10176000030243F303135BB252B29A42C8BF01248F
:10177000FFF77CFB80F00103DBB224B10533D8B264
:10178000F8BD0124E8E7DBB90E4F29683B6806EB9A
:10179000460003EB80000C2201F03CFA3A680C236F
:1017A00003FB062320465C72B2F860130123B340AA
:1017B0000B43A2F86033E3E70620E1E70320DFE70D
:1017C0000420DDE75835002010B4017801290ED936
:1017D000084B18680C234B43C4180022C250C4E9BC
:1017E000012200F5587010BC102200F0A9B80020AA
:1017F00010BC7047583500202DE9F04186B05023C9
:101800008DF81430037A102B074630D14368DD7B06
:101810006DBB0224A8466426062C14D87A68535D52
:1018200003932A44517843EA01230393927843EACD
:1018300002437343CDE9033863B968468DF800402D
:10184000FFF7C2FF0DE0CDF80C808DF81480CDF8C5
:101850001080F2E703AB01A801938DF80840FFF771
:101860005DFF0134E4B2102C05F10305D4D106B0BC
:10187000BDE8F0811FB502680379116849B901A874
:101880008DF80430FFF7A0FF78B1032005B05DF8B4
:1018900004FB02A802928DF80C30FFF73FFF0428EA
:1018A00005D0052805D00028EFD00020EEE7022063
:1018B000ECE70120EAE70000C90020B9034B0B4424
:1018C0009856C0B27047024BF9E700BFDB640308CB
:1018D0009B640308F0B59A42069D03DB9DF9143022
:1018E0009A4220DD0020F0BD03EB430331F814C021
:1018F00005EB830300264CFA06F7FF0707D51F7A8E
:1019000007F00F0E964502DCB2EB171F0DDD013616
:10191000102E03F10C03EED10134E4B22301DBB24B
:101920009842E1D8DEE70024F8E70120DBE78842AF
:1019300004DB9042CCBF002001207047002070479C
:1019400010B51409B4EB111F03464FEA11100ED362
:1019500091420CD202B201F00F0133F81240012083
:1019600000FA01F124EA010123F8121010BD002051
:10197000FCE7F0B528B100EB4105012700209142BA
:1019800000D3F0BD002435F802CB234607FA04F655
:1019900036EA0C0608BF013304F1010408BFDBB2CC
:1019A000102CF3D118440131C0B2C9B2E7E710B529
:1019B00000B149B910BD31F8134020F8134001338C
:1019C000DCB2A242F7D8F5E70023F9E782B030B5E0
:1019D00004880493D2B9B3F5616F15D349F6AF25E6
:1019E00042F21072AB4298BF4FF47A72944238BF01
:1019F00014466143BDE83040C3688B428CBF5B1A1C
:101A00000023C36002B070476422EFE7012C38BFA7
:101A10000124EEE72DE9F04F8FB01546199F03938F
:101A20009DF8603007930C46804603F089FC6A4AB3
:101A30000590A7F5F633303BB3FBF2F3534303F5C0
:101A4000F63B0493182313FB05430BF1300B06936D
:101A500000254FF0FF3A069B9C4207D1002D14BF92
:101A600050464FF0FF300FB0BDE8F08FBDF9683041
:101A7000ADF82430099919973846089703F05CFBB4
:101A80002688B8F1000F5FD1B7F5616F5AD349F6D8
:101A9000AF2242F21073974298BF4FF47A739E427E
:101AA00038BF1E46642E59D1DFF83091A060A1687E
:101AB0000CA803F063FB0D9B0093DDE908120C9B5F
:101AC0000AA803F0B9FA039A0A9B0AB9079A2AB13D
:101AD00022694A4502D1424A93420ED9414BC4F889
:101AE0000C909F4209D90023ADF82C300B99CDF80A
:101AF00028B0584603F020FBA060606808B9C4F81D
:101B00000C90C4F81090B8F1000F04D003F022FC40
:101B1000E3680344E360D4E903329342059B88BF42
:101B2000E26063601B9BE1687343994204D20398AF
:101B3000E8B9B8F1000F1AD001231D442375EDB2A6
:101B4000183488E76423AAE7039B0BB9234BE360AF
:101B5000012EDFF8889038BF0126CEE7B6F57A7FF0
:101B60000ABFDFF88490DFF88490A0609FE7002030
:101B70009342207506D85B1A9A4505F1010528BFE6
:101B80009A46EDB2B8F1000FDAD1642E184AADF8DA
:101B90002C801DD049F6B023B6F57A7F18BF1346C6
:101BA000974281BF049A02F5A83202F5C0729B18D1
:101BB0000A931A9B00930AAE96E80600199B3046DA
:101BC00003F03AFA96E8030003F0B6FA8246B7E764
:101BD0004FF46163E4E700BF8051010040771B00D0
:101BE0007F5101002FEC010080A81201002E93020A
:101BF00030EC01000378032B14D1437803F00F027B
:101C00001B098A704B7083788B80C27843EA022369
